:02000004700288
:10000000464346420004015600000000010303007D
:1000100000000000000000000000000000000000E0
:1000200000000000000000000000000000000000D0
:1000300000000000000000000000000000000000C0
:100040001000000001040700000000000000000094
:100050000000400000000000000000000000000060
:100060000000000000000000000000000000000090
:100070000000000000000000000000000000000080
:10008000EB04180A063204260000000000000000FD
:10009000050404240000000000000000000000002F
:1000A0000000000000000000000000000000000050
:1000B0000604000000000000000000000000000036
:1000C0000000000000000000000000000000000030
:1000D00020041808000000000000000000000000DC
:1000E0000000000000000000000000000000000010
:1000F0000000000000000000000000000000000000
:10010000D8041808000000000000000000000000F3
:100110000204180804200000000000000000000095
:1001200000000000000000000000000000000000CF
:10013000600400000000000000000000000000005B
:1001400000000000000000000000000000000000AF
:10015000000000000000000000000000000000009F
:10016000000000000000000000000000000000008F
:10017000000000000000000000000000000000007F
:10018000000000000000000000000000000000006F
:10019000000000000000000000000000000000005F
:1001A000000000000000000000000000000000004F
:1001B000000000000000000000000000000000003F
:1001C000000100000010000001000000000000001D
:1001D000000001000000000000000000000000001E
:1001E000000000000000000000000000000000000F
:1001F00000000000000000000000000000000000FF
:10100000D10020410020027000000000000000001C
:1010100020100270001002700000000000000000AC
:10102000000000700000400000000000FFFFFFFF14
:1020000000002C207D2402700D2502701125027025
:1020100009250270092502700925027000000000E0
:1020200000000000000000000000000061300270AD
:10203000092502700000000091300270A16A027050
:102040002125027025250270292502702D25027098
:102050003125027035250270392502703D25027048
:102060004125027045250270492502704D250270F8
:102070005125027055250270592502705D250270A8
:102080006125027009250270092502700925027078
:10209000CF970C70DD970C706D250270EB970C706C
:1020A000F9970C7007980C7015980C7023980C70A9
:1020B00085250270892502708D2502709125027098
:1020C00095250270992502709D250270A125027048
:1020D000A5250270A9250270092502700925027044
:1020E00009250270092502708143067009250270D6
:1020F0000925027009250270092502700925027060
:10210000092502700925027009250270092502704F
:10211000092502700925027009250270092502703F
:10212000AD250270B1250270B5250270B925027087
:10213000BD2502700925027009250270092502706B
:10214000092502700925027009250270092502700F
:1021500009250270092502700925027009250270FF
:1021600009250270092502700925027009250270EF
:1021700009250270092502700925027009250270DF
:10218000C1430670092502700925027009250270F5
:1021900009250270092502700925027009250270BF
:1021A0000925027009250270C1250270C52502703B
:1021B000092502700925027009250270092502709F
:1021C000092502700925027009250270092502708F
:1021D000092502705943067009250270092502700D
:1021E000092502700925027009250270C9250270AF
:1021F000CD25027009250270D1250270D525027007
:102200000925027009250270D9250270DD250270AA
:10221000092502700925027009250270092502703E
:10222000092502700925027009250270092502702E
:10223000092502700925027009250270092502701E
:10224000092502700925027009250270092502700E
:1022500009250270092502700925027009250270FE
:1022600009250270092502700925027009250270EE
:1022700009250270092502700925027009250270DE
:1022800009250270092502700925027009250270CE
:1022900009250270092502700925027009250270BE
:1022A000E1250270E5250270E9250270092502701A
:1022B000ED250270092502700925027009250270BA
:1022C000092502700925027009250270092502708E
:1022D000092502700925027009250270092502707E
:1022E000092502700925027009250270092502706E
:1022F000092502700925027009250270092502705E
:10230000092502700925027009250270092502704D
:10231000092502700925027009250270092502703D
:10232000092502700925027009250270092502702D
:10233000092502700925027009250270092502701D
:10234000092502700925027009250270092502700D
:1023500009250270092502700925027009250270FD
:1023600009250270092502700925027009250270ED
:1023700009250270092502700925027009250270DD
:1023800009250270092502700925027009250270CD
:1023900009250270092502700925027009250270BD
:1023A00009250270092502700925027009250270AD
:1023B000092502700925027009250270092502709D
:1023C000092502700925027009250270092502708D
:1023D000092502700925027009250270092502707D
:1023E000092502700925027009250270092502706D
:1023F000092502700925027009250270FFFFFFFF01
:10240000A3F5803A704700BF174B002B08BF134B52
:102410009D46FFF7F5FF00218B460F461348144AEF
:10242000121A3DF1FBFB0E4B002B00D098470D4BD1
:10243000002B00D098470020002104000D000D481B
:10244000002802D00C483CF1C8FB3BF11FFC2000E7
:1024500029001EF0B9FE3BF139FB00BF0000080067
:10246000000000000000000000002C202854038021
:10247000405E3580DBEB15700000000072B6164838
:10248000164901600A6882F3088815488047154993
:10249000154A164B9A42BEBF51F8040B42F8040B82
:1024A000F8E7134A134B9A42BEBF51F8040B42F8A7
:1024B000040BF8E7104B00209A42BCBF42F8040B13
:1024C000FAE70E490E4A00209142BCBF41F8040BC6
:1024D000FAE762B60B48804708ED00E00020027082
:1024E000B165027058473370B89402802854038055
:1024F0000000C0810000C0810098FA812854038048
:10250000405E358009240270FFF7FEBF384800475F
:10251000384800473848004738480047384800479F
:10252000384800473848004738480047384800478F
:10253000384800473848004738480047384800477F
:10254000384800473848004738480047384800476F
:10255000384800473848004738480047384800475F
:10256000384800473848004738480047384800474F
:10257000384800473848004738480047384800473F
:10258000384800473848004738480047384800472F
:10259000384800473848004738480047384800471F
:1025A000384800473848004738480047384800470F
:1025B00038480047384800473848004738480047FF
:1025C00038480047384800473848004738480047EF
:1025D00038480047384800473848004738480047DF
:1025E00038480047384800473848004738480047CF
:1025F0000D25027011250270613002709130027059
:10260000A16A02700925027009250270092502706D
:10261000092502700925027009250270092502703A
:10262000092502700925027009250270092502702A
:10263000092502700925027009250270092502701A
:10264000092502700925027031980C7045980C70AC
:1026500059980C706D980C7081980C7095980C704E
:10266000A9980C70BD980C70214F0C702D4F0C70F8
:10267000394F0C70454F0C70514F0C705D4F0C7002
:10268000694F0C70754F0C7085960C70A5960C7088
:1026900009250270092502700925027009250270BA
:1026A00009250270092502700925027009250270AA
:1026B000092502700925027009250270092502709A
:1026C000092502700925027009250270C5960C7053
:1026D00009250270EC46A0E8F05F80EC108B4FF00B
:1026E00000007047B0E8F05FE54690EC108B080002
:1026F00008BF0120704700BF10F8012B11F8013B03
:10270000012A28BF9A42F7D0D01A70470000000073
:1027100001F0FF01102A2BDB10F0070F08D010F892
:10272000013B013A8B422DD010F0070F42B3F6D196
:10273000F0B441EA012141EA014122F007047FF0AF
:1027400000070023F0E80256083C85EA010586EA06
:10275000010685FA47F5A3FA87F586FA47F6A5FA42
:1027600087F68EB9EED1F0BC01F0FF0102F007024E
:1027700032B110F8013B013A83EA010313B1F8D1F9
:102780000020704701387047002D06BF35460338DA
:10279000073815F0010F07D1013015F4807F02BF13
:1027A000013015F4C03F0130F0BC0138704700BF64
:1027B000034613F8012B002AFBD1181A0138704781
:1027C00081F0004102E000BF83F0004330B54FEAE2
:1027D00041044FEA430594EA050F08BF90EA020F4F
:1027E0001FBF54EA000C55EA020C7FEA645C7FEAE2
:1027F000655C00F0E2804FEA5454D4EB5555B8BF05
:102800006D420CDD2C4480EA020281EA030382EA75
:10281000000083EA010180EA020281EA0303362D07
:1028200088BF30BD11F0004F4FEA01314FF4801CDA
:102830004CEA113102D0404261EB410113F0004FEC
:102840004FEA03334CEA133302D0524263EB4303A3
:1028500094EA050F00F0A780A4F10104D5F1200E41
:102860000DDB02FA0EFC22FA05F2801841F100019C
:1028700003FA0EF2801843FA05F359410EE0A5F170
:1028800020050EF1200E012A03FA0EFC28BF4CF0A1
:10289000020C43FA05F3C01851EBE37101F0004557
:1028A00007D54FF0000EDCF1000C7EEB00006EEB64
:1028B0000101B1F5801F1BD3B1F5001F0CD34908EE
:1028C0005FEA30004FEA3C0C04F101044FEA445245
:1028D00012F5800F80F09A80BCF1004F08BF5FEACC
:1028E000500C50F1000041EB045141EA050130BDAC
:1028F0005FEA4C0C404141EB0101013C28BFB1F5BE
:10290000801FE9D291F0000F04BF01460020B1FA08
:1029100081F308BF2033A3F10B03B3F120020CDADB
:102920000C3208DD02F1140CC2F10C0201FA0CF0B9
:1029300021FA02F10CE002F11402D8BFC2F1200C1E
:1029400001FA02F120FA0CFCDCBF41EA0C019040D4
:10295000E41AA2BF01EB0451294330BD6FEA04041D
:102960001F3C1CDA0C340EDC04F11404C4F1200208
:1029700020FA04F001FA02F340EA030021FA04F31A
:1029800045EA030130BDC4F10C04C4F1200220FA71
:1029900002F001FA04F340EA0300294630BD21FAAF
:1029A00004F0294630BD94F0000F83F4801306BF75
:1029B00081F480110134013D4EE77FEA645C18BF69
:1029C0007FEA655C29D094EA050F08BF90EA020F00
:1029D00005D054EA000C04BF1946104630BD91EAF8
:1029E000030F1EBF0021002030BD5FEA545C05D1FB
:1029F0004000494128BF41F0004130BD14F580043A
:102A00003CBF01F5801130BD01F0004545F0FE41AD
:102A100041F470014FF0000030BD7FEA645C1ABFE2
:102A2000194610467FEA655C1CBF0B46024650EA19
:102A3000013406BF52EA033591EA030F41F4002145
:102A400030BD00BF90F0000F04BF0021704730B5CB
:102A50004FF4806404F132044FF000054FF00001A0
:102A600050E700BF90F0000F04BF0021704730B561
:102A70004FF4806404F1320410F0004548BF404236
:102A80004FF000013EE700BF42004FEAE2014FEA8B
:102A900031014FEA02701FBF12F07F4393F07F4F66
:102AA00081F06051704732F07F4208BF704793F069
:102AB0007F4F04BF41F40021704730B54FF460747C
:102AC00001F0004521F000411CE700BF50EA01027F
:102AD00008BF704730B54FF000050AE050EA010228
:102AE00008BF704730B511F0004502D5404261EB98
:102AF00041014FF4806404F132045FEA915C3FF4D9
:102B0000D8AE4FF003025FEADC0C18BF03325FEA75
:102B1000DC0C18BF033202EBDC02C2F1200300FA26
:102B200003FC20FA02F001FA03FE40EA0E0021FA4B
:102B300002F11444BDE600BF80F0004002E000BF97
:102B400081F0004142001FBF5FEA410392EA030F98
:102B50007FEA226C7FEA236C6AD04FEA1262D2EBE2
:102B60001363C1BFD218414048404140B8BF5B42E7
:102B7000192B88BF704710F0004F40F4000020F080
:102B80007F4018BF404211F0004F41F4000121F096
:102B90007F4118BF494292EA030F3FD0A2F10102E0
:102BA00041FA03FC10EB0C00C3F1200301FA03F11E
:102BB00000F0004302D5494260EB4000B0F5000F41
:102BC00013D3B0F1807F06D340084FEA310102F100
:102BD0000102FE2A51D2B1F1004F40EBC25008BFB2
:102BE00020F0010040EA03007047490040EB00007C
:102BF000013A28BFB0F5000FEDD2B0FA80FCACF17D
:102C0000080CB2EB0C0200FA0CF0AABF00EBC250A9
:102C100052421843BCBFD0401843704792F0000F97
:102C200081F4000106BF80F400000132013BB5E7EA
:102C30004FEA41037FEA226C18BF7FEA236C21D060
:102C400092EA030F04D092F0000F08BF08467047C5
:102C500090EA010F1CBF0020704712F07F4F04D193
:102C6000400028BF40F00040704712F100723CBFA6
:102C700000F50000704700F0004343F0FE4040F4D0
:102C8000000070477FEA226216BF08467FEA23638E
:102C90000146420206BF5FEA412390EA010F40F479
:102CA000800070474FF0000304E000BF10F00043C5
:102CB00048BF40425FEA000C08BF704743F09643AC
:102CC00001464FF000001CE050EA010208BF7047C7
:102CD0004FF000030AE000BF50EA010208BF70474E
:102CE00011F0004302D5404261EB41015FEA010C63
:102CF00002BF84460146002043F0B64308BFA3F15B
:102D00008053A3F50003BCFA8CF2083AA3EBC2533C
:102D100010DB01FA02FC634400FA02FCC2F120025B
:102D2000BCF1004F20FA02F243EB020008BF20F092
:102D30000100704702F1200201FA02FCC2F12002F8
:102D400050EA4C0021FA02F243EB020008BF20EAED
:102D5000DC7070477BB972B90029BEBF00204FF00C
:102D6000004106E008BF00281CBF6FF000414FF093
:102D7000FF3000F02DB9ADF1080C6DE904CE00294B
:102D800009DB002B1ADB3EF1C7FCDDF804E0DDE9CE
:102D9000022304B07047404261EB4101002B1BDB72
:102DA0003EF1BAFCDDF804E0DDE9022304B0404264
:102DB00061EB4101524263EB43037047524263EBC4
:102DC00043033EF1A9FCDDF804E0DDE9022304B091
:102DD000404261EB41017047524263EB43033EF1D5
:102DE0009BFCDDF804E0DDE9022304B0524263EB12
:102DF0004303704753B94AB9002908BF00281CBFD4
:102E00004FF0FF314FF0FF3000F0E2B8ADF1080CA9
:102E10006DE904CE3EF180FCDDF804E0DDE902233B
:102E200004B0704700F1340191E838009C46A64692
:102E30004CF8045D90E8FF0FE54600BD90EC210BD7
:102E4000704700BF80EC210B704700BF90EC200B57
:102E5000704700BF80EC200B704700BFD0EC200B08
:102E6000704700BFC0EC200B704700BFF0EC0201C0
:102E7000F0EC0211F0EC0221F0EC0231F0EC024136
:102E8000F0EC0251F0EC0261F0EC0271F0EC028126
:102E9000F0EC0291F0EC02A1F0EC02B1F0EC02C116
:102EA000F0EC02D1F0EC02E1F0EC02F1704700BF6F
:102EB000E0EC0201E0EC0211E0EC0221E0EC023176
:102EC000E0EC0241E0EC0251E0EC0261E0EC027166
:102ED000E0EC0281E0EC0291E0EC02A1E0EC02B156
:102EE000E0EC02C1E0EC02D1E0EC02E1E0EC02F146
:102EF000704700BFB0FC0181B0FC0191B0FC01A1A2
:102F0000B0FC01B1704700BFA0FC0181A0FC0191A1
:102F1000A0FC01A1A0FC01B1704700BFEC4600B5C8
:102F20002DE900502DE9FF1F4FF000032DE90C00A3
:102F300001A93EF1A3FEDDF840E012B0704700BFEA
:102F4000EC4600B52DE900502DE9FF1F4FF00003BE
:102F50002DE90C0001A93EF1CDFEDDF840E012B0F4
:102F6000704700BFEC4600B52DE900502DE9FF1F6A
:102F70004FF000032DE90C0001A93EF1DBFEDDF866
:102F800040E012B0704700BFEC4600B52DE900509C
:102F90002DE9FF1F4FF000032DE90C0001AB3EF1BE
:102FA000A1FEDDF840E012B0704700BFEC4600B56E
:102FB0002DE900502DE9FF1F4FF000032DE90C0013
:102FC00001AA3EF10BFFDDF840E012B0704700BFF0
:102FD000704700BF0348044B834202D0034B03B148
:102FE00018477047285403802854038000000000CD
:102FF0000548064B1B1AD90F01EBA301491002D05B
:10300000034B03B1184770472854038028540380AA
:103010000000000010B5064C237843B9FFF7DAFF33
:10302000044B13B10448AFF300800123237010BD9B
:1030300028540380000000001C4B197008B5054B94
:103040001BB105490548AFF30080BDE80840FFF714
:10305000CFBF00BF000000002C5403801C4B197030
:10306000074B19680868B0E8F04F80F30988BFF390
:103070006F8F4FF0000080F311887047AFF300802E
:1030800098550380000000000000000000000000D0
:10309000EFF30980BFF36F8F154B1A681EF0100F06
:1030A00008BF20ED108A20E9F04F10602DE90900DB
:1030B0004FF0200080F31188BFF34F8FBFF36F8F65
:1030C00003F0A2FC4FF0000080F3118809BC1968DE
:1030D0000868B0E8F04F1EF0100F08BFB0EC108A7F
:1030E00080F30988BFF36F8F704700BFAFF3008094
:1030F00098550380064A13681968064B19B94FF0B2
:10310000FF321A6070471268D2681268F9E700BF90
:10311000DC540380D45403802DE9F84F584B1B68CE
:10312000002B40F0A680574B1C6801341C60BCB9D2
:10313000554B1A68126842B14FF0200383F311888F
:10314000BFF36F8FBFF34F8FFEE7504A19681068C7
:10315000186011604E4A136801331360FFF7CAFF0D
:103160004C4D00204C4A2B68DFF83CC19C4211D2E8
:10317000DCF800301421DB6A4B43D358022B474B59
:103180001B6828BF0120464B1B68002B18BF01207D
:10319000BDE8F88F3C4F434E3B681B681BB94FF0AE
:1031A000FF332B60E4E73B68DB68DB6859688C42DF
:1031B00001D22960DCE7D3F8148003F1040ED3E9CF
:1031C0000219C1F80890C9F80410D8F80410714524
:1031D0004FF0000108BFC8F804905961D8F80010FA
:1031E0000139C8F80010D3F82880B8F1000F15D0C5
:1031F00003F1180AD3E90719C1F80890C9F80410B7
:10320000D8F8041051454FF0000108BFC8F80490E9
:103210009962D8F800100139C8F80010D96A4FF047
:103220000108D6F8009008FA01F848EA0908C6F83B
:1032300000804FF0140808FB01F802EB080ADAF8E6
:103240000490D9F808B0C3F80890C3F80CB0CBF8D4
:1032500004E0C9F808E0C3F814A052F808300133BC
:1032600042F80830DCF80030DB6A994288BF012060
:1032700092E70A4A002013680133136088E700BF11
:1032800014550380DC550380DC540380D85403803C
:10329000E0550380D45403801C550380E054038020
:1032A00018550380945503809855038030B50C68F9
:1032B000631C0AD103695A684A6091608B60596047
:1032C000036808610133036030BD00F10802134652
:1032D00052681568A542FAD9EDE70000914208B599
:1032E000416000610AD8D21A83699A420DD2011D49
:1032F000074B1868FFF7DAFF002008BD9A4201D299
:10330000994202D2011D034BF3E70120F5E700BF0C
:10331000AC540380B854038070B50B46044616467F
:10332000A569324620461D442946FFF7D7FF00B95C
:1033300070BD236A204698472B46F1E770477047D7
:10334000012070470020704701207047704738B552
:103350000D46046B04B938BD2368204629469B6896
:103360009847A468F6E738B50D46046B04B938BD34
:10337000236820462946DB689847A468F6E738B5F5
:103380000D46046B04B938BD2368204629461B69E5
:103390009847A468F6E738B50D46046B04B938BD04
:1033A0002368204629465B699847A468F6E7002011
:1033B0007047F8B50E461746046B00250CB9284631
:1033C000F8BD236820463A4631469B699847A46871
:1033D000002818BF0546F1E7D0E90303184770B588
:1033E00004460D4622F043FFA36B4BB1013D012D76
:1033F00006D86168204621F00301BDE870401847F7
:1034000070BD036B37B504460D4633B91A46042127
:103410004FF48070009333F009F9246B0CB903B0BA
:1034200030BD2368204629465B6A9847A468F5E7C3
:1034300013B5094C236863B19B68A34206D00023EF
:10344000882149201A46009333F0F0F823680022BF
:103450009A6002B010BD00BF7854038013B5094CC8
:10346000236863B19B68A34206D0002388214920CA
:103470001A46009333F0DAF8236800229A6002B00B
:1034800010BD00BF7454038010B504465030F5F0F1
:10349000ABF804F14800F5F0A7F804F14000F5F0AE
:1034A000A3F804F13800F5F09FF8034B20462360A1
:1034B000F5F00CF9204610BDC05B167010B504463F
:1034C0006030F5F091F804F15800F5F08DF804F152
:1034D0004800F5F089F804F13800F5F085F8034B61
:1034E00020462360F5F0F2F8204610BDC05B167050
:1034F000034B10B504460360F5F0E8F8204610BD14
:10350000BC57167010B50446FFF7D8FF7821204647
:1035100035F16EFA204610BD10B50446FFF7E8FFFE
:10352000F821204635F164FA204610BD10B5044656
:10353000FFF7AAFF6821204635F15AFA204610BD50
:10354000054B10B5044640F8903BECF035FE2046A4
:10355000F3F0B6FE204610BD145B167010B504469D
:10356000FFF7EEFFA021204635F142FA204610BDBC
:10357000054B10B5044640F89C3BF5F035F8204665
:10358000FFF7DEFF204610BD3C52167010B5044612
:10359000FFF7EEFFA821204635F12AFA204610BD9C
:1035A00010B504460830F4F051F9204610BD10B5AE
:1035B00004461830F5F018F82046FFF7F1FF2046D2
:1035C00010BD10B504462830F5F00EF82046FFF780
:1035D000EEFF204610BD10B504463830F5F004F873
:1035E0002046FFF7EEFF204610BD10B50446FFF75A
:1035F000F2FF4021204635F1FBF9204610BD0000C6
:10360000074B10B5044640F8803BF4F01FF904F175
:103610007800F4F0E9FF2046FFF750FF204610BD88
:103620001C5A167010B50446FFF7EAFF9021204699
:1036300035F1DEF9204610BD10B504464030F4F0F7
:1036400005F904F13000F4F0CFFF04F12000F4F0AC
:10365000CBFF04F11000F4F0C7FF204610BD10B5F9
:103660000446FFF7E9FF5021204635F1C1F9204615
:1036700010BD10B504463030F4F0E8F804F1200035
:10368000F4F0B2FF04F11000F4F0AEFF204610BDDC
:1036900010B50446FFF7EDFF4021204635F1A8F9AB
:1036A000204610BD10B504465030F4F0CFF804F1B8
:1036B0004000F4F099FF04F13000F4F095FF04F1BC
:1036C0002000F4F091FF04F11000F4F08DFF20468B
:1036D00010BD10B50446FFF7E5FF6021204635F127
:1036E00087F9204610BD0000144B10B50446036056
:1036F00000F58470F4F0AAF804F1C000FFF76BFF46
:1037000004F1B800F4F070FF04F1B000F4F06CFFC5
:1037100004F1A800F4F068FF04F19C00ECF04CFD0B
:1037200004F1940024F068FD04F19000F4F05CFFD3
:103730002046F3F0C5FD204610BD00BF885B167023
:1037400010B50446FFF7D0FF4FF48C71204635F1D9
:103750004FF9204610BD0000064B10B5044603602B
:1037600000F58A70F4F040FF2046FFF7BDFF2046C9
:1037700010BD00BF685A167010B50446FFF7ECFF85
:103780004FF49071204635F133F9204610BD00000A
:10379000084B10B50446036000F59470F4F024FF64
:1037A00004F58C70F4F020FF2046FFF79DFF2046C3
:1037B00010BD00BF1C4C167010B50446FFF7E8FFA3
:1037C0004FF49C71204635F113F9204610BD0000DE
:1037D000084B10B50446036000F59470F4F004FF44
:1037E00004F58C70F4F000FF2046FFF77DFF2046C3
:1037F00010BD00BFE44B167010B50446FFF7E8FF9C
:103800004FF49C71204635F1F3F8204610BD0000BE
:10381000114B10B5044640F8BC3BECF0CDFC04F174
:10382000B400F4F0E1FE04F1AC00F4F0DDFE04F1CC
:10383000A400F4F0D9FE04F19C00F4F0D5FE04F1EC
:10384000940024F0D9FC04F19000F4F0CDFE204661
:10385000F3F036FD204610BD4C57167010B50446E7
:10386000FFF7D6FFC821204635F1C2F8204610BD2B
:10387000054B10B5044640F8303BF4F014FC2046EC
:10388000F4F024FF204610BD4C5B1670034B10B5BE
:1038900004460360FFF7ECFF204610BDA05A1670E7
:1038A00010B50446FFF7F2FF3C21204635F1A0F8A1
:1038B000204610BD00F5A0738B4201D126F088BAD6
:1038C000184625F0B9BF0000154B10B5044640F866
:1038D000F03BF3F0BBFF04F1E800F4F085FE04F1E7
:1038E000E000F4F081FE04F1C000F7F023FE04F1E3
:1038F000B000F4F079FED4F8AC3004F190003BB1A4
:10390000084A126822B100225A610122064B1A703D
:10391000ECF052FC2046F3F0D3FC204610BD00BF73
:10392000B8581670485403804454038010B50446B8
:10393000FFF7CAFF4FF48071204635F159F8204651
:1039400010BD0000224B10B50446036000F5D8708E
:10395000F3F07CFF04F5B470FFF73DFE04F5AE70A4
:10396000F4F042FE04F5AA70F4F03EFE04F5A670F1
:10397000F4F03AFE04F5A270F4F036FE04F59E7001
:10398000F4F032FE04F59A70F4F02EFE04F5967011
:10399000F4F02AFE04F59270F4F026FE04F58E7021
:1039A000F4F022FE04F58A70F4F01EFE04F5867031
:1039B000F4F01AFE04F58270F4F016FE04F1FC0037
:1039C000F4F012FE2046FFF77FFF204610BD00BF37
:1039D0008058167010B50446FFF7B4FF4FF4E47139
:1039E000204635F105F8204610BD0000304B10B5DB
:1039F00004460360D0F82406F4F008FBD4F8180657
:103A0000F4F004FBD4F80C06F4F000FBD4F8000644
:103A1000F4F0FCFAD4F8F405F4F0F8FAD4F8E80578
:103A2000F4F0F4FAD4F8DC05F4F0F0FAD4F8D005A8
:103A3000F4F0ECFAD4F8C405F4F0E8FAD4F8B805D8
:103A4000F4F0E4FA04F59660FFF73EFF04F56C70BD
:103A5000FFF73AFF04F52670FFF746FE04F5CC7039
:103A6000FFF732FF04F5A870F4F050FE04F59E70E5
:103A7000F4F004FB04F59270F4F000FB04F586709A
:103A8000F4F0FCFA04F1F400F4F0F8FA04F1DC00CC
:103A9000F4F0F4FA04F1C400F4F0F0FA04F19C003C
:103AA000F7F048FD2046FFF74BFD204610BD00BF54
:103AB0003846167010B50446FFF798FF4FF4C561FD
:103AC000204634F195FF204610BD0000244B10B570
:103AD00004460360D0F8D004F4F098FAD4F8C40493
:103AE000F4F094FAD4F8B804F4F090FAD4F8AC04F2
:103AF000F4F08CFAD4F8A004F4F088FAD4F8940422
:103B0000F4F084FAD4F88804F4F080FA04F56070D4
:103B1000FFF7DAFE04F52070FFF7D6FE04F5B47067
:103B2000FFF7E2FD04F59070F4F0F0FD04F5867007
:103B3000F4F0A4FA04F1F400F4F0A0FA04F1DC00CB
:103B4000F4F09CFA04F1C400F4F098FA04F19C003B
:103B5000F7F0F0FC2046FFF7F3FC204610BD00BF55
:103B60000046167010B50446FFF7B0FF4FF49B6196
:103B7000204634F13DFF204610BD0000324B10B509
:103B800004460360D0F80407F4F040FAD4F8F806CD
:103B9000F4F03CFAD4F8EC06F4F038FAD4F8E00685
:103BA000F4F034FAD4F8D406F4F030FAD4F8C806B5
:103BB000F4F02CFAD4F8BC06F4F028FAD4F8B006E5
:103BC000F4F024FAD4F8A406F4F020FAD4F8980615
:103BD000F4F01CFA04F5B260FFF776FE04F592608B
:103BE000FFF772FE04F55E70FFF77EFD04F5D870F6
:103BF000FFF7A8FE04F5B470F4F088FD04F5AA7090
:103C0000F4F03CFA04F59E70F4F038FA04F5927082
:103C1000F4F034FA04F58670F4F030FA04F1F400AC
:103C2000F4F02CFA04F1DC00F4F028FA04F1C400FA
:103C3000F4F024FA04F19C00F7F07CFC2046FFF736
:103C40007FFC204610BD00BFC845167010B5044665
:103C5000FFF794FF4FF4E161204634F1C9FE20469E
:103C600010BD0000244B10B504460360D0F8D0040A
:103C7000F4F0CCF9D4F8C404F4F0C8F9D4F8B804DA
:103C8000F4F0C4F9D4F8AC04F4F0C0F9D4F8A0040A
:103C9000F4F0BCF9D4F89404F4F0B8F9D4F888043A
:103CA000F4F0B4F904F56070FFF70EFE04F520702F
:103CB000FFF70AFE04F5B470FFF716FD04F59070E7
:103CC000F4F024FD04F58670F4F0D8F904F1F40062
:103CD000F4F0D4F904F1DC00F4F0D0F904F1C400FC
:103CE000F4F0CCF904F19C00F7F024FC2046FFF737
:103CF00027FC204610BD00BF9045167010B5044645
:103D0000FFF7B0FF4FF49B61204634F171FE20466F
:103D100010BD0000304B10B504460360D0F8F80623
:103D2000F4F074F9D4F8EC06F4F070F9D4F8E00685
:103D3000F4F06CF9D4F8D406F4F068F9D4F8C806B5
:103D4000F4F064F9D4F8BC06F4F060F9D4F8B006E5
:103D5000F4F05CF9D4F8A406F4F058F9D4F8980615
:103D6000F4F054F904F5B260FFF7AEFD04F592608B
:103D7000FFF7AAFD04F55E70FFF7B6FC04F5D870F6
:103D8000FFF7E0FD04F5B470F4F0C0FC04F5AA7090
:103D9000F4F074F904F59E70F4F070F904F5927083
:103DA000F4F06CF904F58670F4F068F904F1F400AD
:103DB000F4F064F904F1DC00F4F060F904F1C400FB
:103DC000F4F05CF904F19C00F7F0B4FB2046FFF737
:103DD000B7FB204610BD00BF5845167010B504460D
:103DE000FFF798FF4FF4E061204634F101FE2046D2
:103DF00010BD0000524B10B504460360D0F83409E2
:103E0000F4F004F9D4F82809F4F000F9D4F81C0906
:103E1000F4F0FCF8D4F81009F4F0F8F8D4F8040938
:103E2000F4F0F4F8D4F8F808F4F0F0F8D4F8EC086A
:103E3000F4F0ECF8D4F8E008F4F0E8F8D4F8D4089A
:103E4000F4F0E4F8D4F8C808F4F0E0F8D4F8BC08CA
:103E5000F4F0DCF8D4F8B008F4F0D8F8D4F8A408FA
:103E6000F4F0D4F8D4F89808F4F0D0F8D4F88C082A
:103E7000F4F0CCF8D4F88008F4F0C8F804F5076042
:103E8000F4F0B2FB04F66800F4F0AEFB04F6580060
:103E9000F4F0AAFB04F64800F4F0A6FB04F63800A0
:103EA000F4F0A2FB04F5E360FFF756FC04F5BF60F5
:103EB000FFF752FC04F5B360FFF7F4FB04F58C60E8
:103EC000FFF786FC04F58060FFF7ECFB04F56C70EF
:103ED000FFF7B2FB04F51E70FFF75AFC04F50A70F9
:103EE000FFF7AAFB04F5F070F4F010FC04F5E070A5
:103EF000F4F0B6F804F5CE70F4F0B2F804F5BC7046
:103F0000F4F0AEF804F5AA70F4F0AAF804F598708D
:103F1000F4F0A6F804F58670F4F0A2F804F1E800D5
:103F2000F4F09EF804F1C400F4F09AF804F19C0057
:103F3000F7F000FB2046FFF703FB204610BD00BF53
:103F4000AC4B167010B50446FFF754FF40F638111D
:103F5000204634F14DFD204610BD0000104B10B539
:103F600004460360D0F87802F4F050F804F5A87025
:103F7000FFF7F2FB04F58470F4F0C8FB04F1E800ED
:103F8000F4F06EF804F1C400F4F06AF804F19C0057
:103F9000F7F0D0FA2046FFF7D3FA204610BD00BF55
:103FA0005040167010B50446FFF7D8FF4FF420714B
:103FB000204634F11DFD204610BD00000C4B10B50D
:103FC00004460360D0F89001F4F020F804F58870FE
:103FD000F4F02CFB04F1C800F4F098FB04F1A80005
:103FE000F7F0A8FA204623F073FE204610BD00BF6C
:103FF0005851167010B50446FFF7E0FF4FF4CC712E
:10400000204634F1F5FC204610BD0000164B10B5DB
:1040100004460360D0F8C001F3F0F8FFD4F8B4010F
:10402000F3F0F4FFD4F8A801F3F0F0FF04F5CC703E
:10403000F4F0DAFA04F5C870F4F0D6FA04F5C470B6
:10404000F4F0D2FA04F58870F4F0F0FA04F1C80044
:10405000F4F05CFB04F1A800F7F06CFA204623F0C2
:1040600037FE204610BD00BF3850167010B504460C
:10407000FFF7CCFF4FF4E471204634F1B9FC204641
:1040800010BD0000184B10B504460360D0F81806A8
:10409000F3F0BCFFD4F80C06F3F0B8FFD4F8000638
:1040A000F3F0B4FFD4F8F405F3F0B0FF04F5826048
:1040B000FFF748FC04F51270FFF744FC04F50B70A1
:1040C000F3F0CEFF04F50570F3F0D8FF04F5F870B7
:1040D000F3F0C6FF04F5E670F3F0C2FF2046FFF7E9
:1040E00095FF204610BD00BFF44E167010B5044673
:1040F000FFF7C8FF4FF4C461204634F179FC204635
:1041000010BD00000E4B10B504460360D0F89801B6
:10411000F3F07CFF04F5C470F4F066FA04F58870DF
:10412000F4F084FA04F1C800F4F0F0FA04F1A80005
:10413000F7F000FA204623F0CBFD204610BD00BF6B
:10414000544C167010B50446FFF7DCFF4FF4D071E5
:10415000204634F14DFC204610BD000038B53E4BE2
:1041600000F5805504460360D5F82401F3F04EFFB6
:10417000D5F81801F3F04AFFD5F80C01F3F046FF2B
:10418000D5F80001F3F042FFD5F8F400F3F03EFF5C
:10419000D5F8E800F3F03AFFD5F8DC00F3F036FF8D
:1041A000D5F8D000F3F032FFD5F8C400F3F02EFFBD
:1041B000D5F8B800F3F02AFFD5F8AC00F3F026FFED
:1041C000D5F8A000F3F022FFD5F89400F3F01EFF1D
:1041D000D5F88800F3F01AFFE86FF3F017FF286FA7
:1041E000F3F014FF04F58350F4F0FEF904F6986040
:1041F000FFF7A8FB04F54D60FFF7A4FB04F53B6057
:10420000FFF7AAFA04F51E70FFF7F4FD04F5167027
:10421000F3F026FF04F50D70F3F022FF04F50470AF
:10422000F3F01EFF04F5F670F3F01AFFD4F8E00186
:10423000F3F0ECFED4F8D401F3F0E8FE04F5DE7000
:10424000F3F01CFF04F5D270F3F018FF2046FFF7DF
:1042500059FF204638BD00BF744B167010B5044698
:10426000FFF77CFF41F22811204634F1C1FB2046C4
:1042700010BD000038B5324B00F580550446036090
:10428000D5F8F400F3F0C2FED5F8E800F3F0BEFE76
:10429000D5F8DC00F3F0BAFED5F8D000F3F0B6FEA6
:1042A000D5F8C400F3F0B2FED5F8B800F3F0AEFED6
:1042B000D5F8AC00F3F0AAFED5F8A000F3F0A6FE06
:1042C000D5F89400F3F0A2FED5F88800F3F09EFE36
:1042D000E86FF3F09BFE286FF3F098FE04F56A6038
:1042E000FFF730FB04F6D840FFF72CFB04F6B8309C
:1042F000FFF732FA04F52070FFF77CFD04F5197022
:10430000F3F0AEFE04F51070F3F0AAFE04F50770AA
:10431000F3F0A6FE04F5FC70F3F0A2FE04F5F070D5
:10432000F3F0ACFE04F5E470F3F0A8FE04F5D270EF
:10433000F3F096FE2046FFF7E5FE204638BD00BFAD
:10434000044B167010B50446FFF794FF41F2F801D4
:10435000204634F14DFB204610BD00000E4B10B539
:104360000446036000F59C70FFF784FF04F1F00041
:10437000F4F0CCF904F1DC00F3F080FE04F1C400A9
:10438000F3F07CFE04F19C00F7F0D4F82046FFF730
:10439000D7F8204610BD00BF7C49167010B5044602
:1043A000FFF7DCFF41F23021204634F121FB2046AB
:1043B00010BD00000E4B10B50446036000F59C7064
:1043C000FFF758FF04F1F000F4F0A0F904F1DC006D
:1043D000F3F054FE04F1C400F3F050FE04F19C002D
:1043E000F7F0A8F82046FFF7ABF8204610BD00BF55
:1043F0004449167010B50446FFF7DCFF41F2302146
:10440000204634F1F5FA204610BD0000224B10B5CD
:1044100004460360D0F85407F3F0F8FDD4F84807D9
:10442000F3F0F4FDD4F83C07F3F0F0FDD4F83007D6
:10443000F3F0ECFDD4F82407F3F0E8FDD4F8180706
:10444000F3F0E4FDD4F80C07F3F0E0FD04F5A76009
:10445000FFF778FA04F55C70FFF774FA04F514704E
:10446000FFF77AF904F50D70F3F0FAFD04F5047026
:10447000F3F0F6FD04F5F670F3F0F2FD04F5E470E8
:10448000F3F0EEFD04F5D270F3F0EAFD2046FFF7FD
:1044900039FE204610BD00BF944A167010B5044680
:1044A000FFF7B4FF4FF4EB61204634F1A1FA204648
:1044B00010BD0000264B10B504460360D0F8680715
:1044C000F3F0A4FDD4F85C07F3F0A0FDD4F8500796
:1044D000F3F09CFDD4F84407F3F098FDD4F83807C6
:1044E000F3F094FDD4F82C07F3F090FDD4F82007F6
:1044F000F3F08CFDD4F81407F3F088FDD4F8080726
:10450000F3F084FD04F5BC60FFF726F904F5836041
:10451000FFF718FA04F51470FFF714FA04F50D709C
:10452000F3F09EFD04F50470F3F09AFD04F5F670C7
:10453000F3F096FD04F5E470F3F092FD04F5D2700B
:10454000F3F08EFD2046FFF7DDFD204610BD00BFD5
:10455000244A167010B50446FFF7ACFF4FF4EE6125
:10456000204634F145FA204610BD000010B504463F
:10457000B030F3F06BF904F1A800F4F035F804F171
:10458000A000F4F031F82146054B064841F89C3B69
:1045900033F073F92046FEF7D3FF204610BD00BF6D
:1045A000F05816704C54038010B50446FFF7DEFF38
:1045B000C021204634F11CFA204610BD38B52D4BE1
:1045C00000F5805504460360D5F83C03F3F01EFD6A
:1045D000D5F83003F3F01AFDD5F82403F3F016FDF7
:1045E000D5F81803F3F012FD04F596500830F4F0F6
:1045F0008DF804F59450F4F089F804F53160FFF774
:1046000059FF04F52760FEF79BFF04F54070FFF7A4
:1046100051FF04F51870FEF793FF04F5D070FFF713
:10462000A5FF04F5AC70F4F071F804F5A470F3F094
:1046300025FDD4F83C01F3F0E9FC04F59270F3F0A9
:104640001DFD04F58670F3F019FD04F1F400F3F09C
:1046500015FD04F1DC00F3F011FD04F1C400F3F0EA
:104660000DFD04F19C00F6F065FF2046FEF768FFA3
:10467000204638BDB449167010B50446FFF79EFFBA
:104680004FF49A51204634F1B3F9204610BD000092
:1046900010B50446B030F3F0D9F804F1A800F3F0F7
:1046A000A3FF04F1A000F3F09FFF2146054B06484D
:1046B00041F89C3B33F0E1F82046FEF741FF2046ED
:1046C00010BD00BFF05816704C54038010B504465E
:1046D000FFF7DEFFC021204634F18AF9204610BDE5
:1046E000204B10B504460360D0F84007F3F08EFC71
:1046F000D4F83407F3F08AFCD4F82807F3F086FCEA
:10470000D4F81C07F3F082FC04F5C960FFF7C0FF82
:1047100004F59060FFF716F904F52E70FFF712F913
:1047200004F5CC70FFF718F804F5A870F3F0EEFF6D
:1047300004F59870F3F094FC04F58670F3F090FCA7
:1047400004F1E800F3F08CFC04F1C400F3F088FC01
:1047500004F19C00F6F0EEFE2046FEF7F1FE204646
:1047600010BD00BFDC4D167010B50446FFF7B8FF52
:104770004FF4E961204634F13BF9204610BD0000BA
:10478000364B10B504460360D0F8A80DF3F03EFC9C
:10479000D4F89C0DF3F03AFCD4F8900DF3F036FC0D
:1047A000D4F8840DF3F032FCD4F8780DF3F02EFC3D
:1047B000D4F86C0DF3F02AFCD4F8600DF3F026FC6D
:1047C00004F54860FFF764FF04F6B820FFF7BAF875
:1047D00004F6F810FFF75CFF04F50360FFF7B2F88A
:1047E00004F5CD60FFF7AEF804F59460FFF7AAF882
:1047F00004F56070FEF7B0FF04F53070FFF748FF76
:1048000004F50070FFF7B2FE04F5DC70F3F07EFFF4
:1048100004F5CE70F3F024FC04F5BC70F3F020FC3A
:1048200004F5AA70F3F01CFC04F59870F3F018FC82
:1048300004F58670F3F014FC04F1E800F3F010FCCA
:1048400004F1C400F3F00CFC04F19C00F6F072FEDD
:104850002046FEF775FE204610BD00BFA44D167021
:1048600010B50446FFF78CFF4FF45B61204634F12E
:10487000BFF8204610BD000038B56F4B00F58045ED
:1048800004460360D5F8540FF3F0C0FBD5F8480F89
:10489000F3F0BCFBD5F83C0FF3F0B8FBD5F8300FC4
:1048A000F3F0B4FBD5F8240FF3F0B0FBD5F8180FF4
:1048B000F3F0ACFBD5F80C0FF3F0A8FBD5F8000F24
:1048C000F3F0A4FBD5F8F40EF3F0A0FBD5F8E80E56
:1048D000F3F09CFBD5F8DC0EF3F098FBD5F8D00E86
:1048E000F3F094FB04F59D40F3F010FF04F59C40B9
:1048F0003830F3F00BFF04F59B407030F3F006FF07
:1049000004F59B402830F3F001FF04F59A40603035
:10491000F3F0FCFE04F59A401830F3F0F7FE04F5CE
:104920006F503030FFF71AFC04F56D501030FEF771
:1049300007FE04F528502830FFF710FC04F5255039
:104940002830FFF7A5FE04F523500830FEF7F8FDE8
:1049500004F520502830FEF7F3FD04F51E50083012
:10496000FEF7EEFD04F5B350FFF7F8FB04F5AD508C
:10497000FFF78EFE04F5A850FEF7E2FD04F5A35004
:10498000FEF7DEFD04F59D50FFF7F0FD04F51E7007
:10499000FFF7E4FB04F50C70F3F0B8FE04F50870C3
:1049A000F3F06CFB04F50270F3F068FB04F5F870AB
:1049B000F3F064FB04F5EC70F3F060FB04F5E070D9
:1049C000F3F05CFB04F5D470F3F058FB04F5C87009
:1049D000F3F054FBD4F88401F3F018FBD4F8780119
:1049E000F3F014FB04F5B070F3F048FB04F5A47089
:1049F000F3F044FB04F59870F3F040FB04F58C7081
:104A0000F3F03CFB04F58070F3F038FBD4F8F400CD
:104A1000F3F0FCFA04F1DC00F3F030FB04F1C40025
:104A2000F3F02CFB04F19C00F6F084FD2046FEF729
:104A300087FD204638BD00BF3C4B167010B50446BC
:104A4000FFF71AFF44F65871204633F1D1FF204694
:104A500010BD000038B5514B00F5405504460360C9
:104A6000D5F8E00AF3F0D2FAD5F8D40AF3F0CEFA8A
:104A7000D5F8C80AF3F0CAFAD5F8BC0AF3F0C6FABA
:104A8000D5F8B00AF3F0C2FAD5F8A40AF3F0BEFAEA
:104A9000D5F8980AF3F0BAFAD5F88C0AF3F0B6FA1A
:104AA000D5F8800AF3F0B2FA04F568503030F3F02C
:104AB0002DFE04F567502830F3F028FE04F566500B
:104AC0002030F3F023FE04F565501830F3F01EFE9D
:104AD00004F562501830FFF7DBFD04F55F50383005
:104AE000FEF72EFD04F51C50FFF7C4FB04F519502A
:104AF000FFF73CFD04F5A8501830FFF72FFB04F535
:104B0000A3501830FEF71CFD04F59E501830FEF738
:104B100017FD04F52C70FFF721FB04F50470FEF778
:104B20000FFD04F5E470F3F0F1FD04F5DA70F3F035
:104B3000A5FA04F5CE70F3F0A1FA04F5C270F3F013
:104B40009DFAD4F87801F3F061FA04F5B070F3F04F
:104B500095FA04F5A470F3F091FA04F59870F3F067
:104B60008DFA04F58C70F3F089FA04F58070F3F097
:104B700085FAD4F8F400F3F049FA04F1DC00F3F01C
:104B80007DFA04F1C400F3F079FA04F19C00F6F028
:104B9000D1FC2046FEF7D4FC204638BDCC4A167026
:104BA00010B50446FFF756FF43F6E821204633F1DF
:104BB0001FFF204610BD000038B54E4B00F5405594
:104BC00004460360D5F84C01F3F020FAD5F8400113
:104BD000F3F01CFAD5F83401F3F018FAD5F82801EF
:104BE000F3F014FAD5F81C01F3F010FAD5F810011F
:104BF000F3F00CFAD5F80401F3F008FAD5F8F80050
:104C0000F3F004FA04F542502830F3F07FFD04F588
:104C100041502030F3F07AFD28461830F3F076FD4D
:104C200004F53F501030F3F071FD04F521502030B1
:104C3000FFF740FC04F5B9501830FFF78FFA04F580
:104C4000B4501830FEF77CFC04F5AE60FFF786FA2E
:104C500004F59A60FEF774FC04F58260FFF718FD16
:104C600004F55C70FEF76CFC04F52C70FFF77EFC1D
:104C700004F50470FEF764FC04F5E470F3F046FDFF
:104C800004F5DA70F3F0FAF904F5CE70F3F0F6F902
:104C900004F5C270F3F0F2F904F5B670F3F0EEF932
:104CA000D4F86001F3F0B2F904F5A470F3F0E6F97A
:104CB00004F59870F3F0E2F904F58C70F3F0DEF986
:104CC000D4F80C01F3F0A2F904F1F400F3F0D6F9F2
:104CD00004F1DC00F3F0D2F904F1C400F3F0CEF9F2
:104CE00004F19C00F6F026FC2046FEF729FC204645
:104CF00038BD00BFEC49167010B50446FFF75CFFE5
:104D000043F25011204633F173FE204610BD0000DF
:104D10001C4B10B504460360D0F89404F3F076F908
:104D2000D4F88804F3F072F9D4F87C04F3F06EF947
:104D3000D4F87004F3F06AF9D4F86404F3F066F977
:104D4000D4F85804F3F062F904F58760F3F04CFCF2
:104D500004F57C70F3F0DAFC04F50A70FEF7F2FD5E
:104D600004F59470FEF7B0FD04F1E000F3F0CEFC22
:104D700004F1BC00F6F0DEFB2046FFF789FC20467C
:104D800010BD00BF1440167010B50446FFF7C0FFF9
:104D90004FF49361204633F12BFE204610BD0000F6
:104DA000144B10B504460360D0F81C0FF3F02EF935
:104DB000D4F8100FF3F02AF9D4F8040FF3F026F921
:104DC00004F65820FFF7A4FF04F5B860FFF7A0FF32
:104DD00004F59470FFF79CFF04F1E000F3F096FCFB
:104DE00004F1BC00F6F0A6FB2046FFF7BFFB20460F
:104DF00010BD00BFD83F167010B50446FFF7D0FFB6
:104E00004FF47261204633F1F3FD204610BD0000DF
:104E1000104B10B504460360D0F8740AF3F0F6F8AE
:104E2000D4F8680AF3F0F2F804F5B860FFF770FF01
:104E300004F59470FFF76CFF04F1E000F3F066FCFA
:104E400004F1BC00F6F076FB2046FFF78FFB20460E
:104E500010BD00BF9C3F167010B50446FFF7D8FF89
:104E600040F67821204633F1C3FD204610BD0000F6
:104E700038B5194B00F5805504460360D5F8C403D6
:104E8000F3F0C4F8D5F8B803F3F0C0F8D5F8AC03E4
:104E9000F3F0BCF8D5F8A003F3F0B8F804F56F60B0
:104EA000FFF736FF04F65820FFF732FF04F5B8602D
:104EB000FFF72EFF04F59470FFF72AFF04F1E000DE
:104EC000F3F024FC04F1BC00F6F034FB2046FFF7BD
:104ED0004DFB204638BD00BF003E167010B504469D
:104EE000FFF7C6FF41F2C831204633F181FD20466D
:104EF00010BD0000074B10B503610446064B40F897
:104F00000C3BF3F03FF804F10800F3F0DFF8204623
:104F100010BD00BF6C5816703058167010B504469E
:104F2000FFF7E8FF1421204633F162FD204610BD53
:104F3000074B10B503610446064B40F80C3BF3F0F9
:104F400021F804F10800F3F0C1F8204610BD00BFBD
:104F5000AC5116703058167010B50446FFF7E8FFD4
:104F60001821204633F144FD204610BD064B10B5F4
:104F7000044640F80C3BF3F005F804F10800F3F0A8
:104F8000A5F8204610BD00BF3058167010B5044675
:104F9000FFF7ECFF1021204633F12AFD204610BD1B
:104FA000064B10B5044640F80C3BF2F0EBFF04F161
:104FB0000800F3F08BF8204610BD00BF3058167083
:104FC00010B50446FFF7ECFF1021204633F110FD29
:104FD000204610BD064B10B5044640F80C3BF2F0DD
:104FE000D1FF04F10800F3F071F8204610BD00BFB6
:104FF0003058167010B50446FFF7ECFF102120461C
:1050000033F1F6FC204610BD204B10B5044603607A
:10501000D0F82C06F2F0FAFFD4F82006F2F0F6FFF2
:10502000D4F81406F2F0F2FFD4F80806F2F0EEFF1E
:1050300004F5B760F3F06AFB04F5AE60F3F066FBCD
:1050400004F59A60FEF77CFA04F58160FEF7E0FB58
:1050500004F55A70FEF774FA04F52870FEF7D8FBD1
:1050600004F51670F3F052FB04F50E70F2F0F8FF41
:1050700004F50570F2F0F4FF04F5F670F6F05AFA54
:1050800020469FF065F9204610BD00BF14571670EA
:1050900010B50446FFF7B8FF4FF4C661204633F160
:1050A000A7FC204610BD0000324B10B5044603603B
:1050B000D0F8400AF2F0AAFFD4F8340AF2F0A6FFC2
:1050C000D4F8280AF2F0A2FFD4F81C0AF2F09EFFEE
:1050D000D4F8100AF2F09AFFD4F8040AF2F096FF1E
:1050E000D4F8F809F2F092FFD4F8EC09F2F08EFF50
:1050F000D4F8E009F2F08AFF04F51D60F3F074FAC9
:1051000004F6C810F3F070FA04F51560F3F08EFAA7
:1051100004F60810F3F0FAFA04F50C60F3F0F6FA6E
:1051200004F6180022F0D4FD04F5EF60FEF708FA4B
:1051300004F5DA6022F0CCFD04F2BC60F2F09EFFD0
:1051400004F5D360F2F08CFF04F5D060F2F096FF26
:1051500004F5CD60F2F092FF04F5CA60F2F08EFF24
:1051600004F5C760F2F08AFF2046FFF74DFF2046A6
:1051700010BD00BFDC56167010B50446FFF794FF53
:1051800040F64821204633F133FC204610BD000094
:10519000BE4B10B504460360D0F8E80CF2F036FFC1
:1051A000D4F8DC0CF2F032FFD4F8D00CF2F02EFF81
:1051B000D4F8C40CF2F02AFFD4F8B80CF2F026FFB1
:1051C000D4F8AC0CF2F022FFD4F8A00CF2F01EFFE1
:1051D000D4F8940CF2F01AFFD4F8880CF2F016FF11
:1051E000D4F87C0CF2F012FFD4F8700CF2F00EFF41
:1051F000D4F8640CF2F00AFFD4F8580CF2F006FF71
:10520000D4F84C0CF2F002FFD4F8400CF2F0FEFEA1
:10521000D4F8340CF2F0FAFED4F8280CF2F0F6FED2
:10522000D4F81C0CF2F0F2FED4F8100CF2F0EEFE02
:10523000D4F8040CF2F0EAFED4F8F80BF2F0E6FE33
:10524000D4F8EC0BF2F0E2FED4F8E00BF2F0DEFE64
:10525000D4F8D40BF2F0DAFED4F8C80BF2F0D6FE94
:10526000D4F8BC0BF2F0D2FED4F8B00BF2F0CEFEC4
:10527000D4F8A40BF2F0CAFED4F8980BF2F0C6FEF4
:10528000D4F88C0BF2F0C2FED4F8800BF2F0BEFE24
:10529000D4F8740BF2F0BAFED4F8680BF2F0B6FE54
:1052A000D4F85C0BF2F0B2FED4F8500BF2F0AEFE84
:1052B000D4F8440BF2F0AAFED4F8380BF2F0A6FEB4
:1052C000D4F82C0BF2F0A2FED4F8200BF2F09EFEE4
:1052D000D4F8140BF2F09AFED4F8080BF2F096FE14
:1052E000D4F8FC0AF2F092FED4F8F00AF2F08EFE46
:1052F000D4F8E40AF2F08AFED4F8D80AF2F086FE76
:10530000D4F8CC0AF2F082FED4F8C00AF2F07EFEA5
:10531000D4F8B40AF2F07AFED4F8A80AF2F076FED5
:10532000D4F89C0AF2F072FED4F8900AF2F06EFE05
:1053300004F66820F6F0FEF804F52660F3F054F960
:1053400004F52560F3F050F904F52460F3F04CF90E
:1053500004F52360F3F048F904F52260F3F044F912
:1053600004F52160F3F040F904F52060F3F03CF916
:1053700004F51F60F3F038F904F51E60F3F034F91A
:1053800004F51D60F3F030F904F51C60F3F02CF91E
:1053900004F51B60F3F028F904F51A60F3F024F922
:1053A00004F51960F3F020F904F51860F3F01CF926
:1053B00004F51760F3F018F904F51660F3F014F92A
:1053C00004F51560F3F010F904F51460F3F00CF92E
:1053D00004F51360F3F008F904F51260F3F004F932
:1053E00004F51160F3F000F904F51060F3F0FCF837
:1053F00004F50F60F3F0F8F804F50E60F3F0F4F83C
:1054000004F50960FEF718F904F50560FEF731F9B7
:1054100004F5E760FEF768F904F5DB60FEF742F992
:1054200004F5D160FEF708F904F5C960FEF721F92B
:1054300004F5B46022F04CFC04F59F6022F048FCB7
:1054400004F58A60FEF794F804F58060FEF7F4F83E
:1054500004F57070FEF70DF904F52870FEF77CF97D
:1054600004F5C470FEF740F904F5A070F3F04EF9AE
:1054700004F1C800F3F0DAF804F1A800F6F05AF8E5
:10548000204622F025FC204610BD00BFF0511670CA
:1054900010B50446FFF77CFE4FF44F61204633F110
:1054A000A7FA204610BD0000224B10B50446036049
:1054B000D0F86C03F2F0AAFDD4F86003F2F0A6FD78
:1054C000D4F85403F2F0A2FDD4F84803F2F09EFDA4
:1054D00004F54C70F3F088F804F54870F3F084F8A4
:1054E00004F54470F3F080F804F52670F3F09EF8AC
:1054F00004F5FC70FEF724F804F5A87022F0E8FB30
:1055000004F58470F3F002F904F1F400F2F0B6FD52
:1055100004F1DC00F2F0B2FD04F1C400F2F0AEFDE3
:1055200004F19C00F6F006F82046FEF709F8204644
:1055300010BD00BF2051167010B50446FFF7B4FF30
:105540004FF45C71204633F153FA204610BD000041
:105550001E4B10B504460360D0F8A005F2F056FDCE
:10556000D4F89405F2F052FDD4F88805F2F04EFD1F
:10557000D4F87C05F2F04AFDD4F87005F2F046FD4F
:1055800004F59D60F3F052F804F5886022F0A0FB6A
:1055900004F55070FEF798F904F51070FEF794F9D1
:1055A00004F50870F2F05CFD04F5FE70F2F058FDB1
:1055B00004F5F270F2F062FD04F5E670F2F05EFDC3
:1055C0002046FEF723FD204610BD00BF0050167098
:1055D00010B50446FFF7BCFF4FF4B561204633F128
:1055E00007FA204610BD0000164B10B504460360B4
:1055F000D0F8EC02F2F00AFDD4F8E002F2F006FD79
:1056000004F51870F3F012F804F5DC7022F060FB7A
:1056100004F5A070F3F00AF804F1F800F3F076F85E
:1056200004F1E800F2F02AFD04F1D000F2F026FDCA
:1056300004F1A800F5F07EFF204622F049FB204649
:1056400010BD00BFA04F167010B50446FFF7CCFF89
:105650004FF43C71204633F1CBF9204610BD0000D9
:10566000184B10B504460360D0F8F802F2F0CEFCF7
:10567000D4F8EC02F2F0CAFCD4F8E002F2F0C6FC76
:1056800004F51870F2F0D2FF04F5DC7022F020FB74
:1056900004F5A070F2F0CAFF04F1F800F3F036F858
:1056A00004F1E800F2F0EAFC04F1D000F2F0E6FCCC
:1056B00004F1A800F5F03EFF204622F009FB204649
:1056C00010BD00BFC44C167010B50446FFF7C8FFEC
:1056D0004FF44071204633F18BF9204610BD000095
:1056E00038B5364B00F5805504460360D5F8FC0A02
:1056F000F2F08CFCD5F8F00AF2F088FCD5F8E40A58
:10570000F2F084FCD5F8D80AF2F080FCD5F8CC0A87
:10571000F2F07CFCD5F8C00AF2F078FCD5F8B40AB7
:10572000F2F074FCD5F8A80AF2F070FCD5F89C0AE7
:10573000F2F06CFCD5F8900AF2F068FCD5F8840A17
:10574000F2F064FCD5F8780AF2F060FC04F5CF5072
:105750001830F2F06BFF04F59550FEF757FE04F594
:105760008F50183022F0B4FA04F58A50103022F02D
:10577000AFFA04F6F810FEF749FE04F52870FEF7BC
:1057800045FE04F5F070FEF783FF04F59C7022F0EF
:105790009FFA04F1F000F2F0B9FF04F1DC00F2F03E
:1057A0006DFC04F1C400F2F069FC04F19C00F5F01A
:1057B000C1FE2046FDF7C4FE204638BD5C4A167087
:1057C00010B50446FFF78CFF4FF4D851204633F153
:1057D0000FF9204610BD000038B5504B00F5883554
:1057E00004460360D5F8A402F2F010FCD5F8980244
:1057F000F2F00CFCD5F88C02F2F008FCD5F880022F
:10580000F2F004FCD5F87402F2F000FCD5F868025E
:10581000F2F0FCFBD5F85C02F2F0F8FBD5F8500290
:10582000F2F0F4FBD5F84402F2F0F0FBD5F83802C0
:10583000F2F0ECFB05F5F470F2F068FF04F57F4040
:10584000B830FEF7B7FD04F56D408830FEF786FDF1
:1058500004F55A404830FEF7B1FE04F52840F83010
:10586000FFF7AAF904F50D40F830FFF739FF04F50A
:105870000D405830FDF764FE04F5A4407030FFF78A
:10588000E9F804F54670FEF7F7FF04F51670FEF729
:105890006DFE04F50470F2F039FF04F5FE70F2F0CD
:1058A000EDFB04F5F270F2F0E9FB04F5E670F2F0BE
:1058B000E5FB04F5DA70F2F0E1FB04F5CE70F2F0EE
:1058C000DDFB04F5C270F2F0D9FB04F5B670F2F01E
:1058D000D5FB04F5AA70F2F0D1FB04F59E70F2F04E
:1058E000CDFB04F59270F2F0C9FB04F58670F2F07E
:1058F000C5FB04F1F400F2F0C1FB04F1DC00F2F0AE
:10590000BDFB04F1C400F2F0B9FB04F19C00F5F01A
:1059100011FE2046FDF714FE204638BD0C491670D6
:1059200010B50446FFF758FF0249204633F160F8EE
:10593000204610BDA812010038B53F4B00F50055B8
:1059400004460360D5F8B401F2F060FBD5F8A80175
:10595000F2F05CFBD5F89C01F2F058FBD5F8900111
:10596000F2F054FBD5F88401F2F050FBD5F8780141
:10597000F2F04CFB04F503503830F2F057FE04F51A
:1059800002503030F2F0C2FE04F5CD501030FEF778
:10599000C1F904F5A6501830FEF764F904F55D600E
:1059A000FEF7ECF804F6F800FEF790F804F5347012
:1059B000FEF71CF804F50A7022F08AF904F5F0707D
:1059C000F2F0A4FE04F5E670F2F058FB04F5DA708C
:1059D000F2F054FB04F5CE70F2F050FB04F5C27007
:1059E000F2F04CFB04F5B670F2F048FB04F5AA7037
:1059F000F2F044FB04F59E70F2F040FB04F5927067
:105A0000F2F03CFB04F58670F2F038FB04F1F40090
:105A1000F2F034FB04F1DC00F2F030FB04F1C400DE
:105A2000F2F02CFB04F19C00F5F084FD2046FDF71C
:105A300087FD204638BD00BF2045167010B50446CE
:105A4000FFF77AFF42F2B811204632F1D1FF20462B
:105A500010BD0000224B10B504460360D0F8BC070F
:105A6000F2F0D4FAD4F8B007F2F0D0FAD4F8A407E0
:105A7000F2F0CCFAD4F89807F2F0C8FAD4F88C0710
:105A8000F2F0C4FAD4F88007F2F0C0FA04F5E66048
:105A9000F2F03CFE04F5DD60F2F038FE04F5A4609F
:105AA000FDF750FF04F59060FDF74AFD04F56E70B8
:105AB000FDF7AEFE04F55C70F2F028FE04F55870B8
:105AC000F2F0DCFA04F55270F2F0D8FA04F54870FE
:105AD000F5F030FD20469EF0D1FF204610BD00BFFE
:105AE000C854167010B50446FFF7B4FF4FF4F861C0
:105AF000204632F17DFF204610BD00005C4B10B502
:105B000004460360D0F8200CF2F080FAD4F8140CAC
:105B1000F2F07CFAD4F8080CF2F078FAD4F8FC0B26
:105B2000F2F074FAD4F8F00BF2F070FAD4F8E40B57
:105B3000F2F06CFAD4F8D80BF2F068FAD4F8CC0B87
:105B4000F2F064FAD4F8C00BF2F060FAD4F8B40BB7
:105B5000F2F05CFAD4F8A80BF2F058FAD4F89C0BE7
:105B6000F2F054FAD4F8900BF2F050FAD4F8840B17
:105B7000F2F04CFAD4F8780BF2F048FAD4F86C0B47
:105B8000F2F044FAD4F8600BF2F040FA04F5356014
:105B9000F2F02AFD04F64830F2F026FD04F53460F8
:105BA000F2F022FD04F63830F2F01EFD04F5336009
:105BB000F2F01AFD04F62830F2F016FD04F532601A
:105BC000F2F012FD04F61830F2F00EFD04F531602B
:105BD000F2F00AFD04F60830F2F006FD04F530603C
:105BE000F2F002FD04F6F820F2F0FEFC04F52F605E
:105BF000F2F0FAFC04F67820F2F018FD04F66820C2
:105C0000F2F0F2FC04F65820F2F0EEFC04F521600C
:105C1000F2F07CFD04F69810F2F008FD04F688100E
:105C2000F2F0E2FC04F50E6022F052F804F63800BF
:105C300022F04EF804F62800F2F020FAD4F81C08FE
:105C4000F2F0E4F904F60400F2F018FAD4F8F807D8
:105C5000F2F0DCF904F5FC60F2F010FA04F5F960FA
:105C6000F2F00CFA2046FFF7F5FE204610BD00BF0B
:105C70008854167010B50446FFF740FF40F62841DF
:105C8000204632F1B5FE204610BD0000104B10B585
:105C900004460360D0F8440EF2F0B8F9D4F8380E98
:105CA000F2F0B4F904F56260F2F09EFC04F658409C
:105CB000FDF748FE04F64440F2F0E0F904F62C400B
:105CC000F2F0DCF92046FFF719FF204610BD00BFB7
:105CD0004854167010B50446FFF7D8FF40F64861E7
:105CE000204632F185FE204610BD00000E4B10B557
:105CF00004460360D0F8800EF2F088F9D4F8740EF0
:105D0000F2F084F9D4F8680EF2F080F9D4F85C0E61
:105D1000F2F07CF9D4F8500EF2F078F92046FFF753
:105D2000B5FF204610BD00BFE044167010B5044614
:105D3000FFF7DCFF40F68861204632F159FE20462D
:105D400010BD0000124B10B504460360D0F8940E4D
:105D5000F2F05CF9D4F8880EF2F058F9D4F87C0E21
:105D6000F2F054F9D4F8700EF2F050F9D4F8640E51
:105D7000F2F04CF9D4F8580EF2F048F904F6486005
:105D8000F2F032FC2046FFF781FF204610BD00BF35
:105D90005C3F167010B50446FFF7D4FF40F69861DB
:105DA000204632F125FE204610BD00000C4B10B5F8
:105DB00004460360D0F89C0DF2F028F904F5476022
:105DC000FDF7CAFC04F54560F2F04AF904F62C40F0
:105DD000F2F046F92046FFF791FE204610BD00BFC5
:105DE0004853167010B50446FFF7E0FF4FF45A61B0
:105DF000204632F1FDFD204610BD0000034B10B5DA
:105E000004460360FFF7D2FF204610BDC85216704B
:105E100010B50446FFF7F2FF4FF45A61204632F105
:105E2000E7FD204610BD00001C4B10B50446036082
:105E3000D0F8E00FF2F0EAF8D4F8D40FF2F0E6F878
:105E4000D4F8C80FF2F0E2F804F57B60F2F0CCFB76
:105E500004F57A60F2F0C8FB04F6D850FDF772FD45
:105E600004F6B840FDF778FC04F69840F2F0F8F834
:105E700004F54860F2F002F904F65C40F2F0F0F844
:105E800004F63840F2F0ECF8D4F82C0CF2F0BEF83E
:105E90002046FFF733FE204610BD00BF9448167021
:105EA00010B50446FFF7C0FF40F6E871204632F116
:105EB0009FFD204610BD00000E4B10B50446036048
:105EC000D0F8580CF2F0A2F8D4F84C0CF2F09EF88E
:105ED000D4F8400CF2F09AF8D4F8340CF2F096F8BA
:105EE00004F62440F2F080FB2046FFF707FE204630
:105EF00010BD00BF7447167010B50446FFF7DCFFF5
:105F00004FF44661204632F173FD204610BD00007B
:105F100038B5234B00F5805504460360D5F8480199
:105F2000F2F074F8D5F83C01F2F070F8D5F83001D1
:105F3000F2F06CF8D5F82401F2F068F8D5F8180101
:105F4000F2F064F804F588500830F2F04DFB04F5E7
:105F50008850F2F049FB04F6D870FDF7FDFB04F51C
:105F60006160FDF7EFFC04F54F60FDF7F5FB04F50C
:105F70004D60F2F075F804F6AC40F2F071F804F6FA
:105F80008840F2F06DF804F54760F2F077F8D4F845
:105F9000640CF2F03BF82046FFF78EFF204638BD38
:105FA000C040167010B50446FFF7B2FF41F2501121
:105FB000204632F11DFD204610BD000038B58A4B49
:105FC00000F5805504460360D5F8180BF2F01EF872
:105FD000D5F80C0BF2F01AF8D5F8000BF2F016F821
:105FE000D5F8F40AF2F012F8D5F8E80AF2F00EF853
:105FF000D5F8DC0AF2F00AF8D5F8D00AF2F006F883
:10600000D5F8C40AF2F002F8D5F8B80AF1F0FEFFAC
:10601000D5F8AC0AF1F0FAFFD5F8A00AF1F0F6FFD6
:10602000D5F8940AF1F0F2FFD5F8880AF1F0EEFF06
:1060300004F5D3501830F2F0D7FA04F5D3501030ED
:10604000F2F0D2FA04F5D150F2F060FB04F5CD5035
:106050000830F2F0EBFA04F5CB50F2F057FB04F500
:10606000C7500830F2F0E2FA04F5C3501030F2F0F5
:10607000DDFA04F5C1500830F2F048FB04F5BF50DA
:10608000F2F044FB04F5BB500830F2F0CFFA04F50F
:10609000B950F2F03BFB04F5B5500830F2F0C6FA07
:1060A00004F5B350F2F032FB04F5AF500830F2F0D3
:1060B000BDFA04F5AA5021F00BFE04F5A4501830E7
:1060C00021F006FE04F59F50103021F001FE04F58A
:1060D0009A501030FDF734FA04F58C500830FDF773
:1060E00031FC04F5875021F0F3FD04F581501830A0
:1060F00021F0EEFD04F69870FDF722FA04F6F86040
:10610000FDF71EFA04F5656021F0E2FD04F63C603F
:10611000F1F0B4FF04F62460F1F0B0FFD4F8180EEB
:10612000F1F074FF04F56060F1F0A8FF04F6E850A8
:10613000F1F0A4FF04F55D60F1F0A0FF04F6B850A3
:10614000F1F09CFF04F55A60F1F098FF04F68850D6
:10615000F1F094FFD4F87C0DF1F058FF04F6645090
:10616000F1F08CFFD4F8580DF1F050FF04F55460B5
:10617000F1F084FF04F62850F1F080FF04F551603F
:10618000F1F07CFF04F6F840F1F078FF04F54E6082
:10619000F1F074FFD4F8D40CF1F038FF04F6BC40F1
:1061A000F1F06CFFD4F8B00CF1F030FF04F6984039
:1061B000F1F064FFD4F88C0CF1F028FF04F6744081
:1061C000F1F05CFF04F54560F1F04AFF04F6384059
:1061D000F1F054FFD4F82C0CF1F018FF2046FFF733
:1061E0008DFC204638BD00BF3842167010B50446FD
:1061F000FFF7E4FE4FF4D951204632F1F9FB204677
:1062000010BD00000C4B10B50446036000F509609A
:10621000F2F07CFA04F5FE60FDF792F904F5FC60FB
:10622000F1F02CFF04F5F960F1F028FF2046FFF7AC
:1062300011FC204610BD00BFE050167010B504469A
:10624000FFF7E0FF40F6D801204632F1D1FB2046AF
:1062500010BD0000164B10B504460360D0F8D00AFC
:10626000F1F0D4FED4F8C40AF1F0D0FE04F52760B2
:10627000F2F04CFA04F51560FDF76EFA04F63800FA
:10628000FDF732FA04F61C00F1F0EAFE04F5FF60B7
:10629000F1F0E6FE04F5FC60F1F0F0FE04F5F960C3
:1062A000F1F0ECFE2046FFF7D5FB204610BD00BF05
:1062B0003841167010B50446FFF7CCFF40F6D821E0
:1062C000204632F195FB204610BD00000A4B10B568
:1062D00003601C330446143040F8043C14F0F8FA10
:1062E0002046064B40F80C3BF1F04CFE04F1080050
:1062F000F1F0ECFE204610BDD84F167030581670E5
:1063000010B50446FFF7E2FF4FF4A271204632F1C8
:106310006FFB204610BD0000884B4FF0FF3240F667
:10632000B83147F6A8109A66DA661A675A679A670C
:10633000DA67C3F88020824A11668249116401F548
:106340000041116442F2010111634FF4E811C2F8F7
:10635000001110217C4A5A6103F57C2300225A6106
:106360009A61DA611A625A629A62DA621A635A634D
:106370009A63DA631A645A649A64DA641A655A652D
:106380009A65DA651A665A669A66DA661A675A670D
:106390009A67DA67C3F88020C3F88420C3F888209E
:1063A000C3F88C20C3F89020C3F89420C3F8982039
:1063B000C3F89C20C3F8A020C3F8A420C3F8A820E9
:1063C000C3F8AC20C3F8B01041F21001C3F8B420F8
:1063D000C3F8B820C3F80412C3F80812C3F80C12AB
:1063E000C3F81012C3F81412C3F81812C3F81C1221
:1063F000C3F82012C3F82412C3F82812C3F82C12D1
:10640000C3F83012C3F83412C3F83812C3F83C1280
:10641000C3F84012C3F84412C3F84812C3F84C1230
:10642000C3F85012C3F85412C3F85812C3F85C12E0
:10643000C3F86012C3F86412C3F86812C3F86C1290
:10644000C3F87012C3F87412C3F87812C3F87C1240
:10645000C3F88012C3F88412C3F88812C3F88C12F0
:10646000C3F89012C3F89412C3F89812C3F89C12A0
:10647000C3F8A012C3F8A412C3F8A81203F5782336
:106480003249196081219960D9603149196101F15E
:106490000071596101F10071996101F10071D961D7
:1064A0002C4919622C4959622C4999622C49D962AC
:1064B00021211963586040F63170186429485864E6
:1064C000294898642948D864C3F880102849C3F83B
:1064D00084100221C3F89410C3F898204FF00042B2
:1064E000C3F89020234AC3F89C20DA6BD207FCD56E
:1064F0004FF00042C3F890201F4AC3F89C201F4B66
:10650000D96BC807FCD54FF00041C3F89010C3F811
:106510009C20DA6BD107FCD53322C3F8A0204FF0C2
:106520000042C3F89020164AC3F89C20134BDA6B44
:10653000D207FCD5134ADA64704700BF00C00F4091
:1065400000800D400600DC05400D01000400001035
:106550001B00008021000090190000A0170000A877
:106560001B0000A92229650020090100080A21500A
:10657000888888000F005AA50C005AA500002F40FB
:106580000A005AA5090A2150012814BF064B074BDF
:10659000186838B1EFF305820AB1ACF02DBE114690
:1065A000ACF0ACBD704700BFF0550380EC550380E4
:1065B000304A3149D2F8883043F47003C2F8883049
:1065C0000B892E4A23F001031B041B0C0B8113893A
:1065D00023F001031B041B0C13810B88580705D5FE
:1065E0000B8823F004031B041B0C0B8013885B0730
:1065F00005D5138823F004031B041B0C1380204BC8
:106600001A6890042FD51F4A5A604FF6FF729A609D
:106610001A6822F0A00242F020021A604FF0E02334
:106620001A69D10703D51A6922F001021A61114BC8
:106630005A69920315D45A6912F4003211D1BFF38A
:106640004F8FBFF36F8FC3F85022BFF34F8FBFF34D
:106650006F8F5A6942F400325A61BFF34F8FBFF314
:106660006F8FFFF759BE4CF220525A604DF6281238
:10667000CAE700BF00ED00E000800B4000000D40C5
:1066800000C00B4020C528D908480068006880F386
:1066900008884FF0000080F3148862B661B6BFF33B
:1066A0004F8FBFF36F8F00DF00BF000008ED00E0E9
:1066B000DFF80C00016841F47001016070470000D0
:1066C00088ED00E04FF0200383F31188BFF36F8F54
:1066D000BFF34F8FFEE7000008B54FF0200383F3B0
:1066E0001188BFF36F8FBFF34F8F074A13680133D1
:1066F000012B136007D14FF0E023D3F8043DDBB248
:106700000BB1FFF7DFFF08BDC0940280054A08B552
:1067100013680BB9FFF7D6FF013B13600BB983F386
:10672000118808BDC094028008B5EFF305830F2BD4
:1067300007D90E4A9B5C0E4A12789A4201D9FFF79C
:10674000C1FF4FF0E0230B4AD3F80C3D126803F46D
:10675000E063934208D94FF0200383F31188BFF31D
:106760006F8FBFF34F8FFEE708BD00BFF0E300E07F
:10677000E8550380E4550380002307B501930A4BD5
:106780001B68013301D0FFF79DFF4FF0200383F317
:106790001188BFF36F8FBFF34F8F019B002BFCD08D
:1067A00003B05DF804FB00BFC094028010B508B9C7
:1067B000FFF788FF00230A4A52F83310DC008842B2
:1067C00009D1084A002142F8331022445160BDE843
:1067D00010401DF03BB80133082BEDD1F7E700BFA7
:1067E000A05503809C550380034608461A6C10B4DC
:1067F00062B1DC68996814448C42DC605DF8044B3B
:1068000024BF1968D960D96837F148BF5DF8044BD7
:1068100070470000F8B5FFF75FFF90F84550044659
:10682000174E6DB20127002D14DCFF23144E0127F3
:1068300084F84530FFF76AFFFFF74EFF94F84450A5
:106840006DB2002D11DCFF2384F84430BDE8F84020
:10685000FFF75CBF636A002BE7D0206BF1F070FF9D
:1068600000B13760013D6DB2DDE72369002BEAD04E
:10687000E069F1F065FF00B13760013D6DB2E0E71E
:106880001855038008B5FFF727FF806BFFF73EFF21
:10689000B0FA80F0400908BD024A13680133136062
:1068A000704700BF145503802DE9F84FFFF714FF20
:1068B0004D4B1A6842B94FF0200383F31188BFF3A0
:1068C0006F8FBFF34F8FFEE71A68013A1A601B689B
:1068D00023B10020FFF71AFFBDE8F88F434A126882
:1068E000002AF6D042480125424C1426424A434F22
:1068F000DFF810C154E0C368DB68D3F828E003F187
:106900001809D3E90718C1F80880C8F80410DEF8A0
:10691000041049454FF0000108BFCEF80480996289
:10692000DEF800100139CEF80010D3F814E003F1BE
:106930000409D3E90218C1F80880C8F80410DEF889
:1069400004104945DEF8001001F1FF3108BFCEF810
:106950000480D4F80080CEF80010D3F82CE005FABB
:106960000EF141EA080106FB0EF802EB080A21606D
:10697000DAF80410D1F808B09960C3F80CB0CBF87D
:106980000490C1F8089052F80810C3F814A001311F
:1069900042F808103968C96A8E4501D9CCF8005010
:1069A00001680029A7D10BB1FCF7A4FB144D2C689A
:1069B00044B1144E0127FCF7AFFB00B13760013C36
:1069C000F9D12C600F4B1B68002B82D00B4B4FF082
:1069D00080521B684FF0E023C3F8042DBFF34F8FA4
:1069E000BFF36F8F012075E714550380F8540380BF
:1069F000E4540380945503801C550380985503800C
:106A0000E054038018550380184B1A68184B10B5D2
:106A100012B101221A6010BD1A60164B1A68B2FA40
:106A200082F2D2B214231449C2F11F025343CC584C
:106A3000C81844B94FF0200383F31188BFF36F8F58
:106A4000BFF34F8FFEE74468083364680B449C42F1
:106A5000446004BFC3684360142303FB02114B6806
:106A6000DA68064B1A601B68D5E700BF145503802F
:106A700018550380945503801C5503809855038056
:106A8000054B1B6833B1054B1868B0FA80F040091C
:106A90004000704701207047FC5403801455038068
:106AA00008B5FFF7EDFF012813D04FF0200383F363
:106AB0001188BFF36F8FBFF34F8FFCF72DFB28B109
:106AC0004FF0E0234FF08052C3F8042D002383F3EE
:106AD0001188BFF34F8F08BDF8B5FFF7FDFD0B68B8
:106AE000DFF844C05A1CDCF8004018D00D4E056891
:106AF00037684268BD4207D0944205D30023012085
:106B00000B60FFF703FEF8BDA71A9F42F6D21B1BCE
:106B100013440B6033680360DCF8003043600020EE
:106B2000EFE700BFE0550380DC55038008B538F17E
:106B30007DFF582303604FF0FF3008BD08B538F1E2
:106B400075FF582303604FF0FF3008BD08B538F1DA
:106B50006DFF582303604FF0FF3008BD08B538F1D2
:106B600065FF582303604FF0FF3008BD08B538F1CA
:106B70005DFF582303604FF0FF3008BD08B538F1C2
:106B800055FF582303604FF0FF3008BD08B538F1BA
:106B90004DFF582303604FF0FF3008BD00F108039C
:106BA0004FF0FF3243600361C0E90223002303601A
:106BB0007047F8B5074648430D46164650301CF05E
:106BC0006FFD044620B32DB300F150032360C4E9E8
:106BD0000F75FFF781FD2168D4E90F3261605343DF
:106BE000C8189B1AA06019440020FF23E160A0632D
:106BF00004F1100084F8443084F84530FFF7CEFFEC
:106C000004F12400FFF7CAFFFFF780FD84F84C6011
:106C10002046F8BD0346D9E702460021012010B501
:106C2000FFF7C7FF044630B10022114682600260C0
:106C3000C260ACF063FA204610BD000038B5194DB3
:106C4000FFF74AFD2C6844BB17490846FFF7A6FF2B
:106C50001648FFF7A3FF164B224619601021154B6B
:106C600018600A20FFF7A5FF2860B0B1124B22463A
:106C700019465D68A84205D101EBC2040F4BC4E977
:106C800000300AE01CB91D68002D08BF1C46013207
:106C90000833082AEDD1002CF0D1BDE83840FFF7C9
:106CA00035BD00BFB45403809854038084540380DE
:106CB000B8540380AC5403809C550380A03B1670ED
:106CC0000369D0E901128A6051605968814208BFA6
:106CD0005A6000220261186801381860704700008D
:106CE0002DE9F8431546026C0446876B002A57D1FC
:106CF0000368002B61D1856835B900200023A360AB
:106D00000137A763BDE8F883374B1B689D4208D065
:106D10004FF0200383F31188BFF36F8FBFF34F8FC2
:106D2000FEE76B6D43B94FF0200383F31188BFF387
:106D30006F8FBFF34F8FFEE7D5F82C90013B2E6D80
:106D40006B65B145D9D0002BD7D105F10408404679
:106D5000FFF7B6FF254B30B901211A6801FA09F196
:106D600022EA01021A60C6F1060201201968AA612E
:106D700000FA06F2EE620A431A6014221C4B5643D4
:106D800099194A68D2F808C0AA60C5F80CC0CCF8B6
:106D90000480C2F808809A59696102449A51ADE7AB
:106DA0006DB9406837F17AFC6368226C1344A268BD
:106DB0009342636024BF236863600020A0E7C0683B
:106DC00037F16CFC226CE36851429B1A22689342B3
:106DD000E3603EBFA3685B18E360022DEDD10FB105
:106DE000013FEAE738468BE79855038094550380C6
:106DF0001C55038070B5FFF76FFC04462F4D00B99A
:106E00002C68261D3046FFF75BFF60B9E06A14234B
:106E10002B4A4343D35833B92A4901220B68824095
:106E200023EA02030B60A36A1BB104F11800FFF709
:106E300047FF254843689A68A360E26056609E60F9
:106E4000036860610133036094F87030012B02D154
:106E5000002384F870301D4EFFF758FC33682BB1C7
:106E6000FFF73AFCFCF746F9FFF750FC2B68A3420A
:106E700017D13368B3B1164B1B6843B14FF02003F1
:106E800083F31188BFF36F8FBFF34F8FFEE74FF08F
:106E9000E0234FF08052C3F8042DBFF34F8FBFF3B0
:106EA0006F8F70BD0B4A11680268914201D12B604F
:106EB000F7E7BDE87040FFF7A7BD00BF9855038016
:106EC0001C5503809455038000550380FC540380B7
:106ED00014550380F854038080B5154C154F164E99
:106EE00023687BB9154B1B68012B09D94FF0E023B0
:106EF0004FF08052C3F8042DBFF34F8FBFF36F8F55
:106F000030BFECE7FFF7E8FBFB68DD68281DFFF703
:106F1000D7FE3368013B33602368013B2360FFF7F2
:106F2000F5FB286B1CF092FC28461CF08FFCD7E781
:106F3000BC540380C0540380F85403801C55038064
:106F40002DE9F843224B0646224C0F461D68224B82
:106F5000D3F80080214BD3F8009020680430FFF76D
:106F6000AFFE40B922681E49D06A01220B688240F8
:106F700023EA02030B60731C14D19FB1194B2168E3
:106F80005A688A6090682168C8602168043141604D
:106F9000216804319160226853611A6801321A60D5
:106FA000BDE8F8832368AD1921685D6001F1040133
:106FB00004D34846BDE8F843FCF778B94046FCF7EF
:106FC00075F9094B1A68AA42EAD91D60E8E700BFC3
:106FD000DC55038098550380DC540380D85403802B
:106FE0009455038000550380D454038008B550B9EC
:106FF0004FF0E0234FF08052C3F8042DBFF34F8FC2
:10700000BFF36F8F08BDFFF747FC074B1B68012BD1
:1070100001D0FFF757FB0021FFF792FFFFF744FC79
:107020000028E5D0EEE700BF14550380064B10B5ED
:107030000C4619681831FCF739F920460121BDE8E2
:107040001040FFF77DBF00BF98550380F0B585B0B5
:107050000E460446019240B94FF0200383F3118895
:10706000BFF36F8FBFF34F8FFEE751B9036C43B18E
:107070004FF0200383F31188BFF36F8FBFF34F8F5F
:10708000FEE7FFF7FDFC50B9019B43B14FF0200331
:1070900083F31188BFF36F8FBFF34F8FFEE7FFF7C6
:1070A0001BFBA56BD5B131462046FFF79DFB013D8B
:1070B0002369A5636BB1E069F1F042FB48B14FF081
:1070C000E0234FF08052C3F8042DBFF34F8FBFF37E
:1070D0006F8F0120FFF71AFB05B0F0BD019B002B5D
:1070E00040D02B4B2F461B6802932A4B1B680393FF
:1070F000FFF70CFBFFF7D0FBFFF7EEFA94F84430F4
:10710000FF2B01D184F8447094F84530FF2B01D156
:1071100084F8457001A902A8FFF7F8FAFFF7DCFC34
:1071200050BB2046FFF7AEFB00B3019904F12400E9
:10713000FFF77CFF2046FFF76DFBFFF7B5FB48B973
:107140004FF0E0234FF08052C3F8042DBFF34F8F70
:10715000BFF36F8FFFF7C0FAA56B002DA3D1019B82
:10716000002BC5D1FFF7D2FA0020B5E72046FFF784
:1071700051FBFFF799FBEDE72046FFF74BFBFFF7CD
:1071800093FB2046FFF77EFB0028E3D0ECE700BF2F
:10719000E0550380DC5503807FB50E46044601921E
:1071A00040B94FF0200383F31188BFF36F8FBFF313
:1071B0004F8FFEE7FFF764FC50B9019B43B14FF0DE
:1071C000200383F31188BFF36F8FBFF34F8FFEE768
:1071D000FFF782FAA56BD5B131462046E568FFF787
:1071E00003FB636AE5606BB1206BF1F0A9FA48B16B
:1071F0004FF0E0234FF08052C3F8042DBFF34F8FC0
:10720000BFF36F8F0120FFF781FA04B070BD019BBF
:10721000002B3FD02A4B1B6802932A4B1B68039319
:10722000FFF774FAFFF738FBFFF756FA94F844308B
:10723000FF2B01D184F8445094F84530FF2B01D145
:1072400084F8455001A902A8FFF760FAFFF744FC53
:1072500050BB2046FFF716FB00B3019904F1240050
:10726000FFF7E4FE2046FFF7D5FAFFF71DFB48B90C
:107270004FF0E0234FF08052C3F8042DBFF34F8F3F
:10728000BFF36F8FFFF728FAA36B002BA4D1019BEC
:10729000002BC5D1FFF73AFA0020B6E72046FFF7EA
:1072A000B9FAFFF701FBEDE72046FFF7B3FAFFF766
:1072B000FBFA2046FFF7E6FA0028E3D0ECE700BF30
:1072C000E0550380DC5503800E4B1B68DB6870B50E
:1072D000DC6805460E46201DFFF7F2FC94F82830C6
:1072E0005A0709D5324629462046FCF715F8236A85
:1072F0002046BDE87040184723F0010384F8283089
:10730000F5E700BFB854038010B5084C23681A682D
:1073100022B9074A11681360216010BDDB684FF085
:10732000FF311868FFF7D0FFF0E700BFB8540380C3
:10733000AC5403808FB54FF00009784F784B396813
:107340001B68DFF8E8811E68DFF8E4A1002E4DD14C
:10735000FFF7A2FAD8F80050A94254D8714B3D600B
:107360001B681968B1FA81F14909DAF80040FFF7A2
:10737000B3F994F84430FF2B01D184F8449094F889
:107380004530FF2B01D184F84590FFF7BFF9A36B7F
:10739000DBB9654BA26A1868D2F808C0C2611868E8
:1073A000C0F820C018681830CCF8040018681B68B2
:1073B0001830906004F124029A62636A01336362B8
:1073C000002953D1701BFFF7BBFD2046FFF722FABF
:1073D000FFF76AFAE0B94FF0E0234FF08052C3F8AC
:1073E000042DBFF34F8FBFF36F8F11E0DB681E6872
:1073F000FFF752FAD8F80050A94204D8AE423D60D7
:107400002DD90021B1E7FFF77FFF3D60FFF74CFA70
:1074100010220021684638F101FC00226946DAF8A2
:107420000000FFF713FE002888D0009B0298002B75
:107430001FDB029C63691BBBD8F800503B68AB4262
:1074400001D9FFF761FF009B3D60013B082BE4D8A9
:10745000DFE803F01A1A3C435C1A1A3C4300FFF7BA
:1074600023FA29463046FFF72FFFD1E74FF0FF30D0
:10747000A9E7019B03999847009B002BCDDBD8E738
:10748000201DFFF71DFCD7E794F828302A46A6698F
:10749000204643F0010384F82830019B1E44314606
:1074A000FBF71CFF0028B8D094F82830590708D5FE
:1074B0002A4631462046FBF72FFF236A204698478D
:1074C000ABE723F0010384F82830F6E794F828307E
:1074D00023F0010384F828309FE794F828300199BD
:1074E00043F00103A16184F8283041B94FF0200333
:1074F00083F31188BFF36F8FBFF34F8FFEE72B46E7
:107500002A4629442046FBF7E9FE86E794F828300E
:107510009A07DDD420461CF099F97EE7B054038029
:10752000B8540380AC54038098550380DC55038025
:10753000B4540380B0EEC07ADFED257A08B5B4EE1E
:10754000677A2DED048BF1EE10FAF0EE408AB0EE82
:10755000608A3ADCB0EEE07AB4EE677AF1EE10FAC7
:1075600033DCB5EEC00AF1EE10FAF5EEC00A4CBFFE
:1075700001220022F1EE10FA4CBF012300239A42AF
:1075800023D130EE600A33F1F5F9B0EE409AB0EE57
:10759000680A33F1EFF9F0EE408AB0EE480A33F1B1
:1075A000E9F9F0EE400AB0EE680A33F1F5FDDFEDDF
:1075B000097A60EE277AB4EEE79AF1EE10FA94BFFA
:1075C00001200020BDEC048B08BD0020FAE700BFBD
:1075D000FFFF7F7F17B7D138B4EE410B08B5F1EE4E
:1075E00010FA2DED068BB0EE409BB0EE418B43D6EA
:1075F000B0EEC07B9FED226BB4EE467BF1EE10FA4D
:107600003ADCB0EEC17BB4EE467BF1EE10FA33DC2F
:10761000B5EEC00BF1EE10FAB5EEC01B4CBF012267
:107620000022F1EE10FA4CBF012300239A4223D12D
:1076300030EE410B32F140FCB0EE40ABB0EE490B06
:1076400032F13AFCB0EE409BB0EE480B32F134FC24
:10765000B0EE401BB0EE490B31F1CAFF9FED0A7B43
:1076600020EE077BB4EEC7ABF1EE10FA94BF012019
:107670000020BDEC068B08BD0020FAE7AFF30080C8
:10768000FFFFFFFFFFFFEF7FBBBDD7D9DF7CDB3DF7
:107690000268032A06D922F003031968C9075CBFF0
:1076A00041685960416831B10B6822F0030203F070
:1076B000030313430B6000234360036803F00303D9
:1076C0000360704738B5114B05460446403045F815
:1076D000343BFFF7DDFF2846F0F0B8F804F1300046
:1076E000F0F0F4FC04F12800F0F07EFF04F120003B
:1076F000F0F07AFF04F11800F0F076FF044B20461A
:10770000236021F0EBF9204638BD00BFEC5916701C
:10771000D859167010B50446FFF7D4FF58212046FB
:1077200031F166F9204610BD70B5314B00F25C4571
:10773000044603602846F0F089F804F5816628467F
:1077400004F21445854203D00C38FFF7A1FFF9E796
:107750003046F0F07BF804F57B70F0F003FC04F5A4
:107760007470F0F0FFFB04F53670FBF7C1FE04F512
:10777000F070FBF7BDFE04F5A070FBF7E1FE04F529
:107780009470F0F031FF04F58C70F0F02DFF04F5EB
:107790008470F0F029FF04F1F800F0F025FF04F107
:1077A000F000F0F021FF04F1E800F0F01DFF04F11B
:1077B000E000F0F019FF04F1D800F0F015FF04F13B
:1077C000C800F0F011FF04F1C000F0F00DFF04F16B
:1077D000B800F0F009FF04F1B000F0F005FF04F18B
:1077E000A000F0F001FF2046FBF7AAFE204670BD86
:1077F0008457167010B50446FFF796FF4FF4956155
:10780000204631F1F5F8204610BD0000124B10B5AE
:1078100004460360D0F86808F0F0F8FBD4F85C0880
:10782000F0F0F4FBD4F85008F0F0F0FB04F5006041
:10783000F0F06CFF04F55670FFF776FF04F5447026
:10784000F0F064FF04F53B70F3F074FE20469DF009
:1078500037F8204610BD00BF8C4C167010B504469A
:10786000FFF7D4FF4FF40761204631F1C1F82046FD
:1078700010BD000038B500F517552F4B04463435C0
:10788000036000F51850FFF703FF284604F5005584
:10789000EFF0DCFFD5F8F005F0F0B8FBD5F8E40523
:1078A000F0F0B4FBD5F8D805F0F0B0FB04F51750B4
:1078B0000830F0F099FE04F515501030F0F0B6FEE7
:1078C00004F514500830F0F021FF04F51350F0F0E7
:1078D0001DFF04F512503830F0F0F8FB04F510509D
:1078E000103020F0F5F904F5FC7011F031FD04F5CD
:1078F000F470FDF73BFB04F5D070F0F007FF04F5E2
:107900009470F0F093FE04F58C70F0F0B7FB04F582
:107910008070F0F0B3FB04F1E800F0F0AFFB04F18D
:10792000D000F0F0ABFB04F1A800F3F003FE20461A
:1079300020F0CEF9204638BDB041167010B504468F
:10794000FFF798FF42F21861204631F151F82046C6
:1079500010BD000038B53B4B00F5A345044603605D
:1079600005F17C007035FFF793FE284604F5A3452A
:10797000EFF06CFF05F158004C35FFF789FE284603
:1079800004F5A045EFF062FFD5F8C801F0F03EFB2A
:10799000D5F8BC01F0F03AFBD5F8B001F0F036FBB9
:1079A000D5F8A401F0F032FBD5F89801F0F02EFBE9
:1079B00004F5A3400830F0F017FE04F5A2401030A3
:1079C000F0F034FE04F5A1404830F0F09FFE04F5DD
:1079D000A140F0F09BFE28462030FBF763FE04F543
:1079E0009E40783020F074F904F5307011F016FDE7
:1079F00004F52C70FDF7D4FA04F5CC70FBF774FE97
:107A000004F5A870F0F082FE04F59870F0F028FB01
:107A100004F58C70F0F032FB04F58070F0F02EFB72
:107A200004F1E800F0F02AFB04F1C400F0F018FBC8
:107A300004F19C00F3F07EFD2046FBF781FD20461B
:107A400038BD00BF403D167010B50446FFF782FFF9
:107A500045F21821204630F1CBFF204610BD000032
:107A600038B52E4B00F5A0450446036005F118001B
:107A70000C35FFF70DFE284604F59F45EFF0E6FEB6
:107A800004F5A0439868F0F0C1FA04F58043D3F8F8
:107A9000FC0FF0F0BBFA05F15C005035FFF7F8FD84
:107AA0002846EFF0D3FE04F59F404830F0F09CFDEF
:107AB00004F59E405030F0F0B9FD04F59E400830CA
:107AC000F0F024FE04F59D404030F0F01FFE04F578
:107AD0009C40183020F0FCF804F5B07011F004FD63
:107AE00004F5A870FDF776FA04F58470F0F00EFE48
:107AF00004F1F400F0F0C2FA04F1DC00F0F0BEFA98
:107B000004F1C400F0F0BAFA04F19C00F3F012FDA5
:107B10002046FBF715FD204638BD00BF483C1670D7
:107B200010B50446FFF79CFF45F23001204630F1C6
:107B30005FFF204610BD000030B587B00D4C0546F4
:107B400004930A9B0291059323688DF80C2001335E
:107B5000B3F57A7F236006DD00232021ED201A464D
:107B600000932EF063FD2B6802A898470023236042
:107B700007B030BD8054038003689A0705D5032BF6
:107B800003D923F00303181D704723F00203036099
:107B90007047036813F0020018BF23F0030070471A
:107BA0001FB50246FFF7F5FF0146039040B103AB56
:107BB000009313460622FFF7BFFF05B05DF804FBF4
:107BC000106800F00100F8E708B50246FFF7E1FF92
:107BD00010B1106800F0010008BDF7B505460C466D
:107BE000FFF7DEFF07462846FFF7D3FFA042064611
:107BF0001CD08CB9E6B92846FFF7BEFF0368032BFB
:107C000063601FD844F00304394628462C6003B053
:107C1000BDE8F04020F031BE002305222146204679
:107C200000932B46FFF788FF0028E3D003B0F0BD98
:107C30002B460322314630460094FFF77DFF002893
:107C4000D9D0F3E723F0030203F003031168C90757
:107C50005CBF211D51600360D4E710B50246FFF7F9
:107C600098FF98B11368416803F0010321F0030104
:107C70000B4313604368032B08D923F0030103F07F
:107C800003030C68E40758BF4A60436010BD10B599
:107C900024220021044637F1C1FF4FF07E532046D5
:107CA000236023612362002384F8243010BD70B563
:107CB0008AB00C4606466846FFF7E9FF2368694626
:107CC0002046DB68354698476C46002345F8083B5C
:107CD0000FCC0FC50FCC0FC594E8030045F8040B7B
:107CE000304629700AB070BD10B52DED028BF0EE54
:107CF000608ADFED270AB0EE408A0446FFF71AFCDF
:107D000060BB94F8243094ED067A062BD4ED077A04
:107D100030D9D4ED025AD4ED006A94ED056AE5EE4F
:107D2000886AC4ED006AD4ED036AE6EE086AC4ED21
:107D3000036AD4ED086AA6EE887AE6EEA87A84EDA6
:107D4000067A94ED017AA5EEA87A84ED017A94ED95
:107D5000047AA6EE287A84ED047A14E0B0EE680A7C
:107D6000DFED0B0AFFF7E6FB0028CAD02046BDEC8A
:107D7000028B10BD012B38EE078A78EEA77A38BF48
:107D8000012384ED068AC4ED077A84F82430EDE7F8
:107D90000000000010B52DED028BB0EE608A0446A5
:107DA000F7EE000AF0EE408AFFF7C4FB20BB94F820
:107DB000243094ED067AD4ED077A012B28EE877AE9
:107DC00068EE277A24D8C4ED008A84ED067A84ED23
:107DD000048AC4ED077AF0EE480AB0EE680AFFF7AD
:107DE000A9FBC0F1030094F82430C0B2984238BF18
:107DF000184684F8240007E0F7EE000AB0EE480ABF
:107E0000FFF798FB0028D2D02046BDEC028B10BDB6
:107E100094ED006A032BD4ED046A28EE866A68EEBE
:107E2000266A84ED006A04D884ED067AC4ED046AFB
:107E3000CFE794ED036A042B84ED067A94ED017A82
:107E400026EE286AC4ED046A27EE087AC4ED077AA4
:107E500084ED036A84ED017ABDD1F0EE480AB0EEFC
:107E6000680AFFF767FB0028B5D1062384F82430A1
:107E7000CAE7DFB5D1E90267044622EAE2720123CC
:107E800069460292ADF80C30CDE90067B0F034FCE1
:107E9000204604B0D0BD836823B14268013B0A602C
:107EA00041608360704703298368CABF0439406812
:107EB000006803FB0100704770B5C46805460E46B4
:107EC000002C07DD013C21462846FFF7ECFFB047B8
:107ED000013CF8D270BD000010B50446FFF7ECFF7E
:107EE0000621054838F030FD036821689B689847F3
:107EF0000023236010BD00BFBC94028010B504466F
:107F0000FFF7EAFF0023C4E90333636110BD38B50E
:107F1000044600680D46884202D0F0F077F82560EC
:107F200038BD37B50446FFF74FFE251D70B120461A
:107F3000FFF72FFE014648B1234600220095FFF7C8
:107F4000FBFD18B1236823F001032360204620F0D5
:107F500053FD284603B030BD37B504461C30FFF74B
:107F6000E0FFB0F9005004F12400FFF7DAFF00232E
:107F7000ADB2028865F30F0362F31F43184603B0E6
:107F800030BD82B002B0FFF7E7BF10B502F1340098
:107F90000C46FFF7C6FF0368236010BD10B502F161
:107FA0002C000C46FFF7BDFF0368236010BD7FB5B2
:107FB00004460D46FFF7EDFD014640B12346012280
:107FC0000095FFF7B9FD68BB2046FFF746FE226823
:107FD000204642F001032360FFF7DBFD10B122F0E1
:107FE000010222600023261D0DF10E0229468DF8A4
:107FF0000E3030460DF10F03B0F05EFB9DF80F30F0
:108000001BB129463046EBF095FE9DF80E304BB182
:108010002046FFF7C5FD0146204604B0BDE870408C
:1080200020F02BBC04B070BD036823F003009B0755
:10803000FAD1FFF7BCBF10B50446FFF7AAFD18B18F
:10804000236823F0010323600B6862689A4209D019
:1080500020466360FFF7A4FD01462046BDE81040BE
:1080600020F00BBC10BD37B504460D46FFF791FD5F
:10807000014640B1234601220095FFF75DFD68B936
:108080002046FFF7EAFD23682946204643F0010316
:10809000236003B0BDE83040FFF7CDBF03B030BD73
:1080A000264A136813F0010370B50C4688B000F13E
:1080B0000406234D05D12B6001232248136036F1BD
:1080C0008CFD2D680DB908B070BD2B6823F003033B
:1080D0009E422ED1012301A82370F0F089F80023DD
:1080E000694602A8CDE90233CDE90433CDE9063370
:1080F000A3690093FFF7B7FFE369694604A80093FB
:1081000021F0D2FB236A694606A8009321F0CCFB3C
:108110006368052B0FD101A9E868EAF023FD06A8E2
:10812000F0F062FA04A8F0F05FFA02A8F0F05CFA4E
:10813000C9E76D68C6E701A92869EEE77C540380AA
:108140007854038031340270F7B5074614460D1F8A
:1081500002EB4306B44201D103B0F0BD55F8040F61
:10816000431C07D0B4F9003001A907EB800001934C
:10817000FFF779FF0234EDE737B504460D46FFF708
:108180000FFD90B92046FFF704FD014630B929469E
:10819000204603B0BDE83040FFF74DBF2346022222
:1081A0000095FFF7C9FC0028F1D003B030BD37B50A
:1081B00004460D46FFF7EDFC18B1236823F00103D8
:1081C00023600DF106030DF10702294604F10800B2
:1081D000AAF044FE9DF806301BB1D5E90023C4E99E
:1081E00002239DF807304BB12046FFF7D9FC01462A
:1081F000204603B0BDE8304020F03FBB03B030BDA7
:10820000036813B504464BB15B68834206D0002374
:108210008B2123201A4600932EF008FA23680BB115
:1082200062685A60626802B113600023C4E90033D7
:1082300002B010BD38B51D4B00F52815044603608B
:1082400005F53870F3F076F905F53070F3F072F952
:1082500005F52E70F0F0C8F905F52670F3F06AF90F
:1082600005F51E70F3F066F905F51A70EFF041FFA1
:1082700004F5A47010F0E4FD04F58070F0F046FA07
:1082800004F1F000EFF0FAFE04F1D800EFF0F6FE92
:1082900004F1BC00FFF7B4FF04F19C00F3F04AF9CD
:1082A0002046FBF74DF9204638BD00BFDC5A16705A
:1082B00010B50446FFF7BEFF0249204630F198FB97
:1082C000204610BD00032A001C4B10B50446036075
:1082D00000F5A470FFF794FF04F1F000FFF7F2F946
:1082E00004F1E000F0F080F904F1D800F0F07CF93E
:1082F00004F1D400EFF0EAFE04F1D000EFF01FFE2D
:1083000004F1CC00EFF01BFE04F1C800EFF017FE03
:1083100004F1C400EFF013FE04F1C000EFF00FFE13
:1083200004F1B000F0F060F904F1A000F0F05CF9A5
:108330002046FBF705F9204610BD00BFA059167076
:1083400010B50446FFF7C0FF4FF4B071204630F17E
:108350004FFB204610BD0000224B10B504460360C1
:1083600000F5C460F0F0D2F904F5C360EFF0AEFEA2
:1083700004F59F60FBF7F0F904F56670FFF7A4FFC2
:1083800004F50E70FFF7A0FF04F5E070F0F04EF971
:1083900004F5BC70F0F0BAF904F5B270EFF06EFEBF
:1083A00004F5A670EFF06AFE04F59870FFF728FF59
:1083B00004F58A70EFF054FE04F1FC00EFF05EFE6D
:1083C00004F1E400EFF05AFE04F1C800FFF718FFD3
:1083D00004F1A800F3F0AEF820461FF079FC204627
:1083E00010BD00BF6859167010B50446FFF7B4FF02
:1083F0004FF4CD61204630F1FBFA204610BD00005D
:108400001E4B10B50446036000F59860EFF05EFE69
:1084100004F55870FFF758FF04F51070FBF79CF94E
:1084200004F5E470F0F002F904F5C070F0F06EF9B4
:1084300004F5B670EFF022FE04F5AA70EFF01EFE10
:1084400004F59C70FFF7DCFE04F59270FFF7D8FE90
:1084500004F58870FFF7D4FE04F1F400EFF000FE9D
:1084600004F1D000EFF0FCFD04F1A800F3F062F895
:1084700020461FF02DFC204610BD00BFA4561670EC
:1084800010B50446FFF7BCFF4FF49961204630F168
:10849000AFFA204610BD0000484B10B504460360FB
:1084A000D0F8B408EFF0B2FDD4F8A808EFF0AEFDB4
:1084B000D4F89C08EFF0AAFDD4F89008EFF0A6FDE0
:1084C000D4F88408EFF0A2FDD4F87808EFF09EFD10
:1084D000D4F86C08EFF09AFDD4F86008EFF096FD40
:1084E000D4F85408EFF092FDD4F84808EFF08EFD70
:1084F000D4F83C08EFF08AFDD4F83008EFF086FDA0
:1085000004F60800F3F016F804F5FD60F3F012F835
:1085100004F5FC60F0F068F804F5FB60F0F064F836
:1085200004F5FA60F0F060F804F5F960F0F05CF83A
:1085300004F5EA60F0F07AF804F5B160FBF702FAAE
:1085400004F59C601FF0C4FB04F57070FBF704F9A0
:1085500004F51870FFF7B8FE04F50670F0F0D6F8D1
:1085600004F5D070F0F062F804F5C670EFF086FD07
:1085700004F5BA70EFF082FD04F5AE70EFF07EFD09
:1085800004F5A270EFF07AFD04F59070EFF068FD4D
:1085900004F58270FFF734FE04F1F400EFF06EFD95
:1085A00004F1D000EFF05CFD04F1A800F2F0C2FF8E
:1085B00020461FF08DFB204610BD00BF20561670D0
:1085C00010B50446FFF768FF40F6B801204630F1C9
:1085D0000FFA204610BD0000084B10B5044603609A
:1085E000D0F8CC08EFF012FDD4F8C008EFF00EFD83
:1085F0002046FFF751FF204610BD00BFE85516701A
:1086000010B50446FFF7E8FF4FF40D61204630F146
:10861000EFF9204610BD000038B58E4B00F58055AF
:1086200004460360D5F80002EFF0F0FCD5F8F40141
:10863000EFF0ECFCD5F8E801EFF0E8FCD5F8DC0150
:10864000EFF0E4FCD5F8D001EFF0E0FCD5F8C40180
:10865000EFF0DCFCD5F8B801EFF0D8FCD5F8AC01B0
:10866000EFF0D4FCD5F8A001EFF0D0FCD5F89401E0
:10867000EFF0CCFCD5F88801EFF0C8FCD5F87C0110
:10868000EFF0C4FCD5F87001EFF0C0FCD5F8640140
:10869000EFF0BCFCD5F85801EFF0B8FCD5F84C0170
:1086A000EFF0B4FCD5F84001EFF0B0FCD5F83401A0
:1086B000EFF0ACFCD5F82801EFF0A8FCD5F81C01D0
:1086C000EFF0A4FCD5F81001EFF0A0FCD5F8040100
:1086D000EFF09CFCD5F8F800EFF098FCD5F8EC0032
:1086E000EFF094FCD5F8E000EFF090FCD5F8D40062
:1086F000EFF08CFCD5F8C800EFF088FCD5F8BC0092
:10870000EFF084FCD5F8B000EFF080FCD5F8A400C1
:10871000EFF07CFC04F58450EFF0C1FF04F58350CA
:108720001830EFF061FF04F583501030EFF05CFF7C
:1087300004F583500830EFF057FF04F58350EFF055
:1087400053FF04F582501830EFF04EFF04F58250CD
:108750001030EFF049FF04F582500830EFF044FF8D
:1087600004F58250EFF040FF04F6C870EFF05EFFB2
:1087700004F66860FFF7A8FD04F64850FAF7ECFF2E
:1087800004F54A601FF0A4FA04F53860FAF7E4FF34
:1087900004F52C60FBF7EAFE04F6F800FBF7D2F8CC
:1087A00004F5E660FBF7CEF804F5C260FAF7D4FFF3
:1087B00004F59E60FAF7D0FF04F59460FAF73CFFE9
:1087C00004F56070FAF7C8FF04F53C70FAF718FF7B
:1087D00004F52A70EFF09AFF04F50C70EFF026FF15
:1087E00004F50770EFF04AFC04F50170EFF046FC69
:1087F00004F5F670EFF042FC04F5EA70EFF03EFC91
:1088000004F5D870EFF02CFC04F5C670EFF028FCEE
:1088100004F5B470EFF024FC04F5A270EFF020FC36
:1088200004F59670EFF02AFC04F58470EFF018FC64
:1088300004F1E400EFF014FC04F1C800FFF7E0FCE1
:1088400004F1A800F2F076FE20461FF041FA20461F
:1088500038BD00BFB055167010B50446FFF7DCFEFA
:1088600041F20821204630F1C3F8204610BD000037
:1088700038B5294B00F5805504460360D5F82C091E
:10888000EFF0C4FBD5F82009EFF0C0FBD5F81409D0
:10889000EFF0BCFBD5F80809EFF0B8FBD5F8FC0801
:1088A000EFF0B4FBD5F8F008EFF0B0FBD5F8E40832
:1088B000EFF0ACFBD5F8D808EFF0A8FB04F5B85002
:1088C0000830FBF73FF804F5AA50FBF73BF804F536
:1088D0004E70FFF7A1FE04F5B870FBF733F804F50E
:1088E0009470EFF013FF04F58C70EFF0C7FB04F108
:1088F000F400EFF0B5FB04F1DC00EFF0BFFB04F196
:10890000C400EFF0BBFB04F19C00F2F013FE204624
:10891000FAF716FE204638BD0044167010B504461E
:10892000FFF7A6FF41F63011204630F161F82046EE
:1089300010BD000070B5CB4B00F500550446036038
:10894000D5F8F00F04F53A56EFF060FBD5F8E40FD8
:10895000EFF05CFBD5F8D80FEFF058FBD5F8CC0F53
:10896000EFF054FBD5F8C00FEFF050FBD5F8B40F83
:10897000EFF04CFBD5F8A80FEFF048FBD5F89C0FB3
:10898000EFF044FBD5F8900FEFF040FBD5F8840FE3
:10899000EFF03CFBD5F8780FEFF038FBD5F86C0F13
:1089A000EFF034FBD5F8600FEFF030FBD5F8540F43
:1089B000EFF02CFBD5F8480FEFF028FBD5F83C0F73
:1089C000EFF024FBD5F8300FEFF020FBD5F8240FA3
:1089D000EFF01CFBD5F8180FEFF018FBD5F80C0FD3
:1089E000EFF014FBD5F8000FEFF010FBD5F8F40E04
:1089F000EFF00CFBD5F8E80EEFF008FBD5F8DC0E35
:108A0000EFF004FBD5F8D00EEFF000FBD5F8C40E64
:108A1000EFF0FCFA06F124001836FEF739FE304676
:108A2000EEF014FFD5F8940EEFF0F0FAD5F8880EBA
:108A3000EFF0ECFAD5F87C0EEFF0E8FAD5F8700E0E
:108A4000EFF0E4FAD5F8640EEFF0E0FAD5F8580E3E
:108A5000EFF0DCFAD5F84C0EEFF0D8FAD5F8400E6E
:108A6000EFF0D4FA04F538503030EFF0BDFD04F5E6
:108A700038502830EFF0B8FD04F536503030EFF0C4
:108A8000D5FD04F534503830EFF0D0FD04F5335007
:108A9000EFF0CCFD04F532503030EFF0A5FD04F5D9
:108AA00032502030EFF0A0FD04F532501030EFF0DE
:108AB0009BFD04F53250EFF097FD04F5305008307F
:108AC000EFF0B4FD04F52F503830EFF08DFD04F5D4
:108AD0002F502830EFF088FD04F52F501830EFF0BC
:108AE00083FD04F52F500830EFF07EFD04F52F5084
:108AF000EFF0ECFA04F52C5018301FF0E9F804F50B
:108B0000295030301FF0E4F804F5275008301FF0EA
:108B1000DFF804F521502830FFF7D6FB04F51D508F
:108B20000830FAF719FE04F5AA50FFF775FD04F5B1
:108B3000A45018301FF0CCF804F6C830FFF74CFDF5
:108B400004F62830FAF7FCFC04F51660FAF7FAFE92
:108B500004F50460FAF700FE04F5CF60FAF7F2FEC0
:108B600004F5C560FAF768FD04F5B0601FF0B0F8D1
:108B700004F58C60FAF7F0FD04F58360EFF0C6FDB4
:108B800004F56870EFF052FD04F56470EFF076FACA
:108B900004F55E70EFF072FA04F55770FFF730FBE2
:108BA00004F55070EFF05CFA04F54770EFF058FAF6
:108BB00004F53E70EFF054FA04F53570EFF050FA1A
:108BC00004F52C70EFF04CFA04F52370EFF048FA3E
:108BD00004F51A70EFF044FA04F51170EFF040FA62
:108BE00004F50870EFF03CFA04F5FE70EFF038FA87
:108BF00004F5EC70EFF034FA04F5E070EFF03EFAB3
:108C000004F5CE70EFF02CFAD4F89001EFF0FEF9F5
:108C100004F5BC70EFF032FA04F5AA70EFF020FA18
:108C2000D4F84801EFF0F2F904F59270EFF018FA79
:108C3000D4F81801EFF0EAF9D4F80C01EFF0E6F9F6
:108C400004F1E800EFF00CFA04F1D000EFF016FAAE
:108C500004F1A800F2F06EFC20461FF039F820461F
:108C600070BD00BF7855167010B50446FFF762FE60
:108C700042F6F87120462FF1BBFE204610BD0000E1
:108C8000304B10B504460360D0F8540FEFF0BEF936
:108C9000D4F8480FEFF0BAF9D4F83C0FEFF0B6F97A
:108CA000D4F8300FEFF0B2F904F6D860EFF02EFDF3
:108CB00004F56660EFF0BAFC04F6E850EFF0B6FC9D
:108CC00004F554601FF004F804F58D60FDF79AFA7E
:108CD00004F54270FFF7F8FA04F518701EF0F8FF7B
:108CE00004F50670EFF012FD04F5D070EFF09EFC75
:108CF00004F5C070EFF0B4F904F5AE70EFF0B0F920
:108D000004F5A270EFF0BAF904F59670EFF0B6F939
:108D100004F58A70EFF0B2F904F1FC00EFF0AEF95F
:108D200004F1E000FFF76CFA04F1D000EFF0A6F9CF
:108D300004F1A800F2F0FEFB20461EF0C9FF204619
:108D400010BD00BFA850167010B50446FFF798FF7D
:108D500040F6587120462FF14BFE204610BD000012
:108D6000064B10B50446036000F65870F2F0E2FBC3
:108D70002046FFF785FF204610BD00BF70501670DB
:108D800010B50446FFF7ECFF40F6787120462FF14E
:108D90002FFE204610BD0000384B10B5044603607E
:108DA000D0F88C09EFF032F9D4F88009EFF02EF901
:108DB000D4F87409EFF02AF9D4F86809EFF026F92D
:108DC000D4F85C09EFF022F9D4F85009EFF01EF95D
:108DD000D4F84409EFF01AF9D4F83809EFF016F98D
:108DE000D4F82C09EFF012F904F61C10EFF0FCFB9C
:108DF00004F61410EFF0F8FB04F60C10EFF0F4FB9F
:108E000004F51060EFF0F0FB04F6B800EFF07EFC24
:108E100004F50B60EFF05AF904F5DD60FAF792FD06
:108E200004F5C960FAF78CFB04F59D60FFF74CFA76
:108E300004F57270FAF790FC04F56A70EFF010F91F
:108E400004F56170EFF00CF904F55B70EFF016F9C2
:108E500004F55570EFF012F904F54C70EFF000F9DD
:108E600004F54370EFF0FCF804F53C70FFF7C8F927
:108E70002046FCF7B9FB204610BD00BF684F1670B6
:108E800010B50446FFF788FF4FF4196120462FF113
:108E9000AFFD204610BD0000224B10B50446036014
:108EA00000F5C760EFF032FC04F5A360FAF754FC5C
:108EB00004F56E70FFF708FA04F51670FFF704FA70
:108EC00004F5F070EFF0B2FB04F5CC70EFF01EFC8F
:108ED00004F5C470EFF0D2F804F5B870EFF0CEF8F6
:108EE00004F5AA70FFF78CF904F59C70EFF0B8F860
:108EF00004F58A70EFF0B4F804F1FC00EFF0BEF86E
:108F000004F1E400EFF0BAF804F1C800FFF778F9D3
:108F100004F1A800F2F00EFB20461EF0D9FE204618
:108F200010BD00BF4C4E167010B50446FFF7B4FFDD
:108F30004FF4D06120462FF15BFD204610BD0000AC
:108F400038B5454B00F5983504460360D5F8480719
:108F5000EFF05CF8D5F83C07EFF058F8D5F830079B
:108F6000EFF054F8D5F82407EFF050F8D5F81807CB
:108F700004F59B35EFF04AF805F58470EFF034FB0B
:108F800005F58070EFF030FB05F1F800EFF02CFBF9
:108F900005F1F000EFF028FB05F1E800EFF024FB0D
:108FA00005F1E000EFF020FB05F1680004F59A35CB
:108FB000EFF03CFB05F5F870EFF038FB05F5A47019
:108FC0001EF086FE04F5993004F5903500F5F47036
:108FD000FFF77AF905F5DC70FBF7ECF905F15800BD
:108FE000FFF772F904F55B60FCF7F6FB04F5A86087
:108FF000FEF70CFC04F59060FBF74AFB04F5767075
:109000001EF066FE04F57270EFF038F804F56C702F
:10901000EFF034F804F56570FFF7F2F804F56170CD
:10902000EFF02CF804F55B70EFF028F804F55470BD
:10903000FFF7E6F804F55070EFF020F804F54A70F9
:10904000EFF01CF804F54170EFF00AF82046FCF749
:1090500007FB204638BD00BFD448167010B5044643
:10906000FFF76EFF024920462FF1C2FC204610BDDB
:10907000503701002C4B10B504460360D0F8B806F9
:10908000EEF0C4FFD4F8AC06EEF0C0FFD4F8A006B2
:10909000EEF0BCFFD4F89406EEF0B8FFD4F88806E2
:1090A000EEF0B4FFD4F87C06EEF0B0FFD4F8700612
:1090B000EEF0ACFF04F5BE60EFF0B8FA04F58560A1
:1090C000FAF740FC04F560701EF002FE04F508702B
:1090D000FFF7FAF804F5EC70EFF018FB04F5B07048
:1090E000EFF0A4FA04F5A270EEF0BAFF04F5967062
:1090F000EEF0C4FF04F58A70EEF0C0FF04F1F80052
:10910000FFF77EF804F1E800EEF0B8FF04F1D000BC
:10911000EEF0B4FF04F1A800F2F00CFA20461EF0C5
:10912000D7FD204610BD00BF5C48167010B5044640
:10913000FFF7A0FF4FF4D86120462FF159FC2046DD
:1091400010BD000038B52E4B00F580550446036075
:10915000D5F8340BEEF05AFFD5F8280BEEF056FF99
:10916000D5F81C0BEEF052FFD5F8100BEEF04EFFC9
:10917000D5F8040BEEF04AFFD5F8F80AEEF046FFFA
:1091800004F5D5500830EFF0C1FA04F5D450103092
:10919000FBF7B0FE04F5C6500830FAF7D3FB04F530
:1091A0001B600FF03DFF04F50F60FBF7DFF904F5DE
:1091B000FA60FAF7D1FA04F5E660FAF7C1F904F5B6
:1091C000E460EEF05BFF04F20470FFF719F804F5B9
:1091D000DD60EEF045FF04F2C460EEF041FF04F5FF
:1091E000D460EEF03DFF04F5D160EEF047FF04F5EA
:1091F000CE60EEF043FF2046FFF7AEF8204638BDC4
:10920000F857167010B50446FFF79CFF41F6383149
:1092100020462FF1EDFB204610BD000038B5554B20
:1092200000F5005504460360D5F8BC08EEF0EEFEEC
:10923000D5F8B008EEF0EAFED5F8A408EEF0E6FEA8
:10924000D5F89808EEF0E2FED5F88C08EEF0DEFED8
:10925000D5F88008EEF0DAFED5F87408EEF0D6FE08
:10926000D5F86808EEF0D2FED5F85C08EEF0CEFE38
:10927000D5F85008EEF0CAFE04F51B502830FFF771
:1092800023F804F508502030FFF7BAF804F5EA5047
:109290001830FFF7B5F804F5C4501030FFF7B0F8F8
:1092A00004F59E500830FFF7ABF804F57060FFF747
:1092B000A7F804F59760FBF7F7FE04F56670FAF778
:1092C0004BFA04F54870EFF0B1F904F53670EFF0A1
:1092D0001DFA04F52F70EEF0C3FE04F52870FEF7BA
:1092E0008FFF04F52470EEF0C9FE04F51E70EEF059
:1092F000C5FE04F51570EEF0B3FE04F50E70FEF732
:109300007FFF04F50770EEF0ABFE04F5FC70EEF0A5
:10931000A7FE04F5EE70FEF773FF04F5E070EEF0C3
:109320009FFE04F5D270FEF76BFF04F5C470EEF0FB
:1093300097FE04F5B270EEF093FE04F5A470FEF70C
:109340005FFF04F59A70FEF75BFF04F58C70EEF09A
:1093500087FE04F1F400EEF083FE04F1D000EEF09D
:109360007FFE04F1A800F2F0E5F820461EF0B0FC04
:10937000204638BD6C56167010B50446FFF74EFFF8
:109380004FF4235120462FF133FB204610BD00003F
:10939000184B10B504460360D0F83C0AEEF036FED8
:1093A00004F62820EFF020F904F61820EFF01CF95D
:1093B00004F50560FAF7C6FA04F5E660FAF7CCF9A9
:1093C00004F5DB60FEF77EF904F2BC60EEF048FEC7
:1093D00004F5D360EEF044FE04F27C60FEF710FF6B
:1093E00004F5CD60FEF70CFF2046FEF7B5FF2046E2
:1093F00010BD00BF4055167010B50446FFF7C8FFFA
:109400004FF4246120462FF1F3FA204610BD0000EE
:1094100038B5224B0446036004F55965D0F8E00DD9
:10942000EEF0F4FDD4F8D40DEEF0F0FDD4F8C80D54
:10943000EEF0ECFDD4F8BC0DEEF0E8FD04F69C5027
:10944000FEF726F92846EEF001FAD4F88C0DEEF07E
:10945000DDFDD4F8800DEEF0D9FD04F66850EFF094
:10946000C3F804F64840FAF777F904F6F830FAF74B
:10947000E3F804F6D820FAF76FF904F68820FAF733
:10948000DBF804F66C20EEF0EBFD04F64820EEF07D
:10949000E7FD2046FFF77CFF204638BD08551670D3
:1094A00010B50446FFF7B4FF40F6E85120462FF10F
:1094B0009FFA204610BD000038B5244B00F57565B5
:1094C0000446036000F65C70FEF7E2F82846EEF012
:1094D000BDF9D4F84C0FEEF099FDD4F8400FEEF042
:1094E00095FDD4F8340FEEF091FDD4F8280FEEF08E
:1094F0008DFDD4F81C0FEEF089FDD4F8100FEEF0BE
:1095000085FDD4F8040FEEF081FD04F6F460EFF071
:109510006BF804F56F60EEF0D9FD04F69860FEF785
:10952000D1F804F68460FEF76BFE04F56760FEF781
:1095300067FE04F65C60FEF763FE04F64860FEF723
:109540005FFE2046FCF7A2FB204638BD085416708B
:1095500010B50446FFF7B0FF40F6787120462FF1B2
:1095600047FA204610BD000070B5634B00F58054EB
:1095700005460360D4F8180A05F5C956EEF046FD15
:10958000D4F80C0AEEF042FDD4F8000AEEF03EFDED
:10959000D4F8F409EEF03AFDD4F8E809EEF036FD1F
:1095A000D4F8DC09EEF032FDD4F8D009EEF02EFD4F
:1095B000D4F8C409EEF02AFDD4F8B809EEF026FD7F
:1095C000D4F8AC09EEF022FDD4F8A009EEF01EFDAF
:1095D000D4F89409EEF01AFDD4F88809EEF016FDDF
:1095E000D4F87C09EEF012FDD4F87009EEF00EFD0F
:1095F000D4F86409EEF00AFDD4F85809EEF006FD3F
:10960000D4F84C09EEF002FD06F10C00FEF740F82C
:109610003046EEF01BF9D4F81C09EEF0F7FCD4F854
:109620001009EEF0F3FCD4F80409EEF0EFFCD4F8E6
:10963000F808EEF0EBFCD4F8EC08EEF0E7FCD4F818
:10964000E008EEF0E3FCD4F8D408EEF0DFFCD4F848
:10965000C808EEF0DBFCD4F8BC08EEF0D7FCD4F878
:10966000B008EEF0D3FC05F5BF500830FAF77EFFE6
:1096700005F5B9500830FAF779FF05F5AB50FAF760
:1096800061F905F5A250FAF767F805F59950FAF770
:1096900063F805F59050FAF75FF805F5815018303A
:1096A000FAF750F905F67870FAF760FF05F55B6098
:1096B000FAF748F905F54F60FAF758FF05F6D84074
:1096C000FEF79EFD05F6BC40EEF0CAFC05F698409C
:1096D000EEF0C6FC05F67440EEF0C2FC05F5456000
:1096E000EEF0BEFC05F62C40EEF0BAFC2846FCF786
:1096F00005FA284670BD00BFC853167010B5044661
:10970000FFF732FF4FF4D15120462FF171F9204677
:1097100010BD000038B500F58054894B0546036044
:10972000D4F8B006EEF072FCD4F8A406EEF06EFCAD
:10973000D4F89806EEF06AFCD4F88C06EEF066FCDD
:10974000D4F88006EEF062FCD4F87406EEF05EFC0D
:10975000D4F86806EEF05AFCD4F85C06EEF056FC3D
:10976000D4F85006EEF052FCD4F84406EEF04EFC6D
:10977000D4F83806EEF04AFC05F5AF501430F1F09D
:10978000CBFED4F8E405EEF041FCD4F8D805EEF0B9
:109790003DFCD4F8CC05EEF039FCD4F8C005EEF071
:1097A00035FCD4F8B405EEF031FCD4F8A805EEF0A1
:1097B0002DFCD4F89C05EEF029FCD4F89005EEF0D1
:1097C00025FCD4F88405EEF021FCD4F87805EEF001
:1097D0001DFCD4F86C05EEF019FCD4F86005EEF031
:1097E00015FCD4F85405EEF011FCD4F84805EEF061
:1097F0000DFCD4F83C05EEF009FCD4F83005EEF091
:1098000005FCD4F82405EEF001FCD4F81805EEF0C0
:10981000FDFBD4F80C05EEF0F9FBD4F80005EEF0F2
:10982000F5FBD4F8F404EEF0F1FBD4F8E804EEF024
:10983000EDFBD4F8D404EEF0E9FBD4F8C804EEF064
:10984000E5FBD4F8BC04EEF0E1FBD4F8B004EEF094
:10985000DDFBD4F8A404EEF0D9FBD4F89804EEF0C4
:10986000D5FBD4F88C04EEF0D1FBD4F88004EEF0F4
:10987000CDFBD4F87404EEF0C9FBD4F86804EEF024
:10988000C5FBD4F85C04EEF0C1FBD4F85004EEF054
:10989000BDFBD4F84404EEF0B9FB05F5A150EEF0A1
:1098A000FEFE05F59850F9F757FF05F59350103077
:1098B000F9F7A6FE05F59150F9F7BEFE05F58850BB
:1098C000F9F74AFF05F57E60F9F746FF05F56C608C
:1098D000F9F742FF05F55A60F9F73EFF05F68450A7
:1098E000EEF0BEFB05F66850FEF78AFC05F64C501C
:1098F000EEF0B6FB05F62850EEF0B2FB05F604508C
:10990000EEF0AEFB05F54E60EEF0AAFB05F6BC40AE
:10991000EEF0A6FB05F69840EEF0A2FB05F67440CB
:10992000EEF09EFB05F54560EEF09AFB05F62C4047
:10993000EEF096FB2846FCF7E1F8284638BD00BF5C
:109940008853167010B50446FFF7E4FE41F2B86183
:1099500020462FF14DF8204610BD0000104B10B5E9
:1099600004460360D0F8EC0DEEF050FBD4F8E00DA7
:10997000EEF04CFBD4F8D40DEEF048FBD4F8C80D53
:10998000EEF044FBD4F8BC0DEEF040FB04F55A6059
:10999000FEF736FC2046FCF709FA204610BD00BF52
:1099A0000853167010B50446FFF7D8FF4FF45F61F7
:1099B00020462FF11DF8204610BD00001A4B10B5AF
:1099C00004460360D0F8F00DEEF020FBD4F8E40D6F
:1099D000EEF01CFBD4F8D80DEEF018FBD4F8CC0D4B
:1099E000EEF014FBD4F8C00DEEF010FBD4F8B40D7B
:1099F000EEF00CFBD4F8A80DEEF008FB04F548607F
:109A0000F9F7AAFE04F66440EEF02AFB04F5446080
:109A1000EEF026FB04F62440FEF7F2FB2046FCF7AE
:109A20006DF8204610BD00BF8852167010B5044670
:109A3000FFF7C4FF40F6F85120462EF1D9FF20462B
:109A400010BD000038B5B04B00F53045044603604A
:109A5000D5F8C001EEF0DAFAD5F8B401EEF0D6FA96
:109A6000D5F8A801EEF0D2FAD5F89C01EEF0CEFAC6
:109A7000D5F89001EEF0CAFAD5F88401EEF0C6FAF6
:109A8000D5F87801EEF0C2FAD5F86C01EEF0BEFA26
:109A9000D5F86001EEF0BAFAD5F85401EEF0B6FA56
:109AA000D5F84801EEF0B2FAD5F83C01EEF0AEFA86
:109AB000D5F83001EEF0AAFAD5F82401EEF0A6FAB6
:109AC000D5F81801EEF0A2FAD5F80C01EEF09EFAE6
:109AD000D5F80001EEF09AFAD5F8F400EEF096FA17
:109AE000D5F8E800EEF092FAD5F8DC00EEF08EFA48
:109AF000D5F8D000EEF08AFAD5F8C400EEF086FA78
:109B0000D5F8B800EEF082FAD5F8AC00EEF07EFAA7
:109B1000D5F8A000EEF07AFAD5F89400EEF076FAD7
:109B2000D5F88800EEF072FAE86FEEF06FFA28468A
:109B30006C30EEF059FD28466430EEF055FD2846B5
:109B40006030EEF0C3FA04F523407030FBF720FBE1
:109B500004F516408030FBF71BFB04F50D40B030D8
:109B6000FEF73AFD04F5FF403830FFF727FF04F514
:109B7000FB407030F9F7E6FE04F5E0405030FCF7AA
:109B80003DF904F5DF407830FDF79CFD04F5DC403D
:109B90003030F9F7D7FE04F5B8402830FEF73CFD29
:109BA00004F5B6400830F9F7D7FD04F5B340283086
:109BB000FEF78AFB04F597403830FFF7CFFE04F537
:109BC0005450FFF7A7FD04F5515018301EF080F8EF
:109BD00004F54A501030F9F7B5FE04F5C3501030C3
:109BE000FFF7C2FC04F5B5500830F9F7ABFE04F5F9
:109BF000E660FFF761FC04F5D1601EF069F804F53A
:109C0000AD60F9F7A9FD04F59560FAF7AFFC04F52E
:109C10008C60EEF07BFD04F24440EEF021FA04F596
:109C20008460EEF01DFA04F20440FEF7E9FA04F550
:109C30007C70FEF7E5FA04F57870EEF01FFA04F593
:109C40006F70EEF00DFA04F56370EEF0F7F904F5BD
:109C50005A70EEF005FA04F55470EEF00FFA04F5C0
:109C60004B70EEF0FDF904F54270EEF0F9F904F5F1
:109C70003B70FEF7C5FA04F53470EEF0F1F904F527
:109C80002B70EEF0EDF904F52270EEF0E9F904F531
:109C90001970EEF0E5F904F51070EEF0E1F904F555
:109CA0000770EEF0DDF904F5FC70EEF0D9F904F57B
:109CB000EA70EEF0D5F904F5D870EEF0D1F904F5BC
:109CC000C670EEF0CDF904F5B870FEF799FA04F518
:109CD000AA70EEF0C5F904F59870EEF0C1F904F53C
:109CE0008670EEF0BDF904F1E800EEF0B9F904F188
:109CF000C400EEF0B5F904F19C00F1F01BFC204625
:109D0000F9F71EFC204638BDB851167010B5044650
:109D1000FFF798FE4BF2C81120462EF169FE20464F
:109D200010BD000038B500F57045DE4B04460360F9
:109D3000D5F8FC02EEF06AF9D5F8F002EEF066F91B
:109D4000D5F8E402EEF062F9D5F8D802EEF05EF94B
:109D5000D5F8CC02EEF05AF9D5F8C002EEF056F97B
:109D6000D5F8B402EEF052F9D5F8A802EEF04EF9AB
:109D7000D5F89C02EEF04AF9D5F89002EEF046F9DB
:109D8000D5F88402EEF042F9D5F87802EEF03EF90B
:109D9000D5F86C02EEF03AF9D5F86002EEF036F93B
:109DA000D5F85402EEF032F9D5F84802EEF02EF96B
:109DB000D5F83C02EEF02AF9D5F83002EEF026F99B
:109DC000D5F82402EEF022F9D5F81802EEF01EF9CB
:109DD000D5F80C02EEF01AF9D5F80002EEF016F9FB
:109DE000D5F8F401EEF012F9D5F8E801EEF00EF92D
:109DF000D5F8DC01EEF00AF9D5F8D001EEF006F95D
:109E0000D5F8C401EEF002F9D5F8B801EEF0FEF88D
:109E1000D5F8AC01EEF0FAF8D5F8A001EEF0F6F8BE
:109E2000D5F89401EEF0F2F8D5F88801EEF0EEF8EE
:109E3000D5F87C01EEF0EAF8D5F87001EEF0E6F81E
:109E4000D5F86401EEF0E2F8D5F85801EEF0DEF84E
:109E5000D5F84C01EEF0DAF8D5F84001EEF0D6F87E
:109E6000D5F83401EEF0D2F8D5F82801EEF0CEF8AE
:109E7000D5F81C01EEF0CAF8D5F81001EEF0C6F8DE
:109E8000D5F80401EEF0C2F8D5F8F800EEF0BEF80F
:109E9000D5F8EC00EEF0BAF8D5F8E000EEF0B6F840
:109EA000D5F8D400EEF0B2F8D5F8C800EEF0AEF870
:109EB0002846A030F1F03EFB28468030F1F03AFB16
:109EC00028463830EEF022FC04F56F40F030EEF01A
:109ED0001DFC04F56F40A830EEF018FC04F56F404F
:109EE0006030EEF013FC04F56E40C030F9F728FB4B
:109EF00004F56B405030FBF7D7FA04F56940B830F1
:109F0000FAF75CF804F5694010301DF0E1FE04F545
:109F100068405030FAF72AFB04F562403030FAF717
:109F2000B1F804F560406830F9F70CFD04F55F40C6
:109F3000C0301DF0CDFE04F55A401830FBF708FB89
:109F400004F54B40D030FBF7A1FE04F53D408830CE
:109F5000FBF79CFE04F53C40C830FAF799FB04F58A
:109F60003C402830F9F7ECFA04F532409830FEF71F
:109F700013FF04F523404030FEF782FE04F51E4037
:109F80009830FDF7D1FB04F51D40F0301DF0A0FE28
:109F900004F518404830FBF7DBFA04F518402C3084
:109FA000FAF7C6FF04F51640E830FCF78FF904F520
:109FB0000840A030FBF76AFE04F50740F8301DF0BA
:109FC00087FE04F595400FF05DF904F6E8300FF0D8
:109FD000F3F804F534601DF07BFE04F698201DF0C4
:109FE00077FE04F59E60FBF7B3FA04F589601DF077
:109FF0006FFE04F56270FAF7B9FA04F538701DF0D7
:10A0000067FE04F52670EEF081FB04F51E70EEF09D
:10A0100027F804F51870EEF031F804F51270EEF040
:10A020002DF804F50B70FEF7EBF804F50670FEF75B
:10A03000E7F804F5FE70EEF013F804F5EC70EEF0BE
:10A040000FF804F5DA70EEF00BF804F5CE70EEF0D0
:10A0500015F804F5C270EEF011F804F5B470FEF7CF
:10A06000CFF804F5A670EDF0FBFF04F59870FEF74D
:10A07000C7F804F58A70EDF0F3FF04F1F800FEF77D
:10A08000BFF804F1DC00EDF0EBFF04F1C400EDF0EB
:10A09000F5FF04F19C00F1F04DFA2046F9F750FA73
:10A0A000204638BDBC4E167010B50446FFF73AFE88
:10A0B0004FF4734120462EF19BFC204610BD00005A
:10A0C00070B5B84B00F5C83504460360D5F8CC032D
:10A0D000EDF09CFFD5F8C003EDF098FFD5F8B40380
:10A0E000EDF094FFD5F8A803EDF090FFD5F89C03B0
:10A0F000EDF08CFFD5F89003EDF088FFD5F88403E0
:10A10000EDF084FFD5F87803EDF080FFD5F86C030F
:10A11000EDF07CFFD5F86003EDF078FFD5F854033F
:10A12000EDF074FFD5F84803EDF070FFD5F83C036F
:10A13000EDF06CFFD5F83003EDF068FFD5F824039F
:10A14000EDF064FFD5F81803EDF060FFD5F80C03CF
:10A15000EDF05CFFD5F80003EDF058FFD5F8F40200
:10A16000EDF054FFD5F8E802EDF050FFD5F8DC0231
:10A17000EDF04CFFD5F8D002EDF048FFD5F8C40261
:10A18000EDF044FFD5F8B802EDF040FFD5F8AC0291
:10A19000EDF03CFF04F5C93000F180068C30FDF78E
:10A1A00077FA3046EDF052FBD5F87C02EDF02EFF49
:10A1B000D5F87002EDF02AFFD5F86402EDF026FF25
:10A1C000D5F85802EDF022FFD5F84C02EDF01EFF55
:10A1D000D5F84002EDF01AFFD5F83402EDF016FF85
:10A1E000D5F82802EDF012FFD5F81C02EDF00EFFB5
:10A1F000D5F81002EDF00AFFD5F80402EDF006FFE5
:10A2000005F5EE70F1F096F905F5DE70F1F092F9D2
:10A2100005F5DA70EEF0E8F905F5CC70EEF03FFAEE
:10A2200005F5A870EEF072FA05F58470EEF06EFA9E
:10A2300005F1C000EEF06AFA05F17800EEF066FA7A
:10A2400004F5C13004F5C0353030FBF71FFD05F5CE
:10A25000C4701DF03DFD05F1F800F9F7D1F904F5E2
:10A26000B930B030FBF712FD04F5B83000F5F870E6
:10A27000FAF77CF904F5B4306030FEF78DFD04F593
:10A28000B33000F5E070F9F75BF904F5E9404030D0
:10A29000FFF748FD04F5CA404830FEF761FD04F5BC
:10A2A000C740F9F74FFB04F5C5404030FAF75EF9B7
:10A2B00004F5BE405030FBF7F7F804F5B540283000
:10A2C000FDF732FA04F5B2401030F9F777FE04F5E5
:10A2D000B0405030FAF74AF904F5AF4028301DF08D
:10A2E000F7FC04F596600EF001FF04F56470F9F7D1
:10A2F00033FA04F55E70FAF71BFE04F53670F9F7D1
:10A300001FF904F52470EEF001FA04F51E70FDF754
:10A3100077FF04F51970FDF773FF04F51270EDF087
:10A320009FFE04F50C70EDF0A9FE04F50370EDF04E
:10A3300097FE04F5FA70EDF0A1FE04F5EE70EDF075
:10A340009DFE04F5DC70EDF08BFE04F5CA70EDF0B7
:10A3500087FE04F5BC70FDF753FF04F5AE70EDF019
:10A360007FFE04F5A270EDF089FE04F59070EDF02B
:10A3700077FE04F58470EDF081FE04F1F000EDF05D
:10A380007DFE04F1D800EDF079FE04F1BC00FDF78C
:10A3900037FF04F19C00F1F0CDF82046F9F7D0F832
:10A3A000204670BD844E167010B50446FFF788FE37
:10A3B000024920462EF11CFB204610BDD09301001F
:10A3C00038B5684B00F5005504460360D5F8B80869
:10A3D000EDF01CFED5F8AC08EDF018FED5F8A0089D
:10A3E000EDF014FED5F89408EDF010FED5F88808CD
:10A3F000EDF00CFED5F87C08EDF008FED5F87008FD
:10A40000EDF004FED5F86408EDF000FED5F858082C
:10A41000EDF0FCFDD5F84C08EDF0F8FDD5F840085E
:10A42000EDF0F4FDD5F83408EDF0F0FDD5F828088E
:10A43000EDF0ECFDD5F81C08EDF0E8FDD5F81008BE
:10A44000EDF0E4FDD5F80408EDF0E0FDD5F8F807EF
:10A45000EDF0DCFDD5F8EC07EDF0D8FDD5F8E00720
:10A46000EDF0D4FDD5F8D407EDF0D0FDD5F8C80750
:10A47000EDF0CCFD04F51D503830EEF047F904F551
:10A4800019502030F9F730F904F5E6501030FEF796
:10A4900083FC04F5DB501030FDF716FF04F5CD50BA
:10A4A0000830F9F74FFA04F5BF50F9F74BFA04F505
:10A4B000B0501830F9F746FA04F5AA501830FAF7F8
:10A4C00055F804F5E260FBF7E1FB04F5AF60F9F73E
:10A4D00075FD04F56C70F9F735FA04F53C70FAF780
:10A4E00045F804F51470F9F72BF804F50270EEF056
:10A4F0000DF904F5FA70EDF0C1FD04F5EE70EDF024
:10A50000BDFD04F5E270EDF0B9FD04F5D670EDF097
:10A51000B5FD04F5CA70EDF0B1FD04F5BE70EDF0C7
:10A52000ADFD04F5AC70EDF09BFD04F59A70EDF017
:10A5300097FD04F58870EDF093FD04F1EC00EDF06B
:10A540008FFD04F1D000FDF75BFE04F1BC00FDF7C8
:10A5500057FE04F19C00F0F0EDFF2046F8F7F0FF05
:10A56000204638BD144E167010B50446FFF728FF7C
:10A570004FF4235120462EF13BFA204610BD000037
:10A5800038B52F4B00F5005504460360D5F8B002EE
:10A59000EDF03CFDD5F8A402EDF038FDD5F89802B9
:10A5A000EDF034FDD5F88C02EDF030FD04F50950E6
:10A5B0003430EDF08BFD04F509503030EDF086FDC0
:10A5C00004F502502830F9F7BDF904F59850083029
:10A5D000FBF7ECFB04F592500830F9F7C7FF04F5E0
:10A5E0008450F9F7AFF904F57660F9F7B5F804F59A
:10A5F000E070FBF7DBFB04F5BC70EEF087F804F5C8
:10A60000B070FDF7FDFD04F5A270EDF029FD04F535
:10A610009070EDF025FD04F1FC00EDF021FD04F15A
:10A62000D800EDF01DFD04F1BC00FDF7E9FD04F1DB
:10A630009C00F0F07FFF2046F8F782FF204638BDEF
:10A640006C4D167010B50446FFF79AFF42F2B82120
:10A6500020462EF1CDF9204610BD000038B500F59A
:10A660001045904B04460360D5F8D801EDF0CEFCC0
:10A67000D5F8CC01EDF0CAFCD5F8C001EDF0C6FC70
:10A68000D5F8B401EDF0C2FCD5F8A801EDF0BEFCA0
:10A69000D5F89C01EDF0BAFCD5F89001EDF0B6FCD0
:10A6A000D5F88401EDF0B2FCD5F87801EDF0AEFC00
:10A6B000D5F86C01EDF0AAFCD5F86001EDF0A6FC30
:10A6C000D5F85401EDF0A2FCD5F84801EDF09EFC60
:10A6D000D5F83C01EDF09AFCD5F83001EDF096FC90
:10A6E000D5F82401EDF092FCD5F81801EDF08EFCC0
:10A6F000D5F80C01EDF08AFCD5F80001EDF086FCF0
:10A70000D5F8F400EDF082FCD5F8E800EDF07EFC21
:10A71000D5F8DC00EDF07AFCD5F8D000EDF076FC51
:10A72000D5F8C400EDF072FCD5F8B800EDF06EFC81
:10A73000D5F8AC00EDF06AFCD5F8A000EDF066FCB1
:10A74000D5F89400EDF062FCD5F88800EDF05EFCE1
:10A75000E86FEDF05BFC286FEDF058FC686EEDF0F3
:10A7600055FCA86DEDF052FCE86CEDF04FFC286C48
:10A77000EDF04CFC686BEDF049FCA86AEDF046FC8E
:10A78000E869EDF043FC28461030EDF09FFC04F53D
:10A790000840C830F9F7A4FF04F5CC401030FFF7AB
:10A7A000EFFE04F5B0406030F9F7EAFF04F59140A0
:10A7B0006830FEF781FE04F56C503830F9F7E0FFA1
:10A7C00004F5C450FFF7DCFE04F52D60F9F7D8FF5F
:10A7D00004F56270F9F784FF04F54470EDF026FF8C
:10A7E00004F53270EDF092FF04F52A70EDF038FCBC
:10A7F00004F52170EDF034FC04F51A70FDF700FD4E
:10A8000004F51670EDF03AFC04F51070EDF036FC2E
:10A8100004F50A70EDF032FC04F50470EDF02EFC46
:10A8200004F5FC70EDF02AFC04F5EE70FDF7E8FC91
:10A8300004F5E670EDF022FC04F5DA70EDF01EFC94
:10A8400004F5CE70EDF01AFC04F5C270EDF016FCC4
:10A8500004F5B670EDF012FC04F5A870FDF7D0FC1D
:10A8600004F59E70FDF7CCFC04F59670EDF006FC47
:10A8700004F58A70EDF002FC04F1FC00EDF0FEFB43
:10A8800004F1E400EDF0FAFB04F1C800FDF7B8FCB8
:10A8900004F1A800F0F04EFE20461DF019FA204603
:10A8A00038BD00BF344D167010B50446FFF7D6FE14
:10A8B00049F2E01120462EF19BF8204610BD000021
:10A8C00038B5254B00F5405504460360D5F8FC0724
:10A8D000EDF09CFBD5F8F007EDF098FBD5F8E40718
:10A8E000EDF094FBD5F8D807EDF090FB04F55F5040
:10A8F0000830EDF079FE04F55C500830F9F736FECB
:10A9000004F525502830FBF779FA04F5DB501830B0
:10A91000FFF724F804F5AC70FEF726FE04F5887006
:10A92000EDF0F4FE04F1F800FDF76AFCD4F8F40051
:10A93000EDF06CFB04F1D000EDF092FBD4F8C40014
:10A94000EDF064FB04F19C00F0F0F4FD2046F8F714
:10A95000F7FD204638BD00BFFC4C167010B504460C
:10A96000FFF7AEFF4FF4605120462EF141F820462C
:10A9700010BD000038B5304B00F58045044603603B
:10A98000D5F80C01EDF042FBD5F80001EDF03EFBEF
:10A9900004F581403030EDF0B9FE28461030F8F76C
:10A9A000CFFD04F57D503030F8F7CAFD04F5455071
:10A9B0003830FFF703F804F5D650FEF7ABFE04F588
:10A9C000A050FEF757FB04F58360FBF72DFA04F562
:10A9D0008160EDF053FB04F57B70FDF711FC04F58D
:10A9E0007770EDF04BFB04F57170EDF047FB04F56B
:10A9F0006B70EDF043FB04F56270EDF031FB04F594
:10AA00005C70EDF03BFB04F55670EDF037FB04F5A0
:10AA10005070EDF033FB04F54A70EDF02FFB04F5B8
:10AA20004470EDF02BFB04F53E70EDF027FB204663
:10AA3000FAF7DAFD204638BD2448167010B50446F2
:10AA4000FFF798FF44F2101120462DF1D1FF204668
:10AA500010BD000038B5414B00F5143504460360C5
:10AA6000D5F8400BEDF0D2FAD5F8340BEDF0CEFA74
:10AA7000D5F8280BEDF0CAFAD5F81C0BEDF0C6FAA4
:10AA8000D5F8100BEDF0C2FAD5F8040BEDF0BEFAD4
:10AA9000D5F8F80AEDF0BAFAD5F8EC0AEDF0B6FA06
:10AAA000D5F8E00A04F51635EDF0B0FA05F5347086
:10AAB000EDF09AFD05F5327004F50635EDF094FDE4
:10AAC00005F5DC70FFF756FF05F5B070FCF7FAFDF1
:10AAD00004F562401030FEF733FA04F55940403077
:10AAE000FDF77AFD04F558408030F9F73FFD04F595
:10AAF00020408030FFF7E4FE04F513409030FAF771
:10AB000047FB04F5D870FFF7A9FD04F5B470EDF02C
:10AB1000FDFD04F5A670EDF0A3FA04F59A70EDF0D2
:10AB2000ADFA04F58C70FDF76BFB04F58470EDF065
:10AB3000A5FA04F1EC00FDF763FB04F1DC00EDF095
:10AB40009DFA04F1C400EDF099FA04F19C00F0F0D4
:10AB5000F1FC2046F8F7F4FC204638BDEC471670AF
:10AB600010B50446FFF776FF024920462DF140FF5D
:10AB7000204610BD485B020038B53F4B00F500553C
:10AB800004460360286FEDF041FA686EEDF03EFA7E
:10AB9000A86DEDF03BFAE86CEDF038FA286CEDF0BA
:10ABA00035FA686BEDF032FAA86AEDF02FFAE86931
:10ABB000EDF02CFA286904F5FF55EDF027FA05F1C0
:10ABC00010000435FCF764FD2846ECF03FFE04F568
:10ABD0008053D3F8E00FEDF019FA04F5FD5018306A
:10ABE000EDF074FA04F5B1500830FEF7D5F804F52D
:10ABF0005560FBF707FB04F6A800FCF795FD04F58C
:10AC0000A760FAF751FC04F56870F9F7D7F904F575
:10AC10003870F9F7ABFC04F50E701DF059F804F527
:10AC2000F870EDF073FD04F5BC70EDF0FFFC04F579
:10AC3000B470EDF023FA04F5A870EDF01FFA04F5F6
:10AC40009670EDF00DFA04F58A70EDF017FA04F144
:10AC5000F800FDF7D5FA04F1E800EDF00FFA04F181
:10AC6000D000EDF00BFA04F1A800F0F063FC2046F0
:10AC70001DF02EF8204638BDB447167010B50446B6
:10AC8000FFF77AFF42F2780120462DF1B1FE20460F
:10AC900010BD000038B5484B0446036004F69C65BF
:10ACA000D0F84C0FEDF0B2F9D4F8400FEDF0AEF95A
:10ACB000D4F8340FEDF0AAF9D4F8280FEDF0A6F986
:10ACC00004F6E460F0F028FCD4F8E00EEDF09EF914
:10ACD000D4F8D40EEDF09AF904F6A860FCF7D8FC8D
:10ACE0002846ECF0B3FD04F56860EDF0D8FC04F6FE
:10ACF0000860EDF09BFC04F55C60EDF007FD04F6E8
:10AD00004850EDF093FC04F63850EDF06DFC04F67D
:10AD10002850EDF069FC04F61850EDF065FC04F5E0
:10AD20004A60EDF083FC04F62840EDF07FFC04F56A
:10AD30003E60EDF0EBFC04F53D60EDF0DAF904F671
:10AD400028301CF0C5FF04F528601CF0C1FF04F694
:10AD5000D8101CF0BDFF04F513601CF0B9FF04F619
:10AD6000C400F8F791FB04F6B400EDF087F904F69F
:10AD70009C00EDF083F904F67800EDF071F904F52C
:10AD80000660EDF07BF904F64800EDF077F904F584
:10AD90000360EDF073F904F61800EDF06FF904F2BA
:10ADA000FC70FDF72DFA04F5F860F8F76FFD20460A
:10ADB000FAF750FE204638BDE846167010B5044636
:10ADC000FFF768FF4FF4756120462DF111FE204614
:10ADD00010BD000038B5274B00F5805504460360D0
:10ADE000D5F8A00FEDF012F9D5F8940FEDF00EF9AB
:10ADF000D5F8880FEDF00AF9D5F87C0FEDF006F9DB
:10AE0000D5F8700FEDF002F904F5FB50EDF0ECFB16
:10AE100004F5FA501030EDF059F92846FFF73AFFE3
:10AE200004F63860F8F78EFD04F61850F8F794FC35
:10AE300004F6F840EDF014F904F6D440EDF010F902
:10AE400004F6B840FDF7DCF904F69C40EDF008F993
:10AE500004F68440EDF012F9D4F8780CEDF0D6F851
:10AE600004F65C40FDF7CCF92046FBF725F82046B8
:10AE700038BD00BFA846167010B50446FFF7AAFFFC
:10AE800041F6A87120462DF1B3FD204610BD00000B
:10AE900038B52C4B00F5C04504460360D5F82002B8
:10AEA000EDF0B4F8D5F81402EDF0B0F8D5F80802DA
:10AEB000EDF0ACF8D5F8FC01EDF0A8F8D5F8F0010C
:10AEC000EDF0A4F8D5F8E401EDF0A0F8D5F8D8013C
:10AED000EDF09CF8D5F8CC01EDF098F8D5F8C0016C
:10AEE000EDF094F8D5F8B401EDF090F8D5F8A8019C
:10AEF000EDF08CF804F5C2405830EDF007FC04F595
:10AF000083403030FFF766FF04F508500830FFF744
:10AF100061FF04F505500830F9F728FB04F50250ED
:10AF200020301CF0D5FE04F502500830FDF768F91A
:10AF300004F501503430FDF763F92046FFF71CFE9D
:10AF4000204638BD7046167010B50446FFF7A0FFC6
:10AF500046F2282120462DF14BFD204610BD000071
:10AF600038B5314B00F5005504460360D5F864014F
:10AF7000EDF04CF8D5F85801EDF048F8D5F84C0153
:10AF8000EDF044F8D5F84001EDF040F804F5045038
:10AF90001C30EDF09BF804F504501830EDF096F8F5
:10AFA00004F5FF501830F8F7D7FB04F5F1501030D6
:10AFB000F8F7C8FC04F584501030FAF7F7FE04F5F2
:10AFC0000270FAF793FE04F5E070EDF09FFB04F5D4
:10AFD000D670EDF053F804F5C470EDF041F804F5C7
:10AFE000B670FDF70DF904F5A870EDF039F8D4F856
:10AFF0004401EDF00BF804F59470FDF701F904F548
:10B000008670EDF02DF804F1E800EDF029F804F178
:10B01000C400EDF025F804F19C00F0F08BFA204616
:10B02000F8F78EFA204638BDA844167010B50446CD
:10B03000FFF796FF42F2681120462DF1D9FC204619
:10B0400010BD000038B52A4B00F58045044603606A
:10B05000D5F80807ECF0DAFFD5F8FC06ECF0D6FFDF
:10B06000D5F8F006ECF0D2FFD5F8E406ECF0CEFF10
:10B07000D5F8D806ECF0CAFFD5F8CC06ECF0C6FF40
:10B08000D5F8C006ECF0C2FFD5F8B406ECF0BEFF70
:10B09000D5F8A806ECF0BAFF04F514503830FFF7E5
:10B0A0005FFF04F50D503030F8F74CFC04F50270EA
:10B0B000FFF756FF04F5A470F9F758FA04F580700D
:10B0C000EDF024FB04F1E800FDF79AF804F1D40058
:10B0D000FDF796F804F1C400ECF0D0FF04F19C00F9
:10B0E000F0F028FA2046F8F72BFA204638BD00BFCA
:10B0F0007044167010B50446FFF7A4FF44F21071B7
:10B1000020462DF175FC204610BD000038B53E4BA1
:10B1100000F543550446036005F114000835FCF7BB
:10B12000B7FA284604F54055ECF090FBD5F8C4007A
:10B13000ECF06CFFD5F8B800ECF068FFD5F8AC0087
:10B14000ECF064FFD5F8A000ECF060FFD5F89400B7
:10B15000ECF05CFFD5F88800ECF058FFE86FECF0FD
:10B1600055FF286FECF052FF686EECF04FFFA86DB2
:10B17000ECF04CFFE86CECF049FF286CECF046FF7B
:10B1800004F507503030FAF781FD04F500502830FF
:10B19000F8F7D8FB04F594500830FAF72FFE04F5C1
:10B1A0008860FAF773FD04F56070F9F771FA04F539
:10B1B000DC70F8F7C7FB04F5B870EDF0A7FA04F5FA
:10B1C000AA70ECF04DFF04F59C70FDF719F804F53A
:10B1D0009470ECF053FF04F58670FDF711F804F15C
:10B1E000FC00ECF04BFF04F1D800ECF039FF04F167
:10B1F000BC00FDF705F804F19C00F0F09BF9204637
:10B20000F8F79EF9204638BD3844167010B504464C
:10B21000FFF77CFF43F2F00120462DF1E9FB2046C9
:10B2200010BD000038B53C4B00F5185504460360CE
:10B2300005F120001435FCF72BFA284604F51755C4
:10B24000ECF004FB05F13C003035FCF721FA284610
:10B2500004F50055ECF0FAFAD5F8EC05ECF0D6FE62
:10B26000D5F8E005ECF0D2FED5F8D405ECF0CEFE32
:10B27000D5F8C805ECF0CAFED5F8BC05ECF0C6FE62
:10B28000D5F8B005ECF0C2FED5F8A405ECF0BEFE92
:10B29000D5F89805ECF0BAFED5F88C05ECF0B6FEC2
:10B2A000D5F88005ECF0B2FE04F515503030EDF025
:10B2B0009BF904F50E502830F8F744FB04F58D5047
:10B2C000FDF7AAF904F6D870F8F73CFB04F5C8704E
:10B2D000FAF7DCFC04F5A470EDF018FA04F59C70A4
:10B2E000ECF0CCFE04F58A70ECF0BAFE04F1F80044
:10B2F000FCF786FF04F1E800ECF0C0FE04F1C400A6
:10B30000ECF0AEFE04F19C00F0F014F92046F8F7E2
:10B3100017F9204638BD00BFC843167010B5044663
:10B32000FFF780FF42F2386120462DF161FB204695
:10B3300010BD000038B5344B00F5A045044603604D
:10B34000D5F8A005ECF062FED5F89405ECF05EFEB1
:10B35000D5F88805ECF05AFED5F87C05ECF056FEE1
:10B36000D5F87005ECF052FED5F86405ECF04EFE11
:10B37000D5F85805ECF04AFED5F84C05ECF046FE41
:10B38000D5F84005ECF042FED5F83405ECF03EFE71
:10B39000D5F82805ECF03AFE04F5A6405830F8F749
:10B3A000D1FA04F547503030FFF7DAFD04F5845048
:10B3B0000830FFF7D5FD04F6C870F9F7D7F804F5A3
:10B3C000C070FAF763FC04F59C70EDF09FF904F58A
:10B3D0009070FCF715FF04F58670FCF711FF04F17F
:10B3E000FC00ECF04BFE04F1E000FCF709FF04F177
:10B3F000C400ECF035FE04F19C00F0F09BF8204610
:10B40000F8F79EF8204638BD9043167010B50446F4
:10B41000FFF790FF45F2A85120462DF1E9FA2046AA
:10B4200010BD000038B52A4B00F5404504460360C6
:10B43000D5F8F407ECF0EAFDD5F8E807ECF0E6FD06
:10B44000D5F8DC07ECF0E2FDD5F8D007ECF0DEFD36
:10B4500004F5E4402030FFF76DFF04F597406830B5
:10B46000FFF7E0FE04F54A503830FDF701FA04F525
:10B47000E470FFF74BFE04F5C070EDF047F904F5FA
:10B48000B670ECF0FBFD04F5AA70ECF0F7FD04F5E6
:10B490009E70ECF0F3FD04F59270ECF0EFFD04F516
:10B4A0008670ECF0EBFD04F1F400ECF0E7FD04F144
:10B4B000DC00ECF0E3FD04F1C400ECF0DFFD04F18E
:10B4C0009C00F0F037F82046F8F73AF8204638BDEF
:10B4D0005843167010B50446FFF7A4FF4CF2F871FC
:10B4E00020462DF185FA204610BD000038B5514B9D
:10B4F00000F5C04504460360D5F88C0AECF086FDE3
:10B50000D5F8800AECF082FDD5F8740AECF07EFDE7
:10B51000D5F8680AECF07AFDD5F85C0AECF076FD17
:10B52000D5F8500AECF072FDD5F8440AECF06EFD47
:10B53000D5F8380AECF06AFDD5F82C0AECF066FD77
:10B54000D5F8200AECF062FDD5F8140AECF05EFDA7
:10B55000D5F8080AECF05AFDD5F8FC09ECF056FDD8
:10B56000D5F8F009ECF052FDD5F8E409ECF04EFD09
:10B57000D5F8D809ECF04AFDD5F8CC09ECF046FD39
:10B58000D5F8C009ECF042FD04F5D3403430ECF0BE
:10B590009DFD04F5D3403030ECF098FD04F5D24029
:10B5A00008301CF095FB04F5D0406830F7F7C8FF71
:10B5B00004F5CF402830F8F7D9FF04F58C4040302F
:10B5C000FFF7CEFC04F513501830FFF7C9FC04F563
:10B5D0000C501030F8F7B6F904F5D470FFF7C0FC42
:10B5E00004F5B070EDF092F804F5A470FCF708FED5
:10B5F00004F59A70FCF704FE04F59070FCF700FE69
:10B6000004F58870ECF03AFD04F1F400FCF7F8FD65
:10B6100004F1E000FCF7F4FD04F1C400ECF020FDBF
:10B6200004F19C00EFF086FF2046F7F789FF2046E3
:10B6300038BD00BF2043167010B50446FFF756FF13
:10B6400046F6902120462DF1D3F9204610BD00008A
:10B6500038B5514B00F5C04504460360D5F88C0A57
:10B66000ECF0D4FCD5F8800AECF0D0FCD5F8740AE4
:10B67000ECF0CCFCD5F8680AECF0C8FCD5F85C0A14
:10B68000ECF0C4FCD5F8500AECF0C0FCD5F8440A44
:10B69000ECF0BCFCD5F8380AECF0B8FCD5F82C0A74
:10B6A000ECF0B4FCD5F8200AECF0B0FCD5F8140AA4
:10B6B000ECF0ACFCD5F8080AECF0A8FCD5F8FC09D5
:10B6C000ECF0A4FCD5F8F009ECF0A0FCD5F8E40906
:10B6D000ECF09CFCD5F8D809ECF098FCD5F8CC0936
:10B6E000ECF094FCD5F8C009ECF090FC04F5D340E4
:10B6F0003430ECF0EBFC04F5D3403030ECF0E6FCF9
:10B7000004F5D24008301CF0E3FA04F5D04068306C
:10B71000F7F716FF04F5CF402830F8F727FF04F5B8
:10B720008C404030FFF71CFC04F513501830FFF735
:10B7300017FC04F50C501030F8F704F904F5D47038
:10B74000FFF70EFC04F5B070ECF0E0FF04F5A47018
:10B75000FCF756FD04F59A70FCF752FD04F5907065
:10B76000FCF74EFD04F58870ECF088FC04F1F40061
:10B77000FCF746FD04F1E000FCF742FD04F1C400D3
:10B78000ECF06EFC04F19C00EFF0D4FE2046F7F7DD
:10B79000D7FE204638BD00BFE842167010B50446FB
:10B7A000FFF756FF46F6902120462DF121F920465D
:10B7B00010BD000038B52A4B00F5804504460360F3
:10B7C000D5F80807ECF022FCD5F8FC06ECF01EFCDE
:10B7D000D5F8F006ECF01AFCD5F8E406ECF016FC0F
:10B7E000D5F8D806ECF012FCD5F8CC06ECF00EFC3F
:10B7F000D5F8C006ECF00AFCD5F8B406ECF006FC6F
:10B80000D5F8A806ECF002FC04F514503830FFF728
:10B81000A7FB04F50D503030F8F794F804F50270EA
:10B82000FFF79EFB04F5A470F8F7A0FE04F5807006
:10B83000ECF06CFF04F1E800FCF7E2FC04F1D4004A
:10B84000FCF7DEFC04F1C400ECF018FC04F19C00F1
:10B85000EFF070FE2046F7F773FE204638BD00BFBC
:10B86000B042167010B50446FFF7A4FF44F2107101
:10B8700020462DF1BDF8204610BD000038B5414BE3
:10B8800000F5083504460360D5F8C00DECF0BEFBAA
:10B89000D5F8B40DECF0BAFBD5F8A80DECF0B6FB7A
:10B8A000D5F89C0DECF0B2FBD5F8900D04F50B35F6
:10B8B000ECF0ACFB05F5C270ECF008FC05F5C070CF
:10B8C000ECF004FC04F5F3307030FFF773FF04F57F
:10B8D000BD3000F5F070FFF7BBFE04F5883000F5D1
:10B8E000A870FFF703FE04F592405830FFF79AFD69
:10B8F00004F51270FFF7A6FB04F50070ECF006FFEC
:10B9000004F5F470FCF77CFC04F5EA70FCF778FCB5
:10B9100004F5E270ECF0B2FB04F5D670ECF0AEFB8F
:10B9200004F5CA70ECF0AAFB04F5BE70ECF0A6FBBF
:10B9300004F5B070FCF764FC04F5A870ECF09EFB15
:10B9400004F59C70ECF09AFB04F59070ECF096FB1B
:10B9500004F58470ECF092FB04F1F000ECF08EFB47
:10B9600004F1D800ECF08AFB04F1BC00FCF748FCC1
:10B9700004F19C00EFF0DEFD2046F7F7E1FD2046E4
:10B9800038BD00BF7842167010B50446FFF776FF49
:10B99000024920462DF12CF8204610BDC82D02008A
:10B9A00070B5674B00F5004504460360D5F8F00B11
:10B9B00004F50A46ECF02AFBD5F8E40BECF026FB84
:10B9C000D5F8D80BECF022FBD5F8CC0BECF01EFB35
:10B9D000D5F8C00BECF01AFBD5F8B40BECF016FB65
:10B9E000D5F8A80BECF012FBD5F89C0BECF00EFB95
:10B9F000D5F8900BECF00AFBD5F8840BECF006FBC5
:10BA0000D5F8780BECF002FBD5F86C0BECF0FEFAF5
:10BA1000D5F8600BECF0FAFAD5F8540BECF0F6FA26
:10BA2000D5F8480BECF0F2FAD5F83C0BECF0EEFA56
:10BA3000D5F8300BECF0EAFAD5F8240BECF0E6FA86
:10BA400006F58270F836FBF723FE3046EBF0FEFE7B
:10BA5000D5F8F40AECF0DAFAD5F8E80AECF0D6FA00
:10BA600004F50A40D030ECF044FB04F5DF40303000
:10BA7000FAF7A4FA04F5A9401030FAF79FFA04F592
:10BA8000A7407030F7F75CFD04F563501030FAF70B
:10BA900095FA04F5ED501030FAF790FA04F5247099
:10BAA000FAF78CFA04F51270ECF030FE04F50D7024
:10BAB000FCF7A6FB04F50970ECF0E0FA04F503705E
:10BAC000ECF0DCFA04F5F870FCF79AFB04F5F07082
:10BAD000ECF0D4FA04F5E470ECF0D0FA04F5D6708A
:10BAE000FCF78EFB04F5CC70FCF78AFB04F5C47000
:10BAF000ECF0C4FA04F5B270ECF0B2FA04F5A670FA
:10BB0000ECF0BCFA04F59870FCF77AFB04F58A7047
:10BB1000ECF0A6FA04F1F800FCF772FB04F1E8007F
:10BB2000ECF0ACFA04F1C400ECF09AFA04F19C00D9
:10BB3000EFF000FD2046F7F703FD204670BD00BF83
:10BB40000042167010B50446FFF72AFF48F6F83198
:10BB500020462CF14DFF204610BD000070B500F5C9
:10BB60004E35804B044605F5C476036005F5CA7072
:10BB7000FBF78EFD304604F54C36EBF067FED6F849
:10BB80008409ECF043FAD6F87809ECF03FFAD6F8DD
:10BB90006C09ECF03BFAD6F8600905F59876ECF004
:10BBA00035FA05F59E70FBF773FD304605F5847692
:10BBB000EBF04CFE05F58A70FBF76AFD304605F1A7
:10BBC000E006EBF043FE05F1EC00FBF761FD3046CB
:10BBD00005F1B806EBF03AFE05F1C400FBF758FD9D
:10BBE000304605F19006EBF031FE05F19C00FBF7C5
:10BBF0004FFD304605F16806EBF028FE05F17400B4
:10BC0000FBF746FD304605F14006EBF01FFE05F15F
:10BC10004C00FBF73DFD3046EBF018FE05F1180631
:10BC200005F1240004F54D35FBF732FD304605F5EE
:10BC30007C76EBF00BFE05F57F70FBF729FD3046B7
:10BC400005F57276EBF002FE05F57570FBF720FD49
:10BC5000304605F56876EBF0F9FD05F56B70FBF7FE
:10BC600017FD304605F55E76EBF0F0FD05F56170E9
:10BC7000FBF70EFD3046EBF0E9FD05F5067004F527
:10BC80004335FCF721FB04F54430FBF7F3FD05F5E4
:10BC90001A70F8F793F905F5D470F8F767FC04F516
:10BCA000393000F56470FBF7E5FD04F5373000F539
:10BCB0000070FDF771F804F5143000F50270FFF71D
:10BCC0006FFE04F51150FFF7D9FD04F52270F9F766
:10BCD00033FE04F51070ECF019FD04F50C70ECF077
:10BCE000CDF904F50570FCF78BFA04F50070FCF74C
:10BCF00087FA04F5F270ECF0B3F904F5E070ECF0BB
:10BD0000AFF904F5D470ECF0B9F904F5C870ECF0B3
:10BD1000B5F904F5BC70ECF0B1F904F5AE70FCF7C0
:10BD20006FFA04F5A470FCF76BFA04F59670ECF06A
:10BD300097F904F58870FCF763FA04F58070ECF06D
:10BD40009DF904F1E800ECF099F904F1C400ECF07D
:10BD500087F904F19C00EFF0EDFB2046F7F7F0FBCC
:10BD6000204670BD7841167010B50446FFF7F6FE08
:10BD7000024920462CF13CFE204610BDB03903009C
:10BD800038B5334B00F53B550446036005F12400FC
:10BD90001835FBF77DFC2846EBF058FD04F51050F4
:10BDA000FAF758FA04F5C9500830FAF753FA04F5CF
:10BDB0006560FAF74FFA04F55B60F7F7C1FB04F52D
:10BDC0003670FAF747FA04F51870ECF02FFC04F51A
:10BDD0000670ECF09BFC04F50170ECF04FF904F5F3
:10BDE000F670ECF04BF904F5E870FCF709FA04F58D
:10BDF000E070ECF043F904F5D270FCF701FA04F5B9
:10BE0000C470ECF02DF904F5B670FCF7F9F904F5FF
:10BE1000A870ECF025F904F59C70ECF02FF904F50E
:10BE20008E70FCF7EDF904F58070ECF019F904F16F
:10BE3000E800ECF023F904F1D000ECF01FF904F174
:10BE4000A800EFF077FB20461BF042FF204638BDEC
:10BE50000041167010B50446FFF792FF4FF43C51B5
:10BE600020462CF1C5FD204610BD000038B5404BE2
:10BE700000F5E04504460360D5F8EC00ECF0C6F8A8
:10BE8000D5F8E000ECF0C2F8D5F8D400ECF0BEF83C
:10BE9000D5F8C800ECF0BAF8D5F8BC00ECF0B6F86C
:10BEA000D5F8B000ECF0B2F8D5F8A400ECF0AEF89C
:10BEB000D5F89800ECF0AAF8D5F88C00ECF0A6F8CC
:10BEC000D5F88000ECF0A2F8686FECF09FF8A86E4F
:10BED000ECF09CF8E86DECF099F8286DECF096F831
:10BEE0002846ECF013FC04F5BD403030FAF710F8AA
:10BEF00004F5B2400830F9F72BFB04F5A64060309A
:10BF0000F9F726FB04F54E503830FEF763FF04F5D1
:10BF1000A0501030FEF75EFF04F59A501030F8F78D
:10BF200025FB04F5955008301BF0D2FE04F5AC70EB
:10BF3000F9F7EEFF04F58870ECF0E8FB04F1F80087
:10BF4000FCF75EF904F1E400FCF75AF904F1D000C3
:10BF5000FCF756F904F1BC00FCF752F904F19C001F
:10BF6000EFF0E8FA2046F7F7EBFA204638BD00BFBD
:10BF70008840167010B50446FFF778FF47F2F001CD
:10BF800020462CF135FD204610BD000038B5474B4A
:10BF900000F5405504460360D5F83004ECF036F85F
:10BFA000D5F82404ECF032F8D5F81804ECF02EF8AB
:10BFB000D5F80C04ECF02AF8D5F80004ECF026F8DB
:10BFC000D5F8F403ECF022F8D5F8E803ECF01EF80D
:10BFD000D5F8DC03ECF01AF8D5F8D003ECF016F83D
:10BFE000D5F8C403ECF012F8D5F8B803ECF00EF86D
:10BFF00004F54E501830ECF069F804F54750103055
:10C00000F7F7A0FC04F50C503830F9F79BFE04F567
:10C01000A550F9F797FE04F596501830F7F792FC03
:10C0200004F588501030F7F78DFC04F53270F9F7FD
:10C030002DFE04F52070ECF069FB04F51970ECF0AE
:10C040000FF804F51070ECF00BF804F50470EBF049
:10C05000F5FF04F5F670ECF003F804F5E870FCF772
:10C06000CFF804F5DA70EBF0FBFF04F5C870EBF0E5
:10C07000F7FF04F5B670EBF0F3FF04F59E70EBF0FC
:10C08000DDFF04F58670EBF0D9FF04F1E800EBF07A
:10C09000E7FF04F1C400EBF0E3FF04F19C00EFF0D4
:10C0A00049FA2046F7F74CFA204638BD243F16706F
:10C0B00010B50446FFF76AFF43F2384120462CF1E1
:10C0C00097FC204610BD00006F4B70B5044603601E
:10C0D00000F5AE4004F5AE4504F5AC465830EFF03F
:10C0E0001BFA05F134002835FBF7D2FA284604F58F
:10C0F000A045EBF0ABFBD5F82407EBF087FFD5F8B4
:10C100001807EBF083FFD5F80C07EBF07FFFD5F8AD
:10C110000007EBF07BFFD5F8F406EBF077FFD5F8DE
:10C12000E806EBF073FFD5F8DC06EBF06FFFD5F80F
:10C13000D006EBF06BFFD5F8C406EBF067FFD5F83F
:10C14000B806EBF063FFD5F8AC06EBF05FFFD5F86F
:10C15000A006EBF05BFFD5F89406EBF057FFD5F89F
:10C160008806EBF053FF06F160005436FBF790FAB7
:10C170003046EBF06BFBD5F85006EBF047FFD5F8F7
:10C180004406EBF043FFD5F83806EBF03FFFD5F857
:10C190002C06EBF03BFFD5F82006EBF037FF04F55B
:10C1A000AC400830ECF020FA04F5AB407830ECF00D
:10C1B0001BFA04F5AB403030ECF0A8FA04F505505A
:10C1C0003830FFF7E3FE04F5B850F8F721FE04F528
:10C1D000FC60F8F7E5FD04F5F260F7F72DFA04F5D9
:10C1E000E860F7F729FA04F5C560F7F77DFA04F57A
:10C1F000A260F7F779FA04F57E70F7F775FA04F59F
:10C200003870F7F771FA04F52470F7F715FA04F5AA
:10C210001270ECF07BFA04F50A70EBF021FF04F5E4
:10C220000170EBF01DFF04F5F070EBF019FF04F561
:10C23000E470EBF023FF04F5D270EBF011FF04F58E
:10C24000C670EBF01BFF04F5B870FBF7D9FF04F5DF
:10C25000AA70EBF005FF04F59870EBF001FF04F510
:10C260008670EBF0FDFE04F1E800EBF0F9FE04F15E
:10C27000C400EBF0F5FE04F19C00EFF05BF9204602
:10C28000F7F75EF9204670BDEC3E167010B5044617
:10C29000FFF71AFF45F2987120462CF1A9FB2046C2
:10C2A00010BD000038B5354B00F5805504460360DD
:10C2B000D5F8C00CEBF0AAFED5F8B40CEBF0A6FE56
:10C2C000D5F8A80CEBF0A2FED5F89C0CEBF09EFE86
:10C2D000D5F8900CEBF09AFED5F8840CEBF096FEB6
:10C2E000D5F8780CEBF092FED5F86C0CEBF08EFEE6
:10C2F000D5F8600CEBF08AFED5F8540CEBF086FE16
:10C3000004F5E2500430ECF06FF904F5E250EBF084
:10C31000DDFE04F6F850F9F7B9FC04F54360F7F7D1
:10C3200011FB04F5F470F8F7BFFE04F5D070ECF0E3
:10C33000EDF904F5C070EBF093FE04F5AE70EBF090
:10C340008FFE04F59C70EBF08BFE04F58E70FBF70E
:10C3500057FF04F58070EBF083FE04F1E800EBF08A
:10C360008DFE04F1C400EBF07BFE04F19C00EFF0C5
:10C37000E1F82046F7F7E4F8204638BDB43E1670E1
:10C3800010B50446FFF78EFF41F6C84120462CF158
:10C390002FFB204610BD000038B5464B0446036015
:10C3A00000F5325004F531551C30EFF0B5F805F1C9
:10C3B00038002C35FBF76CF9284604F53155EBF0C5
:10C3C00045FA05F114000835FBF762F9284604F533
:10C3D0000055EBF03BFAD5F8440CEBF017FED5F81E
:10C3E000380CEBF013FED5F82C0CEBF00FFED5F863
:10C3F000200CEBF00BFED5F8140CEBF007FED5F893
:10C40000080CEBF003FED5F8FC0BEBF0FFFDD5F8C4
:10C41000F00BEBF0FBFD04F52F501830ECF0E4F8D6
:10C4200004F52F500830ECF0DFF804F52E500830FA
:10C43000F7F71FF904F529503030F7F755F904F5EF
:10C4400028502030F7F7F8F804F52450F7F784F96E
:10C4500004F5F4500830F8F7DBFC04F5E070FFF762
:10C4600021FF04F5BC70ECF051F904F5AE70EBF06F
:10C47000F7FD04F59C70EBF0F3FDD4F82C01EBF024
:10C48000C5FD04F58870FBF7BBFE04F58070EBF08A
:10C49000F5FD04F1E800EBF0F1FD04F1C400EBF070
:10C4A000DFFD04F19C00EFF045F82046F7F748F86F
:10C4B000204638BD7C3E167010B50446FFF76CFF71
:10C4C00042F6D84120462CF193FA204610BD0000D8
:10C4D00038B5254B00F5805504460360D5F8CC0EE1
:10C4E000EBF094FDD5F8C00EEBF090FDD5F8B40E4E
:10C4F000EBF08CFDD5F8A80EEBF088FD04F5F450B8
:10C500001830ECF071F804F5F4500830EBF0DEFD73
:10C510002846F9F7EBFB04F63860F7F713FA04F650
:10C520001850F7F719F904F6F840EBF099FD04F606
:10C53000D440EBF095FD04F6B840FBF761FE04F63D
:10C540009C40EBF08DFD04F68440EBF097FDD4F8B1
:10C55000780CEBF05BFD04F65C40FBF751FE2046E7
:10C56000F9F7AAFC204638BD3C3E167010B50446CB
:10C57000FFF7AEFF41F6D06120462CF139FA204694
:10C5800010BD000038B55F4B00F5AD4504460360B3
:10C5900005F170006435FBF77BF8284604F5A045EB
:10C5A000EBF054F9D5F8E006EBF030FDD5F8D40601
:10C5B000EBF02CFDD5F8C806EBF028FDD5F8BC064D
:10C5C000EBF024FDD5F8B006EBF020FDD5F8A4067D
:10C5D000EBF01CFDD5F89806EBF018FDD5F88C06AD
:10C5E000EBF014FDD5F88006EBF010FDD5F87406DD
:10C5F000EBF00CFDD5F86806EBF008FDD5F85C060D
:10C60000EBF004FDD5F8500604F5AC45EBF0FEFC6C
:10C6100005F12C002035FBF73BF82846EBF016F926
:10C6200004F5AB405830ECF071F804F5AB40103035
:10C63000ECF06CF804F5A9407030F6F781FF04F5D2
:10C64000A7407030F7F740F904F55C502830FFF749
:10C6500029FE04F558500830F7F77EF804F55350DA
:10C660003030F7F741F804F504502830F8F700FCB3
:10C6700004F51670FFF72CFF04F50470ECF046F893
:10C6800004F5FA70EBF0ECFC04F5EE70EBF0F6FC60
:10C6900004F5E070FBF7B4FD04F5D870EBF0EEFCA8
:10C6A00004F5C670EBF0DCFC04F5B470EBF0D8FCDC
:10C6B00004F5A270EBF0D4FC04F59670EBF0DEFC10
:10C6C00004F58A70EBF0DAFC04F1F800FBF798FD52
:10C6D000D4F8F400EBF09AFCD4F8E800EBF096FC08
:10C6E000D4F8DC00EBF092FC04F1C400EBF0C6FCE3
:10C6F00004F19C00EEF01EFF2046F6F721FF2046D5
:10C7000038BD00BFC83D167010B50446FFF73AFFAC
:10C7100045F2087120462CF16BF9204610BD00004F
:10C7200038B5574B00F5405504460360D5F8440131
:10C73000EBF06CFCD5F83801EBF068FCD5F82C0177
:10C74000EBF064FCD5F82001EBF060FCD5F81401A7
:10C75000EBF05CFCD5F80801EBF058FCD5F8FC00D8
:10C76000EBF054FCD5F8F000EBF050FCD5F8E40009
:10C77000EBF04CFCD5F8D800EBF048FCD5F8CC0039
:10C78000EBF044FCD5F8C000EBF040FCD5F8B40069
:10C79000EBF03CFCD5F8A800EBF038FCD5F89C0099
:10C7A000EBF034FCD5F89000EBF030FC04F5415090
:10C7B000EBF0ACFF04F53F503030F6F73DFF04F5E9
:10C7C0003B501830F6F790FF04F53750F6F78CFF22
:10C7D00004F50D500830F8F71BFB04F50650F7F789
:10C7E000B1F804F5FD501830F7F7ACF804F58B50AC
:10C7F0001030F9F74BFA04F53670F9F7A3FA04F59F
:10C800002470EBF083FF04F51970EBF017FC04F5CE
:10C810001370EBF033FC04F50D70EBF02FFC04F516
:10C820000470EBF01DFC04F5F670EBF019FC04F558
:10C83000E470EBF015FC04F5D270EBF011FC04F59C
:10C84000C070EBF00DFC04F5AE70EBF009FC04F5E4
:10C850009670EBF0F3FB04F1FC00EBF0EFFB04F15E
:10C86000D800EBF0FDFB04F1BC00FBF7C9FC04F1C0
:10C870009C00EEF05FFE2046F6F762FE204638BDD3
:10C88000903D167010B50446FFF74AFF43F2481179
:10C8900020462CF1ADF8204610BD000038B5504BB5
:10C8A00000F5804504460360D5F8140FEBF0AEFBAD
:10C8B000D5F8080FEBF0AAFBD5F8FC0EEBF0A6FBC1
:10C8C000D5F8F00EEBF0A2FBD5F8E40EEBF09EFBF2
:10C8D000D5F8D80EEBF09AFBD5F8CC0EEBF096FB22
:10C8E000D5F8C00EEBF092FBD5F8B40EEBF08EFB52
:10C8F000D5F8A80EEBF08AFBD5F89C0EEBF086FB82
:10C90000D5F8900EEBF082FBD5F8840EEBF07EFBB1
:10C91000D5F8780EEBF07AFBD5F86C0EEBF076FBE1
:10C92000D5F8600EEBF072FB04F59C401030EBF094
:10C93000EDFE04F59B404830EBF0E8FE04F599402D
:10C940004830F6F7C1FF04F597403030F6F7CCFEDB
:10C9500004F596401030F6F7F3FD04F5934070307F
:10C96000F6F7FAFE04F558502830F8F781FA04F586
:10C97000F870FFF70BFB04F5D470EBF0C7FE04F57D
:10C98000C670EBF06DFB04F5BA70EBF077FB04F5C5
:10C99000A870EBF065FB04F59670EBF061FB04F515
:10C9A0008A70EBF06BFB04F1F800FBF729FCD4F87C
:10C9B000F400EBF02BFBD4F8E800EBF027FBD4F805
:10C9C000DC00EBF023FB04F1C400EBF057FB04F1B7
:10C9D0009C00EEF0AFFD2046F6F7B2FD204638BDD4
:10C9E000083D167010B50446FFF758FF44F618715D
:10C9F00020462BF1FDFF204610BD000070B5874B8F
:10CA000000F5C04504460360D5F8640404F5C64645
:10CA1000EBF0FCFAD5F85804EBF0F8FAD5F84C0432
:10CA2000EBF0F4FAD5F84004EBF0F0FAD5F8340462
:10CA3000EBF0ECFAD5F82804EBF0E8FAD5F81C0492
:10CA4000EBF0E4FAD5F81004EBF0E0FAD5F80404C2
:10CA5000EBF0DCFAD5F8F803EBF0D8FAD5F8EC03F4
:10CA6000EBF0D4FAD5F8E003EBF0D0FAD5F8D40324
:10CA7000EBF0CCFAD5F8C803EBF0C8FAD5F8BC0354
:10CA8000EBF0C4FAD5F8B003EBF0C0FAD5F8A40384
:10CA9000EBF0BCFA06F184007836FAF7F9FD30467F
:10CAA00004F5C646EAF0D2FED5F87403EBF0AEFA10
:10CAB000D5F86803EBF0AAFAD5F85C03EBF0A6FA18
:10CAC000D5F85003EBF0A2FA06F130002436FAF75D
:10CAD000DFFD3046EAF0BAFED5F8200304F5C5457F
:10CAE000EBF094FA05F17C007035FAF7D1FD284699
:10CAF000EAF0ACFE04F5C5406830EBF075FD04F5D6
:10CB0000C5406030EBF070FD04F5C5405830EBF0E7
:10CB10006BFD04F5C5404830EBF066FD04F5C440FC
:10CB20007030FAF7CFFD04F5A6405030F8F738F929
:10CB300004F5A54028301BF0CBF804F55750203001
:10CB4000FFF7B0FB04F5B8501030FFF7C1FC04F557
:10CB5000AA500830F6F7F6FE04F5A5501BF0B8F819
:10CB600004F59F50F7F702FD04F59750F6F7ACFE79
:10CB700004F59450F6F796FD04F58B500830F6F75F
:10CB8000B3FD04F53470F9F7DDF804F52270EBF02D
:10CB9000BDFD04F51D70EBF071FA04F51170EBF0BA
:10CBA0004DFA04F50870EBF05BFA04F5F870EBF061
:10CBB00045FA04F5EC70EBF061FA04F5DA70EBF08D
:10CBC0004FFA04F5CC70FBF71BFB04F5C270FBF7C2
:10CBD00017FB04F5B470EBF043FA04F5A870EBF022
:10CBE0004DFA04F59C70EBF049FA04F58E70FBF7F2
:10CBF00007FB04F58670EBF041FA04F1E800EBF076
:10CC00002FFA04F1C400EBF02BFA04F19C00EEF0D3
:10CC100091FC2046F6F794FC204670BDD03C16707F
:10CC200010B50446FFF7EAFE46F2684120462BF1B4
:10CC3000DFFE204610BD000038B5314B00F50F5522
:10CC40000446036005F124001835FAF721FD284653
:10CC500004F50055EAF0FAFDD5F8D403EBF0D6F967
:10CC6000D5F8C803EBF0D2F9D5F8BC03EBF0CEF958
:10CC7000D5F8B003EBF0CAF9D5F8A403EBF0C6F988
:10CC8000D5F8980304F50D55EBF0C0F905F1340023
:10CC90002835FAF7FDFC2846EAF0D8FD04F50B50DC
:10CCA0001BF016F804F57C70FFF712FC04F54C70CD
:10CCB000F7F75CFC04F522701BF00AF804F5B87075
:10CCC000F6F712FD04F59470EBF020FD04F5887082
:10CCD000FBF796FA04F1F400EBF0C2F904F1DC0082
:10CCE000EBF0CCF904F1C400EBF0C8F904F19C00BE
:10CCF000EEF020FC2046F6F723FC204638BD00BFAE
:10CD0000983C167010B50446FFF796FF4FF410518B
:10CD100020462BF16DFE204610BD000070B5624B21
:10CD200000F5804504460360D5F8080704F58C46F5
:10CD3000EBF06CF9D5F8FC06EBF068F9D5F8F006E5
:10CD4000EBF064F9D5F8E406EBF060F9D5F8D80615
:10CD5000EBF05CF9D5F8CC06EBF058F9D5F8C00645
:10CD6000EBF054F9D5F8B406EBF050F9D5F8A80675
:10CD7000EBF04CF9D5F89C06EBF048F9D5F89006A5
:10CD8000EBF044F9D5F88406EBF040F9D5F87806D5
:10CD9000EBF03CF9D5F86C06EBF038F9D5F8600605
:10CDA000EBF034F906F140003436FAF771FC304606
:10CDB000EAF04CFDD5F8300604F58C45EBF026F989
:10CDC00005F10C00FAF764FC284604F58B45EAF0FF
:10CDD0003DFD05F164005835FAF75AFC2846EAF0A3
:10CDE00035FD04F589405830F6F76EFD04F58840AE
:10CDF00030301AF06DFF04F515502030FFF768FB56
:10CE000004F511502030F6F75FFD04F50E50383070
:10CE10001AF05EFF04F50A502030F6F765FC04F5C1
:10CE20007470FFF755FB04F54A701AF051FF04F5D2
:10CE30001A70F7F79BFB04F50270F6F733FC04F564
:10CE4000E070EBF063FC04F5D670EBF017F904F535
:10CE5000C870FBF7D5F904F5C070EBF00FF904F5D5
:10CE6000AE70EBF0FDF804F5A270EBF007F904F5F5
:10CE70009670EBF003F904F58870FBF7C1F904F143
:10CE8000F400EBF0EDF804F1DC00EBF0F7F804F15E
:10CE9000C400EBF0F3F804F19C00EEF04BFB2046ED
:10CEA000F6F74EFB204670BD103C1670036813B5B4
:10CEB00004464BB19B68834206D000238B2123207C
:10CEC0001A46009329F0B2FB23680BB162689A609E
:10CED000626802B113600023C4E9003302B010BDE0
:10CEE0002DE9F041066892B004468846174666B1BF
:10CEF00006F10801227901F10C0342B1012220461A
:10CF000012B0BDE8F0411BF049BD3146F2E7A06820
:10CF10006D468DF84420CDE90B010121CDE90F329A
:10CF2000CDE90D1312AB13E90F0007C52B700BAB46
:10CF300004A80ECBA6F020FAE168A6EB0802304662
:10CF4000B847054B04A81C7EEBF030F884F00104D0
:10CF5000204612B0BDE8F08158540380014AD02128
:10CF6000FFF7BEBF9D7F0270014AE821FFF7B8BFFF
:10CF70008B7F02700B680BB10360586041600860E2
:10CF800070470000F0B500F52815364B002605F572
:10CF90001E772DED028B93B0384604930A96FAF76C
:10CFA000C0FF014604A8E6F0C5FE04A905F5D87047
:10CFB000FBF73AF83846FAF7B4FF014604A8E6F062
:10CFC000B9FE04A905F5DE70FBF72EF805F526700D
:10CFD000FAF7A7FF014604A8E6F0ACFE04A905F5A0
:10CFE000DA70FBF721F805F52E70FAF79AFF90ED4D
:10CFF000008A6846B8EEC88BEBF0FAF8324669460C
:10D000000BA88DED028BFAF734FF0BA904A8E6F00C
:10D01000D7FE0BA81CF01FF904A905F5E070FBF77B
:10D0200003F805F53070FAF77CFF014604A8E6F036
:10D0300081FE04A905F5E270FAF7F6FF05F53870F0
:10D04000FAF76FFF014604A8E6F074FE04A905F59F
:10D05000DC70FAF7E9FF04A81CF0FDF813B0BDEC92
:10D06000028BF0BD42721870074B10B5044640F8B1
:10D07000C03BEBF04BFB04F19C00EEF05BFA20466A
:10D08000F6F75EFA204610BD1867167010B5044614
:10D09000FFF7EAFF4FF4847120462BF1A9FC2046EC
:10D0A00010BD0000074B10B5044640F8C03BEBF044
:10D0B0002DFB04F19C00EEF03DFA2046F6F740FA15
:10D0C000204610BD8065167010B50446FFF7EAFFD4
:10D0D0004FF4847120462BF18BFC204610BD0000DC
:10D0E000074B10B5044640F8C03BEBF00FFB04F1D2
:10D0F0009C00EEF01FFA2046F6F722FA204610BDFB
:10D100001065167010B50446FFF7EAFF4FF48471FE
:10D1100020462BF16DFC204610BD0000074B10B5DA
:10D12000044640F8C03BEBF0F1FA04F19C00EEF04D
:10D1300001FA2046F6F704FA204610BDD8641670AE
:10D1400010B50446FFF7EAFF4FF4847120462BF137
:10D150004FFC204610BD0000074B10B5044640F8B8
:10D16000C03BEBF0D3FA04F19C00EEF0E3F920466B
:10D17000F6F7E6F9204610BDA064167010B5044617
:10D18000FFF7EAFF4FF4847120462BF131FC204673
:10D1900010BD0000074B10B5044640F8C03BEBF053
:10D1A000B5FA04F19C00EEF0C5F92046F6F7C8F98F
:10D1B000204610BD6864167010B50446FFF7EAFFFC
:10D1C0004FF4847120462BF113FC204610BD000063
:10D1D000074B10B5044640F8C03BEBF097FA04F15A
:10D1E0009C00EEF0A7F92046F6F7AAF9204610BDFC
:10D1F000F861167010B50446FFF7EAFF4FF484712A
:10D2000020462BF1F5FB204610BD0000064B10B563
:10D21000044640F80C3BEAF0B5FE04F10800EAF0E1
:10D2200055FF204610BD00BF3058167010B504469B
:10D23000FFF7ECFF102120462BF1DAFB204610BD52
:10D24000064B10B5044640F80C3BEAF09BFE04F197
:10D250000800EAF03BFF204610BD00BF30581670B2
:10D2600010B50446FFF7ECFF102120462BF1C0FB60
:10D27000204610BD064B10B5044640F80C3BEAF0C2
:10D2800081FE04F10800EAF021FF204610BD00BF36
:10D290003058167010B50446FFF7ECFF10212046F9
:10D2A0002BF1A6FB204610BD064B10B5044640F8F6
:10D2B0000C3BEAF067FE04F10800EAF007FF2046A5
:10D2C00010BD00BF3058167010B50446FFF7ECFFD4
:10D2D000102120462BF18CFB204610BD064B10B5CB
:10D2E000044640F80C3BEAF04DFE04F10800EAF079
:10D2F000EDFE204610BD00BF3058167010B5044634
:10D30000FFF7ECFF102120462BF172FB204610BDE9
:10D31000074B10B503610446064B40F80C3BEAF09E
:10D3200031FE04F10800EAF0D1FE204610BD00BF36
:10D33000686A16703058167010B50446FFF7E8FF9B
:10D34000142120462BF154FB204610BD064B10B58E
:10D35000044640F80C3BEAF015FE04F10800EAF040
:10D36000B5FE204610BD00BF3058167010B50446FB
:10D37000FFF7ECFF102120462BF13AFB204610BDB1
:10D38000064B10B5044640F80C3BEAF0FBFD04F1F7
:10D390000800EAF09BFE204610BD00BF3058167012
:10D3A00010B50446FFF7ECFF102120462BF120FBBF
:10D3B000204610BD074B10B503610446064B40F8EC
:10D3C0000C3BEAF0DFFD04F10800EAF07FFE2046A6
:10D3D00010BD00BFF86816703058167010B50446BE
:10D3E000FFF7E8FF142120462BF102FB204610BD79
:10D3F000074B10B503610446064B40F80C3BEAF0BE
:10D40000C1FD04F10800EAF061FE204610BD00BF36
:10D410001C6016703058167010B50446FFF7E8FF10
:10D42000142120462BF1E4FA204610BD074B10B51D
:10D4300003610446064B40F80C3BEAF0A3FD04F1FF
:10D440000800EAF043FE204610BD00BF485F16709A
:10D450003058167010B50446FFF7E8FF1421204637
:10D460002BF1C6FA204610BD074B10B503610446E8
:10D47000064B40F80C3BEAF085FD04F10800EAF0A9
:10D4800025FE204610BD00BFE45E167030581670B1
:10D4900010B50446FFF7E8FF142120462BF1A8FA47
:10D4A000204610BD074B10B503610446064B40F8FB
:10D4B0000C3BEAF067FD04F10800EAF007FE2046A5
:10D4C00010BD00BFDC5D16703058167010B50446F4
:10D4D000FFF7E8FF142120462BF18AFA204610BD01
:10D4E000204B10B504460360D0F8B409EAF08EFD75
:10D4F000D4F8A809EAF08AFDD4F89C09EAF086FD80
:10D50000D4F89009EAF082FD04F51160EBF08EF892
:10D5100004F6C800EBF0FAF804F50860EBF0F6F852
:10D5200004F5FB601AF0D4FB04F5E760F6F708F8A1
:10D5300004F5D2601AF0CCFB04F5D060EAF09EFD51
:10D5400004F5CD60EAF09AFD04F5CA60EAF096FDB4
:10D5500004F5C760EAF092FD2046F7F755FD204636
:10D5600010BD00BF0074167010B50446FFF7B8FF79
:10D5700040F6B81120462BF13BFA204610BD0000C2
:10D58000054B10B5044640F8A83BEBF02DF82046BB
:10D590001AF09EFB204610BD905C167010B5044634
:10D5A000FFF7EEFFB02120462BF122FA204610BDF6
:10D5B000034B10B504460360F6F7D8FF204610BDB4
:10D5C000506C167010B50446FFF7F2FFC0212046DC
:10D5D0002BF10EFA204610BD034B10B50446036034
:10D5E000F6F7C4FF204610BD8867167010B50446D4
:10D5F000FFF7F2FFC02120462BF1FAF9204610BDBB
:10D60000064B10B50446036000F62440EAF0ECFF38
:10D610002046F8F773FA204610BD00BFEC6E167076
:10D6200010B50446FFF7ECFF4FF4436120462BF1A1
:10D63000DFF9204610BD00000B4B10B50446036017
:10D6400000F58A501C30EAF0CFFF04F58A50143000
:10D65000EAF0CAFF04F58A500C30EAF0C5FF204614
:10D66000F8F756FC204610BDD866167010B5044673
:10D67000FFF7E2FF41F2681120462BF1B9F920468D
:10D6800010BD0000064B10B50446036000F5EC50D9
:10D690001830EAF0A9FF20460CF0EEFB204610BD42
:10D6A000585F167010B50446FFF7ECFF41F6A8511D
:10D6B00020462BF19DF9204610BD0000144B10B5FB
:10D6C00004460360D0F8FC0DEAF0A0FCD4F8F00D9D
:10D6D000EAF09CFCD4F8E40DEAF098FCD4F8D80DFC
:10D6E000EAF094FCD4F8CC0DEAF090FCD4F8C00D2C
:10D6F000EAF08CFCD4F8B40DEAF088FCD4F8A80D5C
:10D70000EAF084FC2046F8F751FB204610BD00BF2C
:10D71000485D167010B50446FFF7D0FF4FF4606106
:10D7200020462BF165F9204610BD00000E4B10B5C8
:10D7300004460360D0F8D80DEAF068FCD4F8CC0DAC
:10D74000EAF064FCD4F8C00DEAF060FCD4F8B40D43
:10D75000EAF05CFCD4F8A80DEAF058FC2046F8F793
:10D7600025FB204610BD00BFC85C167010B50446EE
:10D77000FFF7DCFF4FF45E6120462BF139F92046BC
:10D7800010BD0000104B10B504460360D0F88C0E9D
:10D79000EAF03CFCD4F8800EEAF038FCD4F8740EC1
:10D7A000EAF034FCD4F8680EEAF030FCD4F85C0EF1
:10D7B000EAF02CFCD4F8500EEAF028FC2046F8F7EA
:10D7C00065FA204610BD00BF085D167010B504460E
:10D7D000FFF7D8FF4FF4696120462BF109F9204685
:10D7E00010BD10B50446FFF799FA44F210712046B7
:10D7F0002BF1FEF8204610BD244B10B50446036003
:10D80000D0F8F805EAF002FCD4F8EC05EAF0FEFBEB
:10D81000D4F8E005EAF0FAFBD4F8D405EAF0F6FB18
:10D8200004F5B760EAF0E0FE04F5B560EAF0DCFE6E
:10D8300004F5A660EAF0FAFE04F59D60EAF066FFE2
:10D8400004F58E60EAF0F2FE04F52A70F6F77AF835
:10D8500004F500701AF03CFA04F5AC701AF038FACE
:10D8600004F58870EAF052FF04F1FC00EAF006FCCF
:10D8700004F1E400EAF002FC04F1BC00EDF05AFE11
:10D880002046F6F705FF204610BD00BFAC6A1670B3
:10D8900010B50446FFF7B0FF4FF4C06120462BF1EE
:10D8A000A7F8204610BD000038B52D4B00F51755E0
:10D8B0000446036005F138002C35F9F7E9FE2846E7
:10D8C00004F50055E9F0C2FFD5F8E805EAF09EFB43
:10D8D000D5F8DC05EAF09AFBD5F8D005EAF096FB1E
:10D8E00004F515501030EAF0A1FE04F5145008308C
:10D8F000EAF00CFF04F51350EAF008FF04F51250AB
:10D900003830EAF0E3FB04F528700BF053FE04F521
:10D91000FC701AF0DDF904F5F470FFF777FC04F5FC
:10D92000D070EAF0F3FE04F59470EAF07FFE04F59F
:10D930008C70EAF0A3FB04F58070EAF09FFB04F121
:10D94000E800EAF09BFB04F1D000EAF097FB04F159
:10D95000A800EDF0EFFD20461AF0BAF9204638BDD8
:10D960007873167010B50446FFF79EFF42F21061FF
:10D9700020462BF13DF8204610BD000038B52D4B58
:10D9800000F525550446036005F138002C35F9F7FC
:10D990007FFE284604F50055E9F058FFD5F86809E0
:10D9A000EAF034FBD5F85C09EAF030FBD5F8500911
:10D9B000EAF02CFB04F523501030EAF037FE04F5B2
:10D9C00022500830EAF0A2FE04F52150EAF09EFE53
:10D9D00004F520503830EAF079FB04F528700BF09C
:10D9E0004FFE04F5FC701AF073F904F5F470FFF7BC
:10D9F00027FC04F5D070EAF089FE04F59470EAF093
:10DA000015FE04F58C70EAF039FB04F58070EAF03D
:10DA100035FB04F1E800EAF031FB04F1D000EAF054
:10DA20002DFB04F1A800EDF085FD20461AF050F919
:10DA3000204638BD2873167010B50446FFF79EFFC8
:10DA400042F6901120462AF1D3FF204610BD000077
:10DA500070B5604B00F547550446036005F148007A
:10DA60003C35F9F715FE04F54456284604F54055B3
:10DA7000E9F0ECFED5F8F801EAF0C8FAD5F8EC01C7
:10DA8000EAF0C4FAD5F8E001EAF0C0FAD5F8D4011A
:10DA9000EAF0BCFAD5F8C801EAF0B8FAD5F8BC014A
:10DAA000EAF0B4FAD5F8B001EAF0B0FAD5F8A4017A
:10DAB000EAF0ACFAD5F89801EAF0A8FAD5F88C01AA
:10DAC000EAF0A4FAD5F88001EAF0A0FAD5F87401DA
:10DAD000EAF09CFAD5F86801EAF098FA06F14800F5
:10DAE0003C36F9F7D5FD304604F54456E9F0AEFE74
:10DAF00006F124001836F9F7CBFD3046E9F0A6FE12
:10DB0000D5F81401EAF082FAD5F80801EAF07EFAB5
:10DB1000D5F8FC00EAF07AFAD5F8F000EAF076FAE7
:10DB2000D5F8E400EAF072FAD5F8D800EAF06EFA17
:10DB300028461030F6F7ACFD04F53B503830F5F7C9
:10DB4000D3FD04F538503830F6F7A2FD04F5315016
:10DB50003030F5F7F7FE04F52E503030F6F798FD2B
:10DB600004F5E8501830F8F7EDF804F59550F7F79C
:10DB70004FF904F58C50F5F7EFFD04F58350F5F7F8
:10DB8000EBFD04F5E470F8F7DDF804F5C070EAF099
:10DB9000BDFD04F5B670EAF071FA04F5A470EAF080
:10DBA0005FFA04F59270EAF05BFA04F58670EAF029
:10DBB00065FA04F1E800EAF053FA04F1C400EAF06F
:10DBC0004FFA04F19C00EDF0B5FC2046F5F7B8FCE7
:10DBD000204670BD7872167010B50446FFF738FF06
:10DBE00043F2202120462AF103FF204610BD000009
:10DBF000144B10B504460360D0F8980FEAF006FA0B
:10DC0000D4F88C0FEAF002FAD4F8800FEAF0FEF9AB
:10DC100004F6A850F5F796FE04F68840F5F79CFD4B
:10DC200004F66840EAF01CFA04F54560EAF026FACA
:10DC300004F62C40EAF014FA2046F7F75FFF20467E
:10DC400010BD00BF2866167010B50446FFF7D0FF60
:10DC50004FF47A6120462AF1CBFE204610BD000029
:10DC600070B5344B00F5805504460360D5F82401A7
:10DC700004F58656EAF0CAF9D5F81801EAF0C6F9B3
:10DC8000D5F80C01EAF0C2F91436D5F80001EAF033
:10DC9000BDF904F58750F9F7FBFC304604F58556CD
:10DCA000E9F0D4FD06F11C001036F9F7F1FC30461E
:10DCB00004F58456E9F0CAFDD5F8AC00EAF0A6F9FF
:10DCC00006F10C00F9F7E4FC304604F58256E9F061
:10DCD000BDFD06F128001C36F9F7DAFC3046E9F004
:10DCE000B5FDA86DEAF092F904F57360F5F734FD1F
:10DCF00004F56160F5F730FD04F54F60F5F72CFD94
:10DD000004F53D60F5F728FD04F52B60F5F724FDDB
:10DD100004F52960EAF0A4F904F66C20EAF0A0F911
:10DD200004F64820EAF09CF92046FBF731FB204638
:10DD300070BD00BFE85D167010B50446FFF790FF98
:10DD400041F2281120462AF153FE204610BD000062
:10DD500038B52C4B00F5805504460360D5F8940285
:10DD6000EAF054F9D5F88802EAF050F9D5F87C02C7
:10DD7000EAF04CF9D5F87002EAF048F9D5F86402F7
:10DD8000EAF044F9D5F85802EAF040F9D5F84C0227
:10DD9000EAF03CF904F591501030EAF025FC04F566
:10DDA00091500830EAF020FC04F589500830F5F76E
:10DDB0008BFD04F57660F5F7C5FD04F56460F5F7B5
:10DDC000CBFC04F55260F5F7C7FC04F55060EAF0AF
:10DDD00047F904F6DC40EAF043F904F6B840EAF00B
:10DDE0003FF9D4F8AC0CEAF011F904F68840EAF0F7
:10DDF00037F904F66440EAF033F92046F8F75CF8A6
:10DE0000204638BDE872167010B50446FFF7A0FF33
:10DE100041F2982120462AF1EBFD204610BD00007A
:10DE200038B51D4B00F5805504460360D5F86C08E5
:10DE3000EAF0ECF8D5F86008EAF0E8F8D5F854080C
:10DE4000EAF0E4F8D5F84808EAF0E0F8D5F83C083C
:10DE5000EAF0DCF804F59C500830F6F759FF04F5B9
:10DE60006F60F6F755FF04F65820F6F751FF04F5FA
:10DE7000B860F6F74DFF04F59470F6F749FF04F12A
:10DE8000E000EAF043FC04F1BC00EDF053FB204657
:10DE9000F6F76CFB204638BDD46F167010B50446FB
:10DEA000FFF7BEFF41F6700120462AF1A1FD204692
:10DEB00010BD000038B5504B00F580550446036096
:10DEC000D5F83407EAF0A2F8D5F82807EAF09EF86A
:10DED000D5F81C07EAF09AF8D5F81007EAF096F89A
:10DEE000D5F80407EAF092F8D5F8F806EAF08EF8CB
:10DEF000D5F8EC06EAF08AF8D5F8E006EAF086F8FC
:10DF0000D5F8D406EAF082F8D5F8C806EAF07EF82B
:10DF1000D5F8BC06EAF07AF8D5F8B006EAF076F85B
:10DF2000D5F8A406EAF072F8D5F89806EAF06EF88B
:10DF3000D5F88C06EAF06AF8D5F88006EAF066F8BB
:10DF400004F5B1501030EAF0E1FB04F5A8501830A8
:10DF5000F5F7CAFB04F68830FAF71EFF04F6C8206E
:10DF6000F6F704FB04F51060F5F7ECFC04F5ED6042
:10DF7000F6F724F804F5D960F5F7E2FA04F5C16084
:10DF8000F6F7F4FA04F58860F5F7DCFC04F51E708A
:10DF9000F5F7D8FC04F50C70EAF0B8FB04F5DC707A
:10DFA000EAF044FB04F5CE70EAF05AF804F5C270CA
:10DFB000EAF064F804F5B070EAF052F804F5A470E1
:10DFC000EAF05CF804F59870EAF058F804F58C7003
:10DFD000EAF054F804F1F400EAF042F804F1D00059
:10DFE000EAF03EF804F1A800EDF0A4FA204619F09A
:10DFF0006FFE204638BD00BF3064167010B5044671
:10E00000FFF758FF41F2387120462AF1F1FC204613
:10E0100010BD000038B52D4B00F5175504460360C0
:10E0200005F138002C35F9F733FB284604F5005587
:10E03000E9F00CFCD5F8E805E9F0E8FFD5F8DC05D7
:10E04000E9F0E4FFD5F8D005E9F0E0FF04F515505C
:10E050001030EAF0EBFA04F514500830EAF056FB01
:10E0600004F51350EAF052FB04F512503830EAF090
:10E070002DF804F528700BF069FB04F5FC7019F01D
:10E0800027FE04F5F470FFF7F5F804F5D070EAF018
:10E090003DFB04F59470EAF0C9FA04F58C70E9F0E0
:10E0A000EDFF04F58070E9F0E9FF04F1E800E9F024
:10E0B000E5FF04F1D000E9F0E1FF04F1A800EDF084
:10E0C00039FA204619F004FE204638BD846D1670DA
:10E0D00010B50446FFF79EFF42F2106120462AF178
:10E0E00087FC204610BD000038B52D4B00F51755B4
:10E0F0000446036005F138002C35F9F7C9FA2846C3
:10E1000004F50055E9F0A2FBD5F8E805E9F07EFF3B
:10E11000D5F8DC05E9F07AFFD5F8D005E9F076FF0F
:10E1200004F515501030EAF081FA04F51450083067
:10E13000EAF0ECFA04F51350EAF0E8FA04F51250AC
:10E140003830E9F0C3FF04F528700BF065FB04F5E7
:10E15000FC7019F0BDFD04F5F470FFF7A5F804F5A7
:10E16000D070EAF0D3FA04F59470EAF05FFA04F59F
:10E170008C70E9F083FF04F58070E9F07FFF04F113
:10E18000E800E9F07BFF04F1D000E9F077FF04F14B
:10E19000A800EDF0CFF9204619F09AFD204638BDD1
:10E1A0008C6C167010B50446FFF79EFF42F21061AA
:10E1B00020462AF11DFC204610BD000070B5414BE1
:10E1C00000F5AA450446036005F10C00F9F760FA72
:10E1D000284604F5A045E9F039FB04F5A946D5F831
:10E1E000FC04E9F013FFD5F8F004E9F00FFFD5F8CF
:10E1F000E404E9F00BFFD5F8D804E9F007FF06F1D5
:10E2000038002C36F9F744FA3046E9F01FFBD5F810
:10E21000A804E9F0FBFE04F5A9401830EAF0E4F99F
:10E2200004F5A8402030EAF001FA04F5A740583080
:10E23000EAF06CFA04F5A7401030EAF067FA04F54A
:10E24000A540683019F044FD04F5C2600BF0B0FB46
:10E2500004F5BF60FFF75CF804F5AB60F5F770F903
:10E2600004F5F470F7F720F904F5D070EAF04EFAEF
:10E2700004F5BC70E9F0E2FE04F5B070E9F0FEFED2
:10E2800004F59E70E9F0ECFE04F59270E9F0F6FEFC
:10E2900004F58670E9F0F2FE04F1F400E9F0EEFE18
:10E2A00004F1DC00E9F0EAFE04F1C400E9F0E6FE66
:10E2B00004F19C00EDF03EF92046F5F741F92046C7
:10E2C00070BD00BF146A167010B50446FFF776FFE4
:10E2D00045F2285120462AF18BFB204610BD000054
:10E2E00038B53D4B00F5A9450446036005F16000D3
:10E2F0005435F9F7CDF9284604F5A045E9F0A6FA1A
:10E30000D5F8D004E9F082FED5F8C404E9F07EFE29
:10E31000D5F8B804E9F07AFED5F8AC04E9F076FE59
:10E32000D5F8A004E9F072FE04F5A9401030EAF037
:10E330005BF904F5A8404830EAF0E8F904F5A74095
:10E340005030EAF073F904F5A7400830EAF0DEF93E
:10E3500004F5A5406830F5F7F3F804F5A440403023
:10E3600019F0B6FC04F5A4403030FEF7EFFF04F5D9
:10E37000AB600BF083FB04F5F470F7F795F804F548
:10E38000D070EAF0C3F904F5C870E9F077FE04F53F
:10E39000BC70E9F073FE04F5B070E9F06FFE04F5AF
:10E3A0009870E9F04BFE04F58C70E9F067FE04F517
:10E3B0008070E9F063FE04F1E800E9F05FFE04F12B
:10E3C000C400E9F04DFE04F19C00EDF0B3F82046E6
:10E3D000F5F7B6F8204638BDC469167010B5044686
:10E3E000FFF77EFF45F2F84120462AF101FB204667
:10E3F00010BD00005C4B10B504460360D0F8A00CC3
:10E40000E9F004FED4F8940CE9F000FED4F8880C8E
:10E41000E9F0FCFDD4F87C0CE9F0F8FDD4F8700CC0
:10E42000E9F0F4FDD4F8640CE9F0F0FDD4F8580CF0
:10E43000E9F0ECFDD4F84C0CE9F0E8FDD4F8400C20
:10E44000E9F0E4FDD4F8340CE9F0E0FDD4F8280C50
:10E45000E9F0DCFDD4F81C0CE9F0D8FDD4F8100C80
:10E46000E9F0D4FDD4F8040CE9F0D0FDD4F8F80BB1
:10E47000E9F0CCFDD4F8EC0BE9F0C8FDD4F8E00BE2
:10E48000E9F0C4FDD4F8D40BE9F0C0FDD4F8C80B12
:10E49000E9F0BCFD04F67830EAF038F904F53360B1
:10E4A000EAF034F904F6E820EAF030F904F52260E5
:10E4B000F5F7AEF904F51860F5F742F804F6B80080
:10E4C000F5F7A6F904F5F460F5F70EF904F5E06048
:10E4D000F5F736F804F5C760F5F79AF904F5B36077
:10E4E000F5F72EF804F59F60F5F72AF804F5866035
:10E4F000F5F78EF904F57A70EAF008F904F576700C
:10E50000E9F0BCFD04F56D70E9F0AAFD04F5677053
:10E51000E9F0B4FD04F55E70E9F0A2FD04F5557074
:10E52000E9F09EFD04F54C70E9F09AFD04F54370A6
:10E53000E9F096FD04F53D70E9F0A0FD04F53770B3
:10E54000E9F09CFD04F52E70E9F08AFD04F52570D4
:10E55000E9F086FD04F51B70ECF0ECFF204695F029
:10E5600027FF204610BD00BFF863167010B50446A3
:10E57000FFF740FF40F6A84120462AF139FA20462D
:10E5800010BD00003A4B10B504460360D0F858099E
:10E59000E9F03CFDD4F84C09E9F038FDD4F8400925
:10E5A000E9F034FDD4F83409E9F030FDD4F8280955
:10E5B000E9F02CFD04F61810EAF016F804F6C8008D
:10E5C000EAF0A4F804F50C60E9F080FD04F5EC60D5
:10E5D000F9F77AFE04F5C960F5F786F804F5B1603D
:10E5E000F5F7C4FF04F59D60F4F7AAFF04F5727017
:10E5F000F5F7B2F804F53270F5F766F904F5207016
:10E60000EAF084F804F50270EAF010F804F5F67008
:10E61000E9F026FD04F5E470E9F022FD04F5D2707E
:10E62000E9F01EFD04F5C070E9F01AFD04F5B270C2
:10E63000F9F7E6FD04F5A470E9F012FD04F5927017
:10E64000E9F00EFD04F58070E9F00AFD04F1E80040
:10E65000E9F014FD04F1D000E9F010FD04F1A80088
:10E66000ECF068FF204619F033FB204610BD00BFD8
:10E670008863167010B50446FFF784FF4FF41661E7
:10E6800020462AF1B5F9204610BD000070B59B4B1D
:10E6900000F50045044603602E46D5F86401E9F014
:10E6A000B5FCD5F85801E9F0B1FCD5F84C01E9F01A
:10E6B000ADFCD5F84001E9F0A9FCD5F83401E9F04A
:10E6C000A5FCD5F82801E9F0A1FCD5F81C01E9F07A
:10E6D0009DFCD5F81001E9F099FCD5F80401E9F0AA
:10E6E00095FCD5F8F800E9F091FCD5F8EC00E9F0DC
:10E6F0008DFCD5F8E000E9F089FCD5F8D400E9F00C
:10E7000085FCD5F8C800E9F081FCD5F8BC00E9F03B
:10E710007DFCD5F8B000E9F079FCD5F8A400E9F06B
:10E7200075FCD5F89800E9F071FCD5F88C00E9F09B
:10E730006DFC5436D5F88000E9F068FC05F1600006
:10E74000F8F7A6FF3046E9F081F8286DE9F05EFCA5
:10E75000686CE9F05BFCA86BE9F058FCE86AE9F04A
:10E7600055FC05F10C00F8F793FF284604F5FF452A
:10E77000E9F06CF805F168005C35F8F789FF284688
:10E7800004F5FF45E9F062F804F5E043D3F8D80F4B
:10E79000E9F03CFC05F134002835F8F779FF28460C
:10E7A000E9F054F804F5FF402030E9F01DFF04F5CE
:10E7B000FF401830E9F018FF04F5FF401030E9F091
:10E7C00013FF04F5FE404830E9F0A0FF04F5FE40D9
:10E7D0003830E9F009FF04F5FD40103019F078FAFF
:10E7E00004F5FB40683019F073FA04F5FB40103073
:10E7F000F8F768FF04F5BD404030FDF769FE04F509
:10E8000083407830FDF74EFD04F58240503019F01A
:10E810005FFA04F506502830FCF7DCFA04F50450E2
:10E820000830F4F78DFE04F5FF501030F4F75CFF6C
:10E8300004F5F6501830F4F757FF04F58250F7F757
:10E8400081FA04F57F60F4F7F7FE04F62860F5F727
:10E8500079F804F66850F5F789FE04F53C70F6F790
:10E86000D7FA04F52A70E9F051FF04F52270E9F0B7
:10E87000F7FB04F51670E9F0E1FB04F50D70E9F023
:10E88000EFFB04F50770E9F0F9FB04F50170E9F01E
:10E89000F5FB04F5EA70E9F0D1FB04F5D870E9F076
:10E8A000DFFB04F5CA70F9F7ABFC04F5C270E9F0C0
:10E8B000E5FB04F5B470F9F7A3FC04F5AC70E9F0DE
:10E8C000DDFB04F59A70E9F0CBFB04F58C70F9F7E9
:10E8D00097FC04F1FC00E9F0C3FB04F1E000F9F758
:10E8E0008FFC04F1C400E9F0BBFB04F19C00ECF0E8
:10E8F00021FE2046F4F724FE204670BDC873167032
:10E9000010B50446FFF7C2FE48F2681120462AF10E
:10E910006FF8204610BD000070B5944B00F53045EF
:10E9200004460360D5F84C0204F53146E9F06EFB6D
:10E93000D5F84002E9F06AFBD5F83402E9F066FB4D
:10E94000D5F82802E9F062FBD5F81C02E9F05EFB7D
:10E95000D5F81002E9F05AFBD5F80402E9F056FBAD
:10E96000D5F8F801E9F052FBD5F8EC01E9F04EFBDF
:10E97000D5F8E001E9F04AFBD5F8D401E9F046FB0F
:10E98000D5F8C801E9F042FBD5F8BC01E9F03EFB3F
:10E99000D5F8B001E9F03AFBD5F8A401E9F036FB6F
:10E9A000D5F89801E9F032FB06F178006C36F8F7FB
:10E9B0006FFE3046E8F04AFFD5F86801E9F026FB23
:10E9C000D5F85C01E9F022FBD5F85001E9F01EFB17
:10E9D000D5F84401E9F01AFBD5F83801E9F016FB47
:10E9E000D5F82C01E9F012FBD5F82001E9F00EFB77
:10E9F000D5F81401E9F00AFBD5F80801E9F006FBA7
:10EA0000D5F8FC00E9F002FBD5F8F000E9F0FEFAD9
:10EA1000D5F8E400E9F0FAFAD5F8D800E9F0F6FA0A
:10EA200004F51E403830FFF793F904F51D4090308F
:10EA300019F04EF904F51C40E83019F049F904F5D5
:10EA40001C404830F4F77CFD04F50940B030FFF776
:10EA50007FF904F50940083019F03AF904F5074048
:10EA6000F030F4F741FE04F50640D830F4F73CFEF0
:10EA700004F506401830F5F779FD04F50540C83077
:10EA8000F4F7DAFD04F5B8403830FEF777FF04F507
:10EA90007D503030FDF706FC04F5CB50FEF704FF47
:10EAA00004F5B360F6F7E4F904F58760F9F70CFCB8
:10EAB00004F54870F4F718FE04F53670E9F026FE08
:10EAC00004F52F70E9F0CCFA04F52870F9F798FBFB
:10EAD00004F52370F9F794FB04F51E70F9F790FB29
:10EAE00004F51A70E9F0CAFA04F51470E9F0C6FAF0
:10EAF00004F50B70E9F0B4FA04F50470F9F780FB43
:10EB000004F5FA70E9F0ACFA04F5E870E9F0A8FA57
:10EB100004F5D670E9F0A4FA04F5C470E9F0A0FA9F
:10EB200004F5B270E9F09CFA04F5A070E9F098FAE7
:10EB300004F58E70E9F094FA04F58270E9F09EFA1B
:10EB400004F1E800F9F75CFB04F1D800E9F096FA6B
:10EB500004F1BC00F9F754FB04F19C00ECF0EAFC72
:10EB60002046F4F7EDFC204670BD00BFB072167071
:10EB700010B50446FFF7D0FE4BF25021204629F194
:10EB800037FF204610BD000038B58F4B00F52645F5
:10EB90000446036005F130002435F8F779FD284676
:10EBA00004F52045E8F052FED5F82006E9F02EFAEB
:10EBB000D5F81406E9F02AFAD5F80806E9F026FA9D
:10EBC000D5F8FC05E9F022FAD5F8F005E9F01EFACF
:10EBD000D5F8E405E9F01AFAD5F8D805E9F016FAFF
:10EBE000D5F8CC05E9F012FAD5F8C005E9F00EFA2F
:10EBF000D5F8B405E9F00AFAD5F8A805E9F006FA5F
:10EC0000D5F89C05E9F002FAD5F89005E9F0FEF98F
:10EC1000D5F88405E9F0FAF9D5F87805E9F0F6F9C0
:10EC2000D5F86C05E9F0F2F9D5F86005E9F0EEF9F0
:10EC3000D5F85405E9F0EAF9D5F8480504F5254575
:10EC4000E9F0E4F905F124001835F8F721FD28462C
:10EC500004F52445E8F0FAFD05F1FC00F035F8F77D
:10EC600017FD284604F52445E8F0F0FD05F1D40031
:10EC7000C835F8F70DFD284604F52445E8F0E6FD13
:10EC800005F1AC00A035F8F703FD284604F524454E
:10EC9000E8F0DCFD05F184007835F8F7F9FC28464A
:10ECA000E8F0D4FD04F524403030E9F02FFD04F500
:10ECB00023403030F4F708FE04F522403030F4F7FA
:10ECC00003FE04F521403030F4F7FEFD04F5024068
:10ECD0006030FDF7FDFB04F5C7401030FDF7F8FB91
:10ECE00004F589404030FDF7F3FB04F51750303050
:10ECF000FDF7EEFB04F5E460FDF7EAFB04F5CC60FC
:10ED0000F5F734FC04F5AC60F4F7DEFD04F597602C
:10ED100018F0DEFF04F56E70F4F7D6FD04F52870E8
:10ED2000F4F7E2FC04F51670E9F0F0FC04F512705B
:10ED3000E9F0A4F904F50C70E9F0A0F904F5067007
:10ED4000E9F09CF904F50070E9F098F904F5F27027
:10ED5000F9F756FA04F5E870F9F752FA04F5E0709D
:10ED6000E9F08CF904F5D270F9F74AFA04F5CA70A3
:10ED7000E9F084F904F5B870E9F072F904F5AA70C5
:10ED8000F9F73EFA04F5A270E9F078F904F590700D
:10ED9000E9F066F904F58270F9F732FA04F1F4004B
:10EDA000E9F06CF904F1DC00E9F068F904F1C40061
:10EDB000E9F064F904F19C00ECF0BCFB2046F4F7A8
:10EDC000BFFB204638BD00BF4072167010B5044628
:10EDD000FFF7DAFE4AF24861204629F109FE204693
:10EDE00010BD000038B5544B00F58A450446036059
:10EDF00005F150004435F8F74BFC284604F58045F2
:10EE0000E8F024FDD5F84005E9F000F9D5F834051F
:10EE1000E9F0FCF8D5F82805E9F0F8F8D5F81C0574
:10EE2000E9F0F4F8D5F81005E9F0F0F8D5F80405A4
:10EE3000E9F0ECF8D5F8F804E9F0E8F8D5F8EC04D6
:10EE4000E9F0E4F8D5F8E004E9F0E0F8D5F8D40406
:10EE5000E9F0DCF8D5F8C804E9F0D8F8D5F8BC0436
:10EE6000E9F0D4F8D5F8B00404F58945E9F0CEF816
:10EE700005F10C00F8F70CFC284604F58845E8F08D
:10EE8000E5FC05F164005835F8F702FC2846E8F087
:10EE9000DDFC04F588401030E9F038FC04F58640CC
:10EEA0001030F4F711FD04F51150FDF711FB04F5D6
:10EEB000AE60FDF70DFB04F59660F5F757FB04F522
:10EEC000816018F005FF04F53C70F4F70DFC04F5C3
:10EED000F870F4F7F9FC04F5D470E9F017FC04F5C8
:10EEE000CA70E9F0CBF804F5BC70F9F789F904F5BC
:10EEF000AE70E9F0B5F804F59C70E9F0B1F804F5EE
:10EF00008E70F9F77DF904F58670E9F0B7F804F131
:10EF1000F400E9F0B3F804F1DC00E9F0AFF804F133
:10EF2000C400E9F0ABF804F19C00ECF003FB2046D0
:10EF3000F4F706FB204638BD0872167010B504467B
:10EF4000FFF750FF44F26851204629F151FD204659
:10EF500010BD000038B5284B00F50055044603608D
:10EF6000D5F8A803E9F052F8D5F89C03E9F04EF87B
:10EF7000D5F89003E9F04AF8D5F88403E9F046F8AB
:10EF8000D5F87803E9F042F804F50D502830E9F09F
:10EF90009DF804F50B5018F09BFE04F5085018304E
:10EFA00018F096FE04F505501830F5F7DFFA04F571
:10EFB0000150F4F799FB04F5B870FDF789FA04F5F0
:10EFC0009470E9F0A3FB04F58870F9F719F904F1DE
:10EFD000F400E9F045F804F1DC00E9F04FF804F141
:10EFE000C400E9F04BF804F19C00ECF0A3FA2046D1
:10EFF000F4F7A6FA204638BDD071167010B5044655
:10F00000FFF7A8FF42F2B031204629F1F1FC20467B
:10F0100010BD000038B5134B0446036000F50053E3
:10F0200004F50F55D3F81404E8F0F0FF05F13400AF
:10F030002835F8F72DFB284604F50F55E8F006FCB7
:10F0400005F10C00F8F724FB2846E8F0FFFB04F577
:10F050000E502C30F9F7D4F82046FFF77BFF2046FE
:10F0600038BD00BF9871167010B50446FFF7D2FF87
:10F0700042F21841204629F1BBFC204610BD000099
:10F0800070B56D4B00F5C04504460360D5F8C0056A
:10F0900004F5C946E8F0BAFFD5F8B405E8F0B6FFC4
:10F0A000D5F8A805E8F0B2FFD5F89C05E8F0AEFF6A
:10F0B000D5F89005E8F0AAFFD5F88405E8F0A6FF9A
:10F0C000D5F87805E8F0A2FFD5F86C05E8F09EFFCA
:10F0D000D5F86005E8F09AFFD5F85405E8F096FFFA
:10F0E000D5F84805E8F092FFD5F83C05E8F08EFF2A
:10F0F000D5F83005E8F08AFFD5F82405E8F086FF5A
:10F10000D5F81805E8F082FF06F178006C36F8F7BC
:10F11000BFFA3046E8F09AFBD5F8E80404F5C94593
:10F12000E8F074FF05F144003835F8F7B1FA2846E5
:10F1300004F5C945E8F08AFB05F11C001035F8F725
:10F14000A7FA284604F5C845E8F080FB05F17400ED
:10F150006835F8F79DFA2846E8F078FB04F5C840D2
:10F160002030E9F0D3FA04F5C6400830F4F7BCFAD1
:10F1700004F5C4400830F4F7A7FB04F5C240603042
:10F1800018F0A6FD04F5C1402030F5F7EFF904F5BD
:10F1900083405030FDF79CF904F581405030F4F77E
:10F1A00093FB04F57F501030F4F78EFB04F5045008
:10F1B000FDF78EF904F50C70FDF78AF904F5F4708B
:10F1C000E9F0A4FA04F5EC70E8F058FF04F5E070FB
:10F1D000E8F054FF04F5D270F9F712F804F5C8709E
:10F1E000F9F70EF804F5C070E8F048FF04F5B470C4
:10F1F000E8F044FF04F5A670F9F702F804F59E70F4
:10F20000E8F03CFF04F58C70E8F02AFF04F1F4000C
:10F21000E8F026FF04F1DC00E8F030FF04F1C40060
:10F22000E8F02CFF04F19C00ECF084F92046F4F7A0
:10F2300087F9204670BD00BF6071167010B5044696
:10F24000FFF71EFF46F2C851204629F1D1FB2046A8
:10F2500010BD000038B5724B00F5C0450446036090
:10F26000D5F8B80BE8F0D2FED5F8AC0BE8F0CEFE3E
:10F27000D5F8A00BE8F0CAFED5F8940BE8F0C6FE6E
:10F28000D5F8880BE8F0C2FED5F87C0BE8F0BEFE9E
:10F29000D5F8700BE8F0BAFED5F8640BE8F0B6FECE
:10F2A000D5F8580BE8F0B2FED5F84C0BE8F0AEFEFE
:10F2B000D5F8400BE8F0AAFED5F8340BE8F0A6FE2E
:10F2C000D5F8280BE8F0A2FED5F81C0BE8F09EFE5E
:10F2D000D5F8100BE8F09AFED5F8040BE8F096FE8E
:10F2E000D5F8F80AE8F092FED5F8EC0AE8F08EFEC0
:10F2F000D5F8E00AE8F08AFED5F8D40AE8F086FEF0
:10F30000D5F8C80AE8F082FED5F8BC0AE8F07EFE1F
:10F31000D5F8B00AE8F07AFED5F8A40AE8F076FE4F
:10F3200004F5D5400C30E9F05FF904F5D540043020
:10F33000E9F05AF904F5D540E8F0C8FE04F5D240EA
:10F340006830F4F7D1F904F5B4404830F5F728FDFA
:10F3500004F5B2403030F4F7C7F904F594401030AA
:10F36000F5F71EFD04F591407830F4F7BDF904F58A
:10F3700090403830F5F78CF904F564501830F5F703
:10F380000FFD04F52A50F6F7DDFC04F500500830B7
:10F39000F5F73EFD04F5FA500830F5F7E7F804F507
:10F3A0002070FCF77FFF04F50E70E9F0AFF904F56B
:10F3B0000770E8F055FE04F50170E8F05FFE04F513
:10F3C000F070E8F04DFE04F5E470E8F057FE04F547
:10F3D000D270E8F045FE04F5C070E8F041FE04F597
:10F3E000AE70E8F03DFE04F5A270E8F047FE04F5CB
:10F3F0009470F8F705FF04F58670E8F031FE04F12B
:10F40000E800E8F02DFE04F1C400E8F029FE04F164
:10F410009C00ECF08FF82046F4F792F8204638BDB7
:10F420002871167010B50446FFF714FF46F6C03178
:10F43000204629F1DDFA204610BD000038B51F4BEB
:10F4400000F5005504460360D5F8080AE8F0DEFD33
:10F45000D5F8FC09E8F0DAFDD5F8F009E8F0D6FDBA
:10F4600004F55260FCF71EFF04F60840F4F73CF97F
:10F4700004F5C870F5F7CCFC04F5A470E9F046F982
:10F4800004F59670E8F0ECFD04F58A70E8F0F6FDFE
:10F4900004F1F800F8F7B4FE04F1DC00E8F0E0FD58
:10F4A00004F1C400E8F0EAFD04F19C00ECF042F83D
:10F4B0002046F4F745F8204638BD00BFF0701670BE
:10F4C00010B50446FFF7BAFF42F61021204629F195
:10F4D0008FFA204610BD000038B52C4B00F5405582
:10F4E00004460360D5F80C09E8F090FDD5F8000952
:10F4F000E8F08CFDD5F8F408E8F088FDD5F8E808C8
:10F50000E8F084FDD5F8DC08E8F080FDD5F8D008F7
:10F51000E8F07CFD04F528503030F6F713FC04F5D4
:10F5200024501830F4F7E0F804F5F550F5F770FCC6
:10F5300004F5EC70FCF7B6FE04F5C870E9F0E6F8E7
:10F5400004F5BA70E8F08CFD04F5A870E8F088FDC9
:10F5500004F59A70F8F754FE04F58C70E8F080FD1D
:10F5600004F58070E8F08AFD04F1E800E8F086FD1B
:10F5700004F1C400E8F074FD04F19C00EBF0DAFF44
:10F580002046F3F7DDFF204638BD00BFB870167087
:10F5900010B50446FFF7A0FF43F61011204629F1ED
:10F5A00027FA204610BD000070B5724B00F5C0452B
:10F5B00004460360D5F8E40504F5C946E8F026FDE5
:10F5C000D5F8D805E8F022FDD5F8CC05E8F01EFD09
:10F5D000D5F8C005E8F01AFDD5F8B405E8F016FD39
:10F5E000D5F8A805E8F012FDD5F89C05E8F00EFD69
:10F5F000D5F89005E8F00AFDD5F88405E8F006FD99
:10F60000D5F87805E8F002FDD5F86C05E8F0FEFCC9
:10F61000D5F86005E8F0FAFCD5F85405E8F0F6FCFA
:10F62000D5F84805E8F0F2FCD5F83C05E8F0EEFC2A
:10F63000D5F83005E8F0EAFCD5F82405E8F0E6FC5A
:10F64000D5F81805E8F0E2FC06F178006C36F8F71A
:10F650001FF83046E8F0FAF8D5F8E80404F5C94593
:10F66000E8F0D4FC05F144003835F8F711F82846E5
:10F6700004F5C945E8F0EAF805F11C001035F8F783
:10F6800007F8284604F5C845E8F0E0F805F17400ED
:10F690006835F7F7FDFF2846E8F0D8F804F5C840CC
:10F6A0002030E9F033F804F5C6400830F4F71CF8D0
:10F6B00004F5C440603018F00BFB04F5C340203063
:10F6C000F4F754FF04F585405030FCF701FF04F5D2
:10F6D00083405030F4F7F8F804F581405030F4F7E7
:10F6E000F3F804F50850FCF7F3FE04F54C70FCF752
:10F6F000EFFE04F50C70F4F7E7F804F5F470E9F0A8
:10F7000005F804F5EC70E8F0B9FC04F5DE70F8F7E4
:10F7100077FD04F5D470F8F773FD04F5CC70E8F0CC
:10F72000ADFC04F5C070E8F0A9FC04F5B470E8F095
:10F73000A5FC04F5A670F8F763FD04F59E70E8F0EB
:10F740009DFC04F59270E8F099FC04F58070E8F0F7
:10F7500087FC04F1DC00E8F083FC04F1C400E8F06D
:10F760008DFC04F19C00EBF0E5FE2046F3F7E8FE8B
:10F77000204670BD8070167010B50446FFF714FF68
:10F7800046F2E851204629F133F9204610BD000029
:10F7900038B53D4B00F532550446036005F12000B5
:10F7A0001435F7F775FF284604F50055E8F04EF8D4
:10F7B000D5F8900CE8F02AFCD5F8840CE8F026FC8B
:10F7C000D5F8780CE8F022FCD5F86C0CE8F01EFCBB
:10F7D000D5F8600CE8F01AFCD5F8540CE8F016FCEB
:10F7E000D5F8480CE8F012FCD5F83C0CE8F00EFC1B
:10F7F000D5F8300CE8F00AFCD5F8240CE8F006FC4B
:10F80000D5F8180CE8F002FC04F506501830F5F7AE
:10F81000FFFA04F50250F3F767FF04F5F5501830CE
:10F82000F4F790F804F583501030F6F72FFA04F54A
:10F83000EC70F6F787FA04F5C870E8F067FF04F596
:10F84000C070E8F01BFC04F5AE70E8F009FC04F5AC
:10F850009C70E8F005FC04F59070E8F00FFC04F5EE
:10F860008270F8F7CDFC04F1E800E8F0F9FB04F150
:10F87000C400E8F0F5FB04F19C00EBF05BFE2046D1
:10F88000F3F75EFE204638BD4870167010B504468A
:10F89000FFF77EFF42F6B841204629F1A9F820463D
:10F8A00010BD000038B5584B0446036000F54A50BF
:10F8B00004F54A553030EBF02FFE05F10C00F7F758
:10F8C000E7FE284604F54055E7F0C0FFD5F87C0276
:10F8D000E8F09CFBD5F87002E8F098FBD5F86402DC
:10F8E000E8F094FBD5F85802E8F090FBD5F84C020C
:10F8F000E8F08CFBD5F8400204F54855E8F086FBAB
:10F9000005F10C00F7F7C4FE2846E7F09FFF04F569
:10F9100046503030E8F0FAFE04F545502830E8F063
:10F92000F5FE04F544502030E8F0F0FE04F54050B8
:10F930000830F3F7D9FE04F53B503030F3F7D4FE2E
:10F9400004F53A502030F3F777FE04F58E50183066
:10F95000FCF7A8FC04F58C500830F3F76DFE04F5B5
:10F96000E260F5F755FA04F5BF60F3F7BDFE04F564
:10F970009C60F3F7B9FE04F57270F3F7B5FE04F579
:10F980002C70F3F7B1FE04F51A70E8F0BFFE04F531
:10F990001370E8F065FB04F50A70E8F061FB04F50C
:10F9A0000170E8F05DFB04F5F070E8F059FB04F538
:10F9B000DE70E8F055FB04F5CC70E8F051FB04F57F
:10F9C000C070E8F05BFB04F5B470E8F057FB04F599
:10F9D000A270E8F045FB04F59070E8F041FB04F5F7
:10F9E0008270F8F70DFC04F1F400E8F047FB04F135
:10F9F000C400E8F023FB04F19C00EBF09BFD2046E3
:10FA0000F3F79EFD204638BD1070167010B5044601
:10FA1000FFF748FF43F2F021204628F1E9FF204696
:10FA200010BD000070B5614B00F5804504460360D1
:10FA3000D5F82C0B04F59446E8F0E8FAD5F8200B3D
:10FA4000E8F0E4FAD5F8140BE8F0E0FAD5F8080B82
:10FA5000E8F0DCFAD5F8FC0AE8F0D8FAD5F8F00AB4
:10FA6000E8F0D4FAD5F8E40AE8F0D0FAD5F8D80AE4
:10FA7000E8F0CCFAD5F8CC0AE8F0C8FAD5F8C00A14
:10FA8000E8F0C4FAD5F8B40AE8F0C0FAD5F8A80A44
:10FA9000E8F0BCFAD5F89C0AE8F0B8FAD5F8900A74
:10FAA000E8F0B4FAD5F8840AE8F0B0FAD5F8780AA4
:10FAB000E8F0ACFA06F158004C36F7F7E9FD3046AD
:10FAC000E7F0C4FED5F8480AE8F0A0FA04F5934040
:10FAD0007830E8F01BFE04F546500830FEF7A0F938
:10FAE00004F541503030F3F7FFFD04F53F5010307E
:10FAF000F3F726FD04F504503830F6F723F904F542
:10FB0000FB501030F3F71EFF04F589500830F6F76C
:10FB1000BDF804F53870F6F7B9F804F52670E8F08A
:10FB2000F5FD04F51E70E8F09BFA04F51570E8F099
:10FB300097FA04F50E70F8F763FB04F50770E8F028
:10FB40008FFA04F5FC70E8F08BFA04F5F070E8F039
:10FB500095FA04F5E270F8F753FB04F5D470E8F079
:10FB60007FFA04F5C870E8F089FA04F5B670E8F099
:10FB700077FA04F5A470E8F073FA04F59270E8F0EF
:10FB80006FFA04F58670E8F079FA04F1E800E8F01D
:10FB900067FA04F1C400E8F063FA04F19C00EBF0AA
:10FBA000C9FC2046F3F7CCFC204670BD9C6F167054
:10FBB00010B50446FFF736FF44F63031204628F1F1
:10FBC00017FF204610BD000070B5754B00F5CB4502
:10FBD0000446036005F174006835F7F759FD04F534
:10FBE000CA46284604F5C045E7F030FED5F8E405DE
:10FBF000E8F00CFAD5F8D805E8F008FAD5F8CC0505
:10FC0000E8F004FAD5F8C005E8F000FAD5F8B40534
:10FC1000E8F0FCF9D5F8A805E8F0F8F9D5F89C0566
:10FC2000E8F0F4F9D5F89005E8F0F0F9D5F8840596
:10FC3000E8F0ECF9D5F87805E8F0E8F9D5F86C05C6
:10FC4000E8F0E4F9D5F86005E8F0E0F9D5F85405F6
:10FC5000E8F0DCF9D5F84805E8F0D8F906F1280015
:10FC60001C36F7F715FD3046E7F0F0FDD5F818051E
:10FC7000E8F0CCF9D5F80C05E8F0C8F9D5F800059E
:10FC8000E8F0C4F9D5F8F404E8F0C0F9D5F8E804D0
:10FC900004F5C945E8F0BAF905F144003835F7F73D
:10FCA000F7FC284604F5C945E7F0D0FD05F11C0036
:10FCB0001035F7F7EDFC284604F5C845E7F0C6FD1A
:10FCC00005F174006835F7F7E3FC2846E7F0BEFD60
:10FCD00004F5C8402030E8F019FD04F5C640203096
:10FCE000F3F7F2FD04F588405030FCF7F1FB04F522
:10FCF0001650FCF7EDFB04F51250F3F7E5FD04F5A3
:10FD0000B660FCF7E5FB04F59E60F4F72FFC04F504
:10FD1000896017F0DDFF04F54C70F3F7E5FC04F59E
:10FD20000C70F3F7D1FD04F5F470E8F0EFFC04F586
:10FD3000EC70E8F0A3F904F5E070E8F09FF904F541
:10FD4000D470E8F09BF904F5C670F8F759FA04F599
:10FD5000BE70E8F093F904F5B270E8F08FF904F59D
:10FD6000A470F8F74DFA04F59670E8F079F904F507
:10FD70008A70E8F083F904F1F800F8F741FA04F129
:10FD8000E800E8F07BF904F1C400E8F069F904F157
:10FD90009C00EBF0CFFB2046F3F7D2FB204670BD72
:10FDA000646F167010B50446FFF70EFF46F210613F
:10FDB000204628F11DFE204610BD000038B500F594
:10FDC0000825FD4B04460360D5F8300FE8F01EF916
:10FDD000D5F8240FE8F01AF9D5F8180FE8F016F95D
:10FDE000D5F80C0FE8F012F9D5F8000FE8F00EF98D
:10FDF000D5F8F40EE8F00AF9D5F8E80EE8F006F9BF
:10FE0000D5F8DC0EE8F002F9D5F8D00EE8F0FEF8EF
:10FE1000D5F8C40EE8F0FAF8D5F8B80EE8F0F6F820
:10FE2000D5F8AC0EE8F0F2F8D5F8A00EE8F0EEF850
:10FE3000D5F8940EE8F0EAF8D5F8880EE8F0E6F880
:10FE4000D5F87C0EE8F0E2F8D5F8700EE8F0DEF8B0
:10FE5000D5F8640EE8F0DAF8D5F8580EE8F0D6F8E0
:10FE6000D5F84C0EE8F0D2F8D5F8400EE8F0CEF810
:10FE7000D5F8340EE8F0CAF8D5F8280EE8F0C6F840
:10FE8000D5F81C0EE8F0C2F8D5F8100EE8F0BEF870
:10FE9000D5F8040EE8F0BAF8D5F8F80DE8F0B6F8A1
:10FEA000D5F8EC0DE8F0B2F8D5F8E00DE8F0AEF8D2
:10FEB000D5F8D40DE8F0AAF8D5F8C80DE8F0A6F802
:10FEC000D5F8BC0DE8F0A2F8D5F8B00DE8F09EF832
:10FED000D5F8A40DE8F09AF8D5F8980DE8F096F862
:10FEE00005F64850E8F012FC04F5022004F5B3359D
:10FEF00000F5E760FFF768FE04F5FB2000F5816080
:10FF0000FFF790FD04F5F52000F58C70FFF7CAFCB3
:10FF100004F5EF2000F58C60FFF73AFC04F5E220D1
:10FF200000F5CF60FFF740FB04F5DB2000F5AD6086
:10FF3000FFF7D2FA04F5D62000F55670FFF77EFAE7
:10FF400004F5C82000F5F360FFF784F904F5BC2040
:10FF500000F5E870FFF794F804F5B72000F5B760F6
:10FF6000FFF758F804F5AF205030FEF73BFF04F5DB
:10FF70009A2000F50270FEF707FE04F5932000F5C5
:10FF8000FD60FDF765FD04F57B3000F5CC70FEF7F4
:10FF9000C3FC04F55B303030FEF778FB04F55830D5
:10FFA00000F51E70FDF79CFA04F5463000F55A7016
:10FFB000FCF7B4FE04F5443000F5EC70F8F7ECFE05
:10FFC00004F5303000F5D470F7F74AFD04F527301A
:10FFD00000F5D470FCF730FE04F50E3000F5A0708B
:10FFE000FCF70CFD04F5F5302830FCF757FC04F560
:10FFF000CC301030F7F7AEFC05F1C800FCF790FBF1
:02000004700387
:1000000005F12800F3F79CFA04F5873000F59070AD
:10001000FCF7B8FA04F5863000F5C470F3F7CEFFAC
:1000200004F56040B030FCF7B7F904F55F40F030FC
:10003000F4F79CFA04F508405830FCF745F804F54D
:100040000540D830F3F78AFF04F5A7500830FBF7D6
:100050000DFF04F5E960F5F7A9FE04F5E060E8F0AE
:1000600055FB04F5DD60F8F7CBF804F5DB60E8F04C
:1000700005F804F5D860E8F001F804F5D560E7F07C
:10008000FDFF04F5D260E7F0F9FF04F5CF60E7F07B
:10009000F5FF04F5CC60E7F0F1FF04F5C960E7F087
:1000A000EDFF04F22C60F8F7ABF804F5C260E7F05E
:1000B000D7FF04F2EC50E7F0D3FF04F2D450E7F09E
:1000C000DDFF04F2BC50E7F0D9FF04F2A450E7F0E2
:1000D000D5FF04F5B060E7F0C3FF04F5AD60E7F0CD
:1000E000CDFF04F5AA60E7F0C9FF04F5A760E7F0CB
:1000F000C5FF04F5A460E7F0C1FF04F5A160E7F0D7
:10010000BDFF04F59E60E7F0B9FF04F59B60E7F0E2
:10011000B5FF04F59860E7F0B1FF04F59560E7F0EE
:10012000ADFF04F59260E7F0A9FF04F58F60E7F0FA
:10013000A5FF04F58C60E7F0A1FF04F58960E7F006
:100140009DFF04F58660E7F099FF04F58360E7F012
:1001500095FF04F58060E7F091FF04F57A70E7F011
:100160008DFF04F57470E7F089FF04F56E70E7F019
:1001700085FF04F56870E7F081FF04F56270E7F031
:100180007DFF04F55C70E7F079FF04F55670E7F049
:1001900075FF04F55070E7F071FF04F54A70E7F061
:1001A0006DFF04F54370F8F72BF804F53E70F8F78F
:1001B00027F804F53A7001E02C6F1670E7F05EFF47
:1001C00004F53470E7F05AFF04F52E70E7F056FF9F
:1001D00004F52870E7F052FF04F52270E7F04EFFB7
:1001E00004F51C70E7F04AFF04F51670E7F046FFCF
:1001F00004F50F70F8F704F804F50B70E7F03EFF14
:1002000004F50570E7F03AFF04F5FE70E7F036FFFD
:1002100004F5F270E7F032FF04F5E670E7F02EFF28
:1002200004F5DA70E7F02AFF04F5CE70E7F026FF58
:1002300004F5C270E7F022FF04F5B670E7F01EFF88
:1002400004F5AA70E7F01AFF04F59E70E7F016FFB8
:1002500004F59270E7F012FF04F58670E7F00EFFE8
:1002600004F1F400E7F00AFF04F1DC00E7F006FF18
:1002700004F1C400E7F002FF04F19C00EBF05AF92E
:100280002046F3F75DF9204638BD00BF10B504469F
:10029000FFF794FD0249204628F1AAFB204610BD35
:1002A000388F080070B5FD4B00F5E045044603604B
:1002B000D5F8380604F5E946E7F0A8FED5F82C068F
:1002C000E7F0A4FED5F82006E7F0A0FED5F8140666
:1002D000E7F09CFED5F80806E7F098FED5F8FC0597
:1002E000E7F094FED5F8F005E7F090FED5F8E405C8
:1002F000E7F08CFED5F8D805E7F088FED5F8CC05F8
:10030000E7F084FED5F8C005E7F080FED5F8B40527
:10031000E7F07CFED5F8A805E7F078FED5F89C0557
:10032000E7F074FED5F89005E7F070FED5F8840587
:10033000E7F06CFED5F87805E7F068FED5F86C05B7
:10034000E7F064FED5F86005E7F060FED5F85405E7
:10035000E7F05CFED5F84805E7F058FED5F83C0517
:10036000E7F054FED5F83005E7F050FED5F8240547
:10037000E7F04CFED5F81805E7F048FED5F80C0577
:10038000E7F044FED5F80005E7F040FE06F1600016
:100390005436F7F77DF93046E7F058FAD5F8D0042F
:1003A000E7F034FED5F8C404E7F030FED5F8B80421
:1003B000E7F02CFED5F8AC04E7F028FED5F8A00451
:1003C000E7F024FED5F89404E7F020FED5F8880481
:1003D000E7F01CFED5F87C04E7F018FED5F87004B1
:1003E000E7F014FED5F86404E7F010FED5F85804E1
:1003F000E7F00CFED5F84C04E7F008FED5F8400411
:10040000E7F004FED5F83404E7F000FED5F8280440
:10041000E7F0FCFDD5F81C04E7F0F8FDD5F8100472
:10042000E7F0F4FDD5F80404E7F0F0FDD5F8F803A3
:10043000E7F0ECFDD5F8EC03E7F0E8FDD5F8E003D4
:10044000E7F0E4FDD5F8D403E7F0E0FDD5F8C80304
:10045000E7F0DCFDD5F8BC03E7F0D8FDD5F8B00334
:10046000E7F0D4FDD5F8A403E7F0D0FDD5F8980364
:10047000E7F0CCFDD5F88C03E7F0C8FDD5F8800394
:10048000E7F0C4FDD5F87403E7F0C0FDD5F86803C4
:10049000E7F0BCFDD5F85C03E7F0B8FDD5F85003F4
:1004A000E7F0B4FDD5F84403E7F0B0FDD5F8380324
:1004B000E7F0ACFDD5F82C03E7F0A8FDD5F8200354
:1004C000E7F0A4FDD5F81403E7F0A0FDD5F8080384
:1004D000E7F09CFDD5F8FC02E7F098FDD5F8F002B6
:1004E000E7F094FDD5F8E402E7F090FDD5F8D802E6
:1004F000E7F08CFDD5F8CC02E7F088FDD5F8C00216
:10050000E7F084FDD5F8B402E7F080FDD5F8A80245
:10051000E7F07CFDD5F89C02E7F078FDD5F8900275
:10052000E7F074FD04F5E540E8F05EF804F5E4401A
:100530007030E8F059F804F5E3403030F4F716F87D
:1005400004F5DF406830F3F7FDF904F5DC402030B6
:10055000F3F7F8F904F5D8405830F3F7F3F904F558
:10056000D6403830F3F7F8F804F5D5406030F7F7A7
:10057000A9F804F5D2401830F3F7E4F904F5D040B7
:100580007830F2F7DDFF04F5CD403030F3F7DAF9DB
:1005900004F5B540FDF734F804F5B3406030F2F7E8
:1005A000CFFF04F597401830F5F770FB04F5934042
:1005B0005030F3F7C7F904F591403030F3F7CCF839
:1005C00004F58D406830F3F7BDF904F56250203032
:1005D000F5F75CFB04F55B501830F3F7B3F904F55D
:1005E00058503830F2F7ACFF04F554501830F3F798
:1005F000B3F804F55150303017F06AFB04F54A5057
:100600002830F3F79FF904F543502030F3F79AF9B7
:1006100004F53F50F3F7A0F804F537503830F3F7FE
:1006200091F904F534503830F3F7A0FF04F52E505B
:100630002030F3F7C3FC04F52A50F3F78DF804F5E6
:1006400003503030F8F7A8FB04F500503030F3F7D2
:100650008DFF04F5FC501030F2F772FF04F5EE50F8
:100660000830F3F76FF904F5E9500830F2F768FF46
:1006700004F68870F5F7C2FB04F55C60F3F762F9E5
:1006800004F55260F2F75CFF04F65830F3F75AF9BC
:1006900004F51960F3F756F902E000BFB46E167066
:1006A00004F5F960F3F74EF904F5F060E8F02EF880
:1006B00004F26470E7F0D4FC04F24C70E7F0DEFC66
:1006C00004F5E560E7F0CCFC04F20C70F7F798FD58
:1006D00004F5DE60E7F0C4FC04F5DB60E7F0CEFC77
:1006E00004F5D860E7F0CAFC04F5D560E7F0C6FC75
:1006F00004F28C60F7F784FD04F5CE60E7F0B0FCFF
:1007000004F24C60E7F0ACFC04F5C560E7F0A8FC2F
:1007100004F20460E7F0A4FC04F5BC60E7F0A0FC80
:1007200004F2C450F7F76CFD04F2B450E7F0A6FCF5
:1007300004F29C50E7F0A2FC04F5AF60E7F090FCF7
:1007400004F5AC60E7F09AFC04F23C50E7F088FC5A
:1007500004F5A360E7F084FC04F5A060E7F08EFCEC
:1007600004F2DC40E7F07CFC04F59760E7F078FCED
:1007700004F29440E7F074FC04F58E60E7F070FC3E
:1007800004F24C40E7F06CFC04F23440E7F076FCF5
:1007900004F21C40E7F072FC04F57E70E7F060FCA8
:1007A00004F57570E7F05CFC04F56E70F7F728FD52
:1007B00004F56770E7F054FC04F55E70E7F050FC58
:1007C00004F55270E7F03AFC04F54670E7F036FCA9
:1007D00004F53D70E7F044FC04F53770E7F04EFC9B
:1007E00004F52E70E7F03CFC04F52870E7F046FCB9
:1007F00004F51F70E7F034FC04F51970E7F03EFCD7
:1008000004F51070E7F02CFC04F50770E7F028FC05
:1008100004F5FC70E7F024FC04F5F070E7F02EFC22
:1008200004F5DE70E7F01CFC04F5CC70E7F018FC72
:1008300004F5BA70E7F014FC04F5A870E7F010FCBA
:1008400004F59670E7F00CFC04F58470E7F008FC02
:1008500004F1F000E7F012FC04F1D400F7F7D0FC4B
:1008600004F1C400E7F00AFC04F19C00EAF062FE27
:100870002046F2F765FE204670BD00BF10B5044665
:10088000FFF710FD47F24061204628F1B1F82046FD
:1008900010BD0000244B10B504460360D0F84C0690
:1008A000E7F0B4FB04F5A860F3F70EF804F58560F3
:1008B000F2F71AFF04F53270F7F706FD04F51C7025
:1008C000F6F700FF04F5FC70E7F0B0FE04F5D87011
:1008D000E7F01CFF04F5CA70E7F0C2FB04F5B8703E
:1008E000E7F0BEFB04F5A670E7F0BAFB04F59470E0
:1008F000E7F0B6FB04F58870E7F0C0FB04F1F80000
:10090000E7F0BCFB04F1DC00F7F77AFC04F1C80067
:10091000F7F776FC04F1A800EAF00CFE204617F089
:10092000D7F9204610BD00BF7C6E167010B5044686
:10093000FFF7B0FF4FF4CA61204628F159F820466E
:1009400010BD000038B55A4B00F58C4504460360D5
:1009500005F184007835F6F79BFE284604F58045BE
:10096000E6F074FFD5F87406E7F050FBD5F868069A
:10097000E7F04CFBD5F85C06E7F048FBD5F85006ED
:10098000E7F044FBD5F84406E7F040FBD5F838061D
:10099000E7F03CFBD5F82C06E7F038FBD5F820064D
:1009A000E7F034FBD5F81406E7F030FBD5F808067D
:1009B000E7F02CFBD5F8FC05E7F028FBD5F8F005AF
:1009C000E7F024FBD5F8E405E7F020FBD5F8D805DF
:1009D00004F58B45E7F01AFB05F134002835F6F7EE
:1009E00057FE284604F58B45E6F030FF05F10C0074
:1009F000F6F74EFE2846E6F029FF04F51A5030308F
:100A0000FBF766FD04F516503030F2F75DFF04F594
:100A10001450083017F05CF904F50F503030F2F73D
:100A200063FE04F50D50083017F052F904F58F609D
:100A3000FBF74EFD04F56E70F3F798FD04F52E708C
:100A4000F2F742FF04F5047017F042F904F5E47080
:100A5000E7F05CFE04F5DC70E7F010FB04F5D07005
:100A6000E7F00CFB04F5C270F7F7CAFB04F5B470AD
:100A7000E7F0F6FA04F59C70E7F0E0FA04F58E7002
:100A8000F7F7BEFB04F58070E7F0EAFA04F1E8003E
:100A9000E7F0F4FA04F1C400E7F0E2FA04F19C0094
:100AA000EAF048FD2046F2F74BFD204638BD00BF76
:100AB000446E167010B50446FFF744FF44F2A0617F
:100AC000204627F195FF204610BD000038B5314B78
:100AD00000F50F550446036005F124001835F6F7BC
:100AE000D7FD284604F50055E6F0B0FED5F8D4034E
:100AF000E7F08CFAD5F8C803E7F088FAD5F8BC031C
:100B0000E7F084FAD5F8B003E7F080FAD5F8A4034B
:100B1000E7F07CFAD5F8980304F50D55E7F076FA7E
:100B200005F134002835F6F7B3FD2846E6F08EFED1
:100B300004F50B5017F0CCF804F57C70FBF7C8FCFB
:100B400004F54C70F3F712FD04F5227017F0C0F8AD
:100B500004F5B870F2F7C8FD04F59470E7F0D6FD1F
:100B600004F58870F7F74CFB04F1F400E7F078FA2D
:100B700004F1DC00E7F082FA04F1C400E7F07EFA49
:100B800004F19C00EAF0D6FC2046F2F7D9FC20469E
:100B900038BD00BF0C6E167010B50446FFF796FF07
:100BA0004FF41051204627F123FF204610BD0000CE
:100BB00038B5574B00F5804504460360D5F85C0D09
:100BC000E7F024FAD5F8500DE7F020FAD5F8440DF7
:100BD000E7F01CFAD5F8380DE7F018FAD5F82C0D27
:100BE000E7F014FAD5F8200DE7F010FAD5F8140D57
:100BF000E7F00CFAD5F8080DE7F008FAD5F8FC0C88
:100C0000E7F004FAD5F8F00CE7F000FAD5F8E40CB8
:100C1000E7F0FCF9D5F8D80CE7F0F8F9D5F8CC0CEA
:100C2000E7F0F4F9D5F8C00CE7F0F0F9D5F8B40C1A
:100C3000E7F0ECF9D5F8A80CE7F0E8F904F57850FE
:100C40000830F5F77FF804F53B502830F4F7A8F8A2
:100C500004F511503030F4F7DBF804F50E50303065
:100C6000F3F784FC04F50A501830F2F73DFD04F563
:100C70000650F2F739FD04F59760FBF713FB04F516
:100C80006870F2F731FD04F55070F2F70BFD04F5D2
:100C90002070F3F7FDFC04F50E70E7F037FD04F566
:100CA0000A70E7F0EBF904F50170E7F0D9F904F503
:100CB000F070E7F0D5F904F5E470E7F0DFF904F53A
:100CC000D270E7F0CDF904F5C070E7F0C9F904F58A
:100CD000AE70E7F0C5F904F5A270E7F0CFF904F5BE
:100CE0009470F7F78DFA04F58670E7F0B9F904F11E
:100CF000E800E7F0B5F904F1C400E7F0B1F904F158
:100D00009C00EAF017FC2046F2F71AFC204638BD9A
:100D1000D46D167010B50446FFF74AFF44F66051D3
:100D2000204627F165FE204610BD000070B5814BBE
:100D300000F5E04504460360D5F8180E04F5F946C1
:100D4000E7F064F9D5F80C0EE7F060F9D5F8000E7D
:100D5000E7F05CF9D5F8F40DE7F058F9D5F8E80DAF
:100D6000E7F054F9D5F8DC0DE7F050F9D5F8D00DDF
:100D7000E7F04CF9D5F8C40DE7F048F9D5F8B80D0F
:100D8000E7F044F9D5F8AC0DE7F040F9D5F8A00D3F
:100D9000E7F03CF9D5F8940DE7F038F9D5F8880D6F
:100DA000E7F034F9D5F87C0DE7F030F9D5F8700D9F
:100DB000E7F02CF9D5F8640DE7F028F9D5F8580DCF
:100DC000E7F024F9D5F84C0DE7F020F9D5F8400DFF
:100DD000E7F01CF9D5F8340DE7F018F9D5F8280D2F
:100DE000E7F014F9D5F81C0DE7F010F9D5F8100D5F
:100DF000E7F00CF906F170006436F6F749FC30466E
:100E0000E6F024FDD5F8E00C04F5F945E7F0FEF82E
:100E100005F13C003035F6F73BFC2846E6F016FDC0
:100E200004F5D4401830FCF793FF04F5D240F2F7F4
:100E30005BFC04F5D040583016F04AFF04F5CF4073
:100E4000303016F045FF04F5CD401830F2F74CFC79
:100E500004F58F404830FBF73BFB04F50650383073
:100E6000FDF7D8F804F50450103016F031FF04F502
:100E700001503030F2F764FB04F5F8501030F7F70A
:100E800023FA04F5F3501030F2F75AFB04F5E5505D
:100E90000830F2F757FD04F591501030F3F7B8FF22
:100EA00004F54470F3F77CFF04F51470F3F75EFB70
:100EB00004F50270E7F02AFC04F5F670E7F0D0F8CC
:100EC00004F5EA70E7F0DAF804F5DE70E7F0D6F83A
:100ED00004F5D070F7F794F904F5C670F7F790F9B8
:100EE00004F5BC70F7F78CF904F5B270F7F788F9E0
:100EF00004F5A470E7F0B4F804F59870E7F0BEF8D4
:100F000004F58C70E7F0BAF804F58070E7F0B6F8F5
:100F100004F1E800E7F0B2F804F1C400E7F0A0F84B
:100F200004F19C00EAF006FB2046F2F709FB20469C
:100F300070BD00BF4C6D167010B50446FFF7F6FE8D
:100F400047F62061204627F153FD204610BD0000E2
:100F500038B5134B0446036000F5005304F50F55F4
:100F6000D3F81404E7F052F805F134002835F6F709
:100F70008FFB284604F50F55E6F068FC05F10C00E0
:100F8000F6F786FB2846E6F061FC04F50E502C309F
:100F9000F7F736F92046FDF7DDFF204638BD00BFE4
:100FA000146D167010B50446FFF7D2FF42F21841D7
:100FB000204627F11DFD204610BD000038B5544BDA
:100FC00000F5A04504460360D5F84006E7F01EF89A
:100FD000D5F83406E7F01AF8D5F82806E7F016F841
:100FE000D5F81C06E7F012F8D5F81006E7F00EF871
:100FF000D5F80406E7F00AF8D5F8F805E7F006F8A2
:10100000D5F8EC05E7F002F8D5F8E005E6F0FEFFCC
:10101000D5F8D405E6F0FAFFD5F8C805E6F0F6FFF6
:10102000D5F8BC05E6F0F2FFD5F8B005E6F0EEFF26
:10103000D5F8A405E6F0EAFFD5F89805E6F0E6FF56
:1010400004F583404830F3F713FF04F54A50283085
:10105000F3F7A6FE04F547502830F3F787FA04F5B6
:101060000D501030F4F76EFE04F508503830F2F7EA
:101070003BFB04F504502030F2F736FB04F58B609F
:10108000FBF710F904F55070F2F72EFB04F5207011
:10109000F3F7FEFA04F50E70E7F038FB04F50A707A
:1010A000E6F0ECFF04F50170E6F0DAFF04F5F0700D
:1010B000E6F0D6FF04F5DE70E6F0D2FF04F5CC7062
:1010C000E6F0CEFF04F5BA70E6F0CAFF04F5A870AA
:1010D000E6F0C6FF04F59C70E6F0D0FF04F58E70D4
:1010E000F7F78EF804F58070E6F0BAFF04F1DC0043
:1010F000E6F0B6FF04F1C400E6F0C0FF04F19C0086
:10110000EAF018FA2046F2F71BFA204638BD00BF75
:10111000DC6C167010B50446FFF750FF45F24861CD
:10112000204627F165FC204610BD000070B5954BA8
:1011300000F5004504460360D5F8300D04F50C4673
:10114000E6F064FFD5F8240DE6F060FFD5F8180D41
:10115000E6F05CFFD5F80C0DE6F058FFD5F8000D71
:10116000E6F054FFD5F8F40CE6F050FFD5F8E80CA3
:10117000E6F04CFFD5F8DC0CE6F048FFD5F8D00CD3
:10118000E6F044FFD5F8C40CE6F040FFD5F8B80C03
:10119000E6F03CFFD5F8AC0CE6F038FFD5F8A00C33
:1011A000E6F034FFD5F8940CE6F030FFD5F8880C63
:1011B000E6F02CFF06F168005C36F6F769FA304677
:1011C000E6F044FBD5F8580CE6F020FFD5F84C0CBF
:1011D000E6F01CFFD5F8400CE6F018FFD5F8340C0B
:1011E000E6F014FFD5F8280CE6F010FFD5F81C0C3B
:1011F000E6F00CFFD5F8100CE6F008FFD5F8040C6B
:10120000E6F004FFD5F8F80BE6F000FFD5F8EC0B9C
:10121000E6F0FCFED5F8E00BE6F0F8FE04F50B4036
:101220001830FCF7C5F92846A030F3F7F1FD04F5B6
:10123000FF40783016F04CFD04F5E1405830F3F7EC
:10124000AFFD04F5BC404030FCF782FD04F5BB4027
:101250002030F2F775F904F5B9406030F3F786F9FC
:1012600004F5B840383016F033FD04F5B640783058
:10127000F3F77CF904F5B4401830F7F725F804F5D6
:1012800050500830FCF730FF04F515503030F4F7BB
:1012900059FD04F512503030F3F7FAF904F50E5009
:1012A0001830F2F721FA04F50D500830F2F7C4F9BE
:1012B00004F5D060FAF7F6FF04F5AD60F2F714FA22
:1012C00004F58A60F2F710FA04F54E70F2F70CFAA2
:1012D00004F53C70E7F01AFA04F53470E6F0C0FE4D
:1012E00004F52E70E6F0CAFE04F52870E6F0C6FE9E
:1012F00004F51F70E6F0B4FE04F51670E6F0B0FEDB
:1013000004F50F70F6F77CFF04F50A70F6F778FF26
:1013100004F50570F6F774FF04F50070F6F770FF3A
:1013200004F5F270E6F09CFE04F5E070E6F098FE3D
:1013300004F5CE70E6F094FE04F5BC70E6F090FE85
:1013400004F5AA70E6F08CFE04F59870E6F088FECD
:1013500004F58C70E6F092FE04F58070E6F08EFEE7
:1013600004F1DC00E6F07CFE04F1C400E6F086FE49
:1013700004F19C00EAF0DEF82046F2F7E1F820469E
:1013800070BD00BF186C167010B50446FFF7CEFE96
:1013900048F63851204627F12BFB204610BD0000AF
:1013A00038B5664B00F5A04504460360D5F8F00D4E
:1013B000E6F02CFED5F8E40DE6F028FED5F8D80DC1
:1013C000E6F024FED5F8CC0DE6F020FED5F8C00DF1
:1013D000E6F01CFED5F8B40DE6F018FED5F8A80D21
:1013E000E6F014FED5F89C0DE6F010FED5F8900D51
:1013F000E6F00CFED5F8840DE6F008FED5F8780D81
:10140000E6F004FED5F86C0DE6F000FED5F8600DB0
:10141000E6F0FCFDD5F8540DE6F0F8FDD5F8480DE2
:10142000E6F0F4FDD5F83C0DE6F0F0FDD5F8300D12
:10143000E6F0ECFDD5F8240DE6F0E8FDD5F8180D42
:10144000E6F0E4FDD5F80C0DE6F0E0FDD5F8000D72
:10145000E6F0DCFDD5F8F40CE6F0D8FDD5F8E80CA4
:10146000E6F0D4FD04F592401830F3F701FD04F5E1
:101470007A502030F3F7CCFC04F53E50F3F790FCA3
:1014800004F514500830F3F7C3FC04F5115008308C
:10149000F3F76CF804F50E500830F3F7F9F804F59B
:1014A00009503030F2F720F904F5B560FAF7FAFE8A
:1014B00004F59260F2F718F904F55E70F2F714F98A
:1014C00004F51870F2F710F904F50670E7F01EF94C
:1014D00004F5FC70E6F0C4FD04F5EA70E6F0C0FD2A
:1014E00004F5D870E6F0BCFD04F5C670E6F0B8FD72
:1014F00004F5BA70E6F0C2FD04F5A870E6F0B0FDA0
:1015000004F59670E6F0ACFD04F58470E6F0A8FDF5
:1015100004F1F000E6F0B2FD04F1D400F6F770FE3D
:1015200004F1C400E6F0AAFD04F19C00EAF002F820
:101530002046F2F705F8204638BD00BFE06B167074
:1015400010B50446FFF72CFF45F6F851204627F169
:101550004FFA204610BD000038B5594B00F58C45B8
:101560000446036005F17C007035F6F791F82846D3
:1015700004F58045E6F06AF9D5F86C06E6F046FD1C
:10158000D5F86006E6F042FDD5F85406E6F03EFDDB
:10159000D5F84806E6F03AFDD5F83C06E6F036FD0B
:1015A000D5F83006E6F032FDD5F82406E6F02EFD3B
:1015B000D5F81806E6F02AFDD5F80C06E6F026FD6B
:1015C000D5F80006E6F022FDD5F8F405E6F01EFD9C
:1015D000D5F8E805E6F01AFDD5F8DC05E6F016FDCD
:1015E000D5F8D00504F58B45E6F010FD05F12C008B
:1015F0002035F6F74DF8284604F58A45E6F026F939
:1016000005F184007835F6F743F82846E6F01EF930
:1016100004F51A502830FAF75BFF04F5165028300D
:10162000F2F752F904F5145016F052FB04F50F507E
:101630002830F2F759F804F50D5016F049FB04F57F
:101640008E60FAF745FF04F56C70F2F78FFF04F532
:101650002C70F2F739F904F5027016F039FB04F535
:10166000E070E7F053F804F5D670E6F007FD04F5F6
:10167000CA70E6F003FD04F5BC70F6F7C1FD04F591
:10168000B470E6F0FBFC04F5A870E6F0F7FC04F596
:101690009A70F6F7B5FD04F58670E6F0CFFC04F11C
:1016A000E800E6F0DDFC04F1C400E6F0D9FC04F14A
:1016B0009C00E9F03FFF2046F1F742FF204638BD8D
:1016C000A86B167010B50446FFF746FF44F2986108
:1016D000204627F18DF9204610BD000070B5464B1D
:1016E00000F5E1450446036005F110000435F5F707
:1016F000CFFF284604F5E045E6F0A8F82E46D5F8D9
:101700008000E6F083FC686FE6F080FC3C36A86E53
:10171000E6F07CFC05F14800F5F7BAFF3046E6F04C
:1017200095F8A86BE6F072FCE86AE6F06FFC286AB0
:10173000E6F06CFC6869E6F069FCA868E6F066FC17
:1017400004F5DF407830E6F04FFF04F5DF407030FD
:10175000E6F04AFF04F5DF406830E6F045FF04F5A7
:10176000DF406030E6F040FF04F5DE406830E6F030
:101770005DFF04F5DE402030E6F0C8FF04F5DD40F3
:101780005830E6F0C3FF04F5DC40303016F0A0FA24
:1017900004F50550183008F0A5F804F50550083098
:1017A000FBF79CFD04F5D070F9F714FB04F5AC7061
:1017B000E6F0ACFF04F59C70E6F052FC04F5907086
:1017C000E6F05CFC04F58470E6F058FC04F1EC00F3
:1017D000F6F716FD04F1DC00E6F050FC04F1C4005D
:1017E000E6F04CFC04F19C00E9F0A4FE2046F1F781
:1017F000A7FE204670BD00BF586B167010B504469A
:10180000FFF76CFF47F2A801204627F1F1F82046C8
:1018100010BD000070B5624B00F5804504460360C2
:10182000D5F8DC0604F58B46E6F0F0FBD5F8D006DB
:10183000E6F0ECFBD5F8C406E6F0E8FBD5F8B80610
:10184000E6F0E4FBD5F8AC06E6F0E0FBD5F8A00640
:10185000E6F0DCFBD5F89406E6F0D8FBD5F8880670
:10186000E6F0D4FBD5F87C06E6F0D0FBD5F87006A0
:10187000E6F0CCFBD5F86406E6F0C8FBD5F85806D0
:10188000E6F0C4FBD5F84C06E6F0C0FBD5F8400600
:10189000E6F0BCFBD5F83406E6F0B8FBD5F8280630
:1018A000E6F0B4FB06F188007C36F5F7F1FE304631
:1018B000E5F0CCFFD5F8F80504F58B45E6F0A6FB7E
:1018C00005F154004835F5F7E3FE284604F58B454D
:1018D000E5F0BCFF05F12C002035F5F7D9FE2846D0
:1018E000E5F0B4FF04F589402030F1F7EDFF04F591
:1018F0008740783016F0ECF904F514502830FAF7E8
:10190000E7FD04F510502830F1F7DEFF04F50E5026
:1019100016F0DEF904F509502830F1F7E5FE04F57C
:101920006670FAF7D5FD04F55270F1F785FE04F5FF
:10193000287016F0CDF904F5F070F2F717FE04F5F3
:10194000CC70E6F0E3FE04F5C270F6F759FC04F53E
:10195000BA70E6F093FB04F5AE70E6F08FFB04F589
:10196000A270E6F08BFB04F59670E6F087FB04F5B9
:101970008870F6F745FC04F1F400E6F071FB04F121
:10198000DC00E6F07BFB04F1C400E6F077FB04F139
:101990009C00E9F0CFFD2046F1F7D2FD204670BD56
:1019A000206B167010B50446FFF734FF44F2E06177
:1019B000204627F11DF8204610BD000038B5244B05
:1019C00000F5005504460360D5F86C02E6F01EFBF6
:1019D000D5F86002E6F01AFBD5F85402E6F016FBE3
:1019E000D5F84802E6F012FBD5F83C02E6F00EFB13
:1019F00004F508502830E6F0F7FD04F505502830CE
:101A0000F2F7B4FD04F5035016F062F904F5F8702E
:101A1000FAF75EFD04F5A47016F05AF904F580702B
:101A2000E6F074FE04F1EC00F6F7EAFB04F1DC00EA
:101A3000E6F024FB04F1C400E6F020FB04F19C0076
:101A4000E9F078FD2046F1F77BFD204638BD00BF68
:101A5000E86A167010B50446FFF7B0FF42F2702135
:101A6000204626F1C5FF204610BD000038B5624B68
:101A700000F5E04504460360D5F88409E6F0C6FAAF
:101A8000D5F87809E6F0C2FAD5F86C09E6F0BEFAA6
:101A9000D5F86009E6F0BAFAD5F85409E6F0B6FAD6
:101AA000D5F84809E6F0B2FAD5F83C09E6F0AEFA06
:101AB000D5F83009E6F0AAFAD5F82409E6F0A6FA36
:101AC000D5F81809E6F0A2FAD5F80C09E6F09EFA66
:101AD000D5F80009E6F09AFAD5F8F408E6F096FA97
:101AE000D5F8E808E6F092FAD5F8DC08E6F08EFAC8
:101AF000D5F8D008E6F08AFAD5F8C408E6F086FAF8
:101B0000D5F8B808E6F082FAD5F8AC08E6F07EFA27
:101B1000D5F8A008E6F07AFA04F5B1407030F9F78C
:101B200059F904F5B040483016F0D2F804F5625087
:101B30002030F9F74FF904F55F50383016F0C8F847
:101B400004F55C503830F2F711FD04F558502030A0
:101B5000F1F7CAFD04F540502030FBF74DFE04F5C7
:101B600028502030FBF748FE04F510502030FBF7DA
:101B700043FE04F50D502030F2F7F8FC04F50A504E
:101B8000383016F0A5F804F54470F9F723F904F598
:101B90001C70F1F7D5FC04F5E47016F099F804F523
:101BA000C070E6F0B3FD04F5B470F6F729FB04F558
:101BB000AC70E6F063FA04F5A070E6F05FFA04F5A5
:101BC0008E70E6F04DFA04F58070F6F719FB04F11B
:101BD000EC00F6F715FB04F1DC00E6F04FFA04F137
:101BE000C400E6F04BFA04F19C00E9F0A3FC2046A7
:101BF000F1F7A6FC204638BD746A167010B504468D
:101C0000FFF734FF47F68811204626F1F1FE204603
:101C100010BD000070B5A94B00F5204504460360D7
:101C2000D5F8DC0304F52246E6F0F0F9D5F8D00348
:101C3000E6F0ECF9D5F8C403E6F0E8F9D5F8B80316
:101C4000E6F0E4F9D5F8AC03E6F0E0F9D5F8A00346
:101C5000E6F0DCF9D5F89403E6F0D8F9D5F8880376
:101C6000E6F0D4F9D5F87C03E6F0D0F9D5F87003A6
:101C7000E6F0CCF9D5F86403E6F0C8F9D5F85803D6
:101C8000E6F0C4F9D5F84C03E6F0C0F9D5F8400306
:101C9000E6F0BCF9D5F83403E6F0B8F9D5F8280336
:101CA000E6F0B4F9D5F81C03E6F0B0F9D5F8100366
:101CB000E6F0ACF9D5F80403E6F0A8F9D5F8F80297
:101CC000E6F0A4F906F1D800CC36F5F7E1FC304691
:101CD000E5F0BCFDD5F8C802E6F098F9D5F8BC02ED
:101CE000E6F094F9D5F8B002E6F090F9D5F8A40240
:101CF000E6F08CF9D5F89802E6F088F9D5F88C0270
:101D0000E6F084F9D5F88002E6F080F9D5F874029F
:101D1000E6F07CF9D5F86802E6F078F9D5F85C02CF
:101D2000E6F074F9D5F85002E6F070F9D5F84402FF
:101D3000E6F06CF9D5F83802E6F068F9D5F82C022F
:101D4000E6F064F9D5F8200204F52145E6F05EF9E5
:101D500005F1FC00F035F5F79BFC284604F521451C
:101D6000E5F074FD05F1D400C835F5F791FC28467F
:101D7000E5F06CFD04F52140C030E6F035FC04F5DB
:101D80000240F030FAF7A4FB04F50240483015F0A9
:101D90009FFF04F5E7403030F3F7D4FF04F5E64049
:101DA000083015F095FF04F5E440603015F090FF21
:101DB00004F5E1401830F1F7C5FD04F5C44050309A
:101DC000F3F764FF04F5A8400830F3F75FFF04F56C
:101DD00051502030F8F7FEFF04F5AC501030FAF700
:101DE00077FB04F5AA50F1F727FC04F5A45018304E
:101DF00015F06EFF04F59F501830F1F7A1FB04F5C4
:101E000099501830F2F7B2FB04F58360F2F7C8FF7F
:101E100004F54070F1F768FC04F52E70E6F076FCEE
:101E200004F52470E6F00AF904F51D70F6F7E8F9F8
:101E300004F51670E6F014F904F51070E6F01EF9DA
:101E400004F50A70E6F01AF904F50170E6F008F9F5
:101E500004F5F070E6F004F904F5E270F6F7D0F955
:101E600004F5D870F6F7CCF904F5CA70E6F0F8F886
:101E700004F5BC70F6F7C4F904F5B270F6F7C0F9D2
:101E800004F5A470E6F0ECF804F59270E6F0E8F8DA
:101E900004F58070E6F0E4F804F1E800E6F0EEF80E
:101EA00004F1C400E6F0DCF804F19C00E9F042FB28
:101EB0002046F1F745FB204670BD00BF8C691670C7
:101EC00010B50446FFF7A6FE4AF2E031204626F19F
:101ED0008FFD204610BD000038B53C4B00F5E045B5
:101EE0000446036005F134002835F5F7D1FB284698
:101EF00004F5E045E5F0AAFC05F110000435F5F71E
:101F0000C7FB284604F5C045E5F0A0FC04F5E04316
:101F10001868E6F07BF8D5F8F40FE6F077F8D5F816
:101F2000E80FE6F073F8D5F8DC0FE6F06FF8D5F8B7
:101F3000D00FE6F06BF804F5DF404030E6F054FBDC
:101F400004F5DE404830E6F071FB04F5DE40E6F0D3
:101F5000DDFB04F5DD403830E6F0D8FB04F5DC406D
:101F6000103015F0B5FE04F50550183007F0ECFD03
:101F700004F505500830FBF703FA04F5D070F8F7C4
:101F800029FF04F5AC70E6F0C1FB04F5A270E6F0A1
:101F900075F804F59470F6F733F904F58C70E6F0F3
:101FA0006DF804F58070E6F069F804F1E800E6F0F9
:101FB00065F804F1C400E6F053F804F19C00E9F080
:101FC000B9FA2046F1F7BCFA204638BD3C691670D4
:101FD00010B50446FFF780FF47F25001204626F176
:101FE00007FD204610BD0000F8B500F5E825FD4BC3
:101FF00004460360D5F8B00B04F5E926E6F006F8D0
:10200000D5F8A40BE6F002F8D5F8980BE5F0FEFF42
:10201000D5F88C0BE5F0FAFFD5F8800BE5F0F6FF6C
:10202000D5F8740BE5F0F2FFD5F8680BE5F0EEFF9C
:10203000D5F85C0BE5F0EAFFD5F8500BE5F0E6FFCC
:10204000D5F8440BE5F0E2FFD5F8380BE5F0DEFFFC
:10205000D5F82C0BE5F0DAFFD5F8200BE5F0D6FF2C
:10206000D5F8140BE5F0D2FFD5F8080BE5F0CEFF5C
:10207000D5F8FC0AE5F0CAFF06F53177D5F8F00A85
:10208000E5F0C4FF06F53470F5F702FB3846E5F0DD
:10209000DDFBD5F8C00AE5F0B9FFD5F8B40AE5F0E4
:1020A000B5FFD5F8A80AE5F0B1FFD5F89C0AE5F030
:1020B000ADFFD5F8900AE5F0A9FFD5F8840AE5F060
:1020C000A5FFD5F8780AE5F0A1FFD5F86C0AE5F090
:1020D0009DFFD5F8600AE5F099FFD5F8540AE5F0C0
:1020E00095FFD5F8480AE5F091FFD5F83C0AE5F0F0
:1020F0008DFFD5F8300AE5F089FFD5F8240AE5F020
:1021000085FFD5F8180AE5F081FFD5F80C0AE5F04F
:102110007DFFD5F8000AE5F079FFD5F8F409E5F080
:1021200075FF06F5DE77D5F8E809E5F06FFF06F5EF
:10213000E470F5F7ADFA384606F5CC77E5F086FBA6
:1021400006F5D270F5F7A4FA384606F5BA77E5F049
:102150007DFB06F5C070F5F79BFA3846E5F076FB97
:10216000D5F87009E5F052FFD5F86409E5F04EFFA7
:10217000D5F85809E5F04AFFD5F84C0906F59075F1
:10218000E5F044FF06F59670F5F782FA2846E5F08B
:102190005DFB06F58C70E6F027FA06F1D000E6F05C
:1021A000B5FA04F5DB2004F59F258030FFF794FE97
:1021B00004F5C62000F59460FFF72CFD04F5C2205D
:1021C00000F50C70FFF7FAFB04F5B42000F5CE60C3
:1021D000FDF740F804F5AA2000F5BC70FCF780F884
:1021E00005F58A60FBF7EAFF05F5E870F1F7B6FE42
:1021F00004F59A2004F54C3500F5EC60FFF7DEFBA2
:1022000004F5962000F59E60FFF7D8FB04F59420B6
:1022100000F5EA60F3F7CAFD04F5852000F5B96022
:10222000FFF724FC04F5812000F55670FFF7C6FB8C
:1022300004F57A30E830FFF7C1FB04F5683000F5AB
:102240000270FFF7E7FA05F5B070FFF747FA05F1FE
:10225000A000F2F78BF904F53A3000F50270FFF7B1
:102260007BF904F523301030FFF79AF804F520309D
:1022700000F51670FBF734F904F5FA3000F59070AC
:10228000FEF754FF04F5F53000F5C870F6F784FD4D
:1022900004F5F43000F5FC70F1F790FE04F5C93058
:1022A00000F5D870FEF78AFE04F5B03000F5C8706E
:1022B000FBF7CEFB04F59E3000F5BC70FEF748FE40
:1022C00004F53F405830FEF731FD04F53E40B8308C
:1022D000F1F736F904F5E2405830FEF769FC04F5F1
:1022E0009A405830FEF7F2FB04F5D760FEF72AFB60
:1022F00004F5CE60E6F00AFA04F25C60E5F0BEFE9A
:1023000004F5C860F5F77CFF04F5C660E5F0B6FE9D
:1023100004F5C360E5F0B2FE04F5C060E5F0AEFE82
:1023200004F5BD60E5F0AAFE04F5BA60E5F0A6FE8E
:1023300004F2B450F5F764FF04F2A450E5F09EFEF9
:1023400004F5B160F5F75CFF04F5AF60E5F096FECB
:1023500004F5AC60E5F092FE04F24450F5F750FF4E
:1023600004F23450E5F08AFE04F21C50E5F086FEDB
:1023700004F20450E5F082FE04F59C60E5F070FE86
:1023800004F59960E5F07AFE04F2A440E5F068FEF9
:1023900004F59060E5F064FE04F58D60E5F06EFEF6
:1023A00004F58A60E5F06AFE04F58760E5F066FEF4
:1023B00004F58460E5F062FE04F20440F5F720FFC6
:1023C00004F57D70E5F05AFE04F57770E5F056FEF1
:1023D00004F57170E5F052FE04F56B70E5F04EFE09
:1023E00002E000BF0469167004F56570E5F046FE72
:1023F00004F55F70E5F042FE04F55970E5F03EFE2D
:1024000004F55370E5F03AFE04F54D70E5F036FE44
:1024100004F54770E5F032FE04F54170E5F02EFE5C
:1024200004F53B70E5F02AFE04F53570E5F026FE74
:1024300004F52F70E5F022FE04F52970E5F01EFE8C
:1024400004F52370E5F01AFE04F51D70E5F016FEA4
:1024500004F51770E5F012FE04F51170E5F00EFEBC
:1024600004F50B70E5F00AFE04F50570E5F006FED4
:1024700004F5FE70E5F002FE04F5F270E5F0FEFDF5
:1024800004F5E670E5F0FAFD04F5DA70E5F0F6FD26
:1024900004F5CE70E5F0F2FD04F5C270E5F0EEFD56
:1024A00004F5B670E5F0EAFD04F5AA70E5F0E6FD86
:1024B00004F59E70E5F0E2FD04F59270E5F0DEFDB6
:1024C00004F58670E5F0DAFD04F1F400E5F0D6FDE0
:1024D00004F1DC00E5F0D2FD04F1C400E5F0CEFD2E
:1024E00004F19C00E9F026F82046F1F729F820468F
:1024F000F8BD00BF10B50446FFF776FD024920463F
:1025000026F176FA204610BDB84B070038B54B4B84
:1025100000F5304504460360D5F84808E5F076FD3F
:10252000D5F83C08E5F072FDD5F83008E5F06EFD11
:10253000D5F82408E5F06AFDD5F81808E5F066FD41
:10254000D5F80C08E5F062FDD5F80008E5F05EFD71
:10255000D5F8F407E5F05AFDD5F8E807E5F056FDA3
:10256000D5F8DC07E5F052FDD5F8D007E5F04EFDD3
:1025700004F537408030E6F0C9F804F537400830FC
:10258000E6F054F804F536409030E6F04FF804F5E4
:1025900036404830E6F0BAF804F53640E6F0B6F8D2
:1025A00004F53540B830E6F0B1F804F52740703056
:1025B000F3F76CFB04F52640C83015F089FB04F5F1
:1025C0002640203015F084FB04F52540783015F0C6
:1025D0007FFB04F5085007F01DFB04F50550F1F7EB
:1025E000C5FF04F504502830FAF7E4FE04F5045062
:1025F0001430F5F705FE04F504500430E5F03EFD17
:1026000004F503502C30E5F039FD04F5035010308B
:10261000F5F7F6FD04F502503430E5F021FD04F540
:1026200002501030E5F01CFD04F501503430F5F790
:10263000E7FD2046F8F7A0FA204638BDA4681670DA
:1026400010B50446FFF762FF4BF65001204626F115
:10265000CFF9204610BD000038B54E4B00F520459F
:1026600004460360D5F8140DE5F0D0FCD5F8080D4C
:10267000E5F0CCFCD5F8FC0CE5F0C8FCD5F8F00C86
:10268000E5F0C4FCD5F8E40CE5F0C0FCD5F8D80CB6
:10269000E5F0BCFCD5F8CC0CE5F0B8FCD5F8C00CE6
:1026A000E5F0B4FCD5F8B40CE5F0B0FCD5F8A80C16
:1026B000E5F0ACFCD5F89C0CE5F0A8FCD5F8900C46
:1026C00004F52C45E5F0A2FC05F170006435F4F743
:1026D000DFFF2846E5F0BAF804F52C404830E5F075
:1026E000DEFF04F52C40E6F011F804F52B408830AD
:1026F000E5F09CFF04F52B404030E6F007F804F5C8
:102700002A40F830E6F002F804F52A40B030E5F04F
:10271000FDFF04F51550183007F0E2FA04F51250E9
:10272000303015F0D5FA04F512501830F2F700FCED
:1027300004F50F501830F1F719FF04F50D5008306B
:10274000F0F75EFF04F50A50203015F0C1FA04F5E9
:102750000650F1F701F804F503502030F0F7F0FED1
:1027600004F503500C30E5F089FC04F502503430D8
:10277000E5F084FC04F502501030E5F071FC04F53E
:1027800001503430F5F73CFD2046F8F7F5F92046C6
:1027900038BD00BF6C68167010B50446FFF75CFFCB
:1027A0004AF61851204626F123F9204610BD0000B4
:1027B00038B5704B00F5704504460360D5F80C023F
:1027C000E5F024FCD5F80002E5F020FCD5F8F40192
:1027D000E5F01CFCD5F8E801E5F018FCD5F8DC01C3
:1027E000E5F014FCD5F8D001E5F010FCD5F8C401F3
:1027F000E5F00CFCD5F8B801E5F008FCD5F8AC0123
:10280000E5F004FCD5F8A001E5F000FCD5F8940152
:10281000E5F0FCFBD5F88801E5F0F8FBD5F87C0184
:10282000E5F0F4FBD5F87001E5F0F0FBD5F86401B4
:10283000E5F0ECFBD5F85801E5F0E8FBD5F84C01E4
:10284000E5F0E4FBD5F84001E5F0E0FB2846F03088
:10285000E5F05CFF04F55E405830FBF779FA04F5CB
:102860004B40C030FBF774FA04F539402830FBF7D1
:102870006FFA04F526409030FBF76AFA04F525401C
:10288000E83015F025FA04F513405030FBF760FAF4
:1028900004F51140F030F5F717FD04F5FE4058300F
:1028A000FBF756FA04F5D9404030FBF751FA04F52E
:1028B000D840F1F75BFE04F5B2406830FBF748FA08
:1028C00004F58D405030FBF743FA04F55050383092
:1028D000FBF73EFA04F506502030FBF739FA04F511
:1028E00006500830F5F78CFC04F505502C30E5F067
:1028F000B7FB04F505501030F5F782FC04F50450E1
:102900003C30F5F77DFC04F504502830F5F778FCF1
:1029100004F504501430F5F773FC04F50450F5F792
:102920006FFC04F503502C30F5F76AFC04F50350F6
:102930001830F5F765FC04F503500430F5F760FC3A
:1029400004F502503030F5F75BFC04F502501C3002
:10295000F5F756FC04F502500830F5F751FC04F584
:1029600001503430F5F74CFC2046F8F705F92046C5
:1029700038BD00BF3468167010B50446FFF718FF65
:102980004FF21021204626F133F8204610BD0000FA
:1029900038B5194B00F5005504460360D5F8880892
:1029A000E5F034FBD5F87C08E5F030FBD5F870088D
:1029B000E5F02CFBD5F86408E5F028FB04F5205081
:1029C0001030E5F0A3FE04F51D501030F1F7CEFDF8
:1029D00004F504503030F1F755FB04F5025008308F
:1029E00015F076F904F501503430F5F709FC20466E
:1029F000F8F7C2F8204638BDFC67167010B50446DB
:102A0000FFF7C6FF42F69001204625F1F1FF204670
:102A100010BD000038B5344B00F500450446036096
:102A2000D5F8EC0CE5F0F2FAD5F8E00CE5F0EEFAAA
:102A3000D5F8D40CE5F0EAFAD5F8C80CE5F0E6FADA
:102A4000D5F8BC0CE5F0E2FAD5F8B00CE5F0DEFA0A
:102A500004F50C406030E5F059FE04F50B40B83049
:102A600015F036F904F5F2402030FBF771F904F562
:102A7000CD400830FBF76CF904F5A7407030FBF748
:102A800067F904F582405830FBF762F904F5065007
:102A90003030F8F79FF904F503503030F1F766FD58
:102AA00004F503501830F5F7ABFB04F50350043080
:102AB000F5F7A6FB04F502503030F5F7A1FB04F55D
:102AC00002501C30F5F79CFB04F502500830F5F776
:102AD00097FB04F501503430F5F792FB2046F8F7E8
:102AE0004BF8204638BD00BFC467167010B50446C9
:102AF000FFF790FF48F6F041204625F179FF204688
:102B000010BD000070B5394B00F5804504460360E8
:102B1000D5F89C0704F58E46E5F078FAD5F89007CD
:102B2000E5F074FAD5F88407E5F070FAD5F878077F
:102B3000E5F06CFAD5F86C07E5F068FAD5F86007AF
:102B4000E5F064FA06F140003436F4F7A1FD3046B2
:102B5000E4F07CFED5F83007E5F058FAD5F8240704
:102B6000E5F054FAD5F81807E5F050FAD5F80C0757
:102B7000E5F04CFAD5F80007E5F048FA04F58D4089
:102B80003030E5F0C3FD04F581401030F1F77AFAFA
:102B900004F569503030F1F775FA04F551501030F2
:102BA000F1F770FA04F538503030F1F76BFA04F5AC
:102BB00020501030F1F766FA04F507503030F1F785
:102BC00061FA04F50550083015F082F804F502505A
:102BD0000830FAF701FD04F501503430F5F710FB29
:102BE0002046F7F7C9FF204670BD00BF506716703A
:102BF00010B50446FFF786FF44F2A071204625F188
:102C0000F7FE204610BD000038B53F4B00F580456B
:102C100004460360D5F8640DE5F0F8F9D5F8580DD1
:102C2000E5F0F4F9D5F84C0DE5F0F0F9D5F8400DE4
:102C3000E5F0ECF9D5F8340DE5F0E8F9D5F8280D14
:102C4000E5F0E4F9D5F81C0DE5F0E0F9D5F8100D44
:102C5000E5F0DCF9D5F8040DE5F0D8F9D5F8F80C75
:102C6000E5F0D4F9D5F8EC0CE5F0D0F9D5F8E00CA6
:102C7000E5F0CCF9D5F8D40CE5F0C8F904F59940A5
:102C80002030E8F057FC04F598405830E5F03EFD60
:102C900004F59740303015F01BF804F58B401030E8
:102CA000F1F7F0F904F57D503030F1F7EBF904F568
:102CB00065501030F1F7E6F904F54C503030F1F77B
:102CC000E1F904F549503030F1F750FC04F50450B7
:102CD0000830FAF7B1FC04F502503030F4F7F2FC9A
:102CE00004F502501C30F5F78BFA04F50250083059
:102CF000F5F786FA04F501503430F5F781FA2046ED
:102D0000F7F73AFF204638BDA066167010B50446A6
:102D1000FFF77AFF44F66851204625F169FE204608
:102D200010BD000038B5514B00F5804504460360E6
:102D3000D5F8AC07E5F06AF9D5F8A007E5F066F933
:102D4000D5F89407E5F062F9D5F88807E5F05EF963
:102D5000D5F87C07E5F05AF9D5F87007E5F056F993
:102D6000D5F86407E5F052F9D5F85807E5F04EF9C3
:102D7000D5F84C07E5F04AF9D5F84007E5F046F9F3
:102D8000D5F83407E5F042F9D5F82807E5F03EF923
:102D9000D5F81C07E5F03AF9D5F81007E5F036F953
:102DA000D5F80407E5F032F9D5F8F806E5F02EF984
:102DB000D5F8EC06E5F02AF9D5F8E00604F58D45DE
:102DC000E5F024F905F13C003035F4F761FC2846C4
:102DD000E4F03CFD04F58C406830E5F097FC04F528
:102DE0008A406830F0F770FD04F587402030F0F736
:102DF000A9FD04F585406030F1F7B8FB04F51050EB
:102E00001030F9F765FB04F50C501030F0F75CFD5D
:102E100004F509501030F1F7A9FB04F506502830ED
:102E200014F056FF04F503502830F1F79FFB04F52A
:102E300003501430E5F022F904F502503C30E5F07F
:102E40001DF904F502502030F5F7DAF904F50250C7
:102E50000C30F5F7D5F904F501503C30E5F00EF9EA
:102E60002046F7F789FE204638BD00BF6866167019
:102E700010B50446FFF756FF44F2B071204625F125
:102E8000B7FD204610BD000038B5464B00F5C045E3
:102E900004460360D5F8680FE5F0B8F8D5F85C0F84
:102EA000E5F0B4F8D5F8500FE5F0B0F8D5F8440FD8
:102EB000E5F0ACF8D5F8380FE5F0A8F8D5F82C0F08
:102EC000E5F0A4F8D5F8200FE5F0A0F8D5F8140F38
:102ED000E5F09CF8D5F8080FE5F098F804F5CA403D
:102EE0007030F5F759FF04F5AB405030FAF780FE2B
:102EF00004F58C403030FAF77BFE04F55A50103060
:102F0000FAF776FE04F557501030F1F72FFB04F571
:102F100018503030FAF76CFE04F5B4501030FAF760
:102F200067FE04F5DE60FAF763FE04F5C660F1F7AC
:102F30001DFB04F5AE60F1F7ABFB04F51C70F2F776
:102F40008FFB04F5D870F1F711FB04F5B470E5F0D0
:102F5000DDFB04F5A870F5F753F904F59E70F5F75D
:102F60004FF904F59470F5F74BF904F58A70F5F70D
:102F700047F904F58070F5F743F904F1EC00F5F733
:102F80003FF904F1DC00E5F079F804F1C400E5F064
:102F900075F804F19C00E8F0CDFA2046F0F7D0FA7D
:102FA000204638BDF065167010B50446FFF76CFF7B
:102FB00046F67071204625F11BFD204610BD00002D
:102FC00070B5ED4B00F5604405460360D4F8A408E5
:102FD00005F56746E5F01AF8D4F89808E5F016F814
:102FE000D4F88C08E5F012F8D4F88008E5F00EF873
:102FF000D4F87408E5F00AF8D4F86808E5F006F8A3
:10300000D4F85C08E5F002F8D4F85008E4F0FEFFCC
:10301000D4F84408E4F0FAFFD4F83808E4F0F6FFF6
:10302000D4F82C08E4F0F2FFD4F82008E4F0EEFF26
:10303000D4F81408E4F0EAFFD4F80808E4F0E6FF56
:1030400006F1E800DC36F4F723FB3046E4F0FEFB43
:10305000D4F8D807E4F0DAFFD4F8CC07E4F0D6FFD0
:10306000D4F8C007E4F0D2FFD4F8B407E4F0CEFF00
:10307000D4F8A807E4F0CAFFD4F89C07E4F0C6FF30
:10308000D4F89007E4F0C2FFD4F88407E4F0BEFF60
:10309000D4F87807E4F0BAFFD4F86C07E4F0B6FF90
:1030A000D4F86007E4F0B2FFD4F85407E4F0AEFFC0
:1030B000D4F84807E4F0AAFFD4F83C07E4F0A6FFF0
:1030C000D4F83007E4F0A2FFD4F82407E4F09EFF20
:1030D000D4F81807E4F09AFFD4F80C07E4F096FF50
:1030E000D4F80007E4F092FFD4F8F406E4F08EFF81
:1030F000D4F8E806E4F08AFFD4F8DC06E4F086FFB2
:10310000D4F8D006E4F082FFD4F8C406E4F07EFFE1
:10311000D4F8B806E4F07AFFD4F8AC06E4F076FF11
:10312000D4F8A006E4F072FFD4F89406E4F06EFF41
:10313000D4F88806E4F06AFFD4F87C06E4F066FF71
:10314000D4F87006E4F062FFD4F86406E4F05EFFA1
:10315000D4F85806E4F05AFFD4F84C06E4F056FFD1
:10316000D4F84006E4F052FFD4F83406E4F04EFF01
:10317000D4F82806E4F04AFFD4F81C06E4F046FF31
:10318000D4F81006E4F042FFD4F80406E4F03EFF61
:10319000D4F8F805E4F03AFFD4F8EC05E4F036FF93
:1031A000D4F8E005E4F032FFD4F8D405E4F02EFFC3
:1031B000D4F8C805E4F02AFFD4F8BC05E4F026FFF3
:1031C000D4F8B005E4F022FFD4F8A405E4F01EFF23
:1031D000D4F89805E4F01AFFD4F88C05E4F016FF53
:1031E000D4F88005E4F012FFD4F87405E4F00EFF83
:1031F000D4F86805E4F00AFFD4F85C05E4F006FFB3
:10320000D4F85005E4F002FF05F56540E5F07EFADC
:1032100005F55E40E030F0F735FF05F55840C03069
:10322000F0F730FF05F55240A030F0F72BFF05F521
:103230004C408030F0F726FF05F546406030F0F74F
:1032400021FF05F540404030F0F71CFF05F53A40FE
:103250002030F0F717FF05F53440F0F713FF05F5C0
:103260002D40E030F0F70EFF05F52740C030F0F7B5
:1032700009FF05F52140A030F0F704FF05F51B40DC
:10328000F830F2F765F905F51B40503014F020FDD9
:1032900005F51A409030F1F769F905F514407030E2
:1032A000F0F7F0FE05F50E405030F0F7EBFE05F5B7
:1032B00008403030F0F7E6FE05F502401030F0F738
:1032C000E1FE05F5F7407030F0F7DCFE05F5EB4068
:1032D0005030F0F7D7FE05F5DF403030F0F7D2FE82
:1032E00005F5D3401030F0F7CDFE05F5C64070303F
:1032F000F0F7C8FE05F5BB404830F2F729F905F5AF
:10330000AF402830F0F7BEFE05F5A3400830F0F7D7
:10331000B9FE05F596406830F0F7B4FE05F58A4031
:103320004830F0F7AFFE05F57C502830F0F7AAFEE4
:1033300005F564500830F0F7A5FE05F54B50283030
:10334000F0F7A0FE05F533500830F0F79BFE05F5C9
:103350001A502830F0F796FE05F502500830F0F7C5
:1033600091FE05F501503430F4F74AFF2846F7F78F
:1033700003FC284670BD00BFB865167010B5044642
:10338000FFF71EFE4EF6A801204625F131FB204630
:1033900010BD000038B5294B00F5C0450446036058
:1033A000D5F84401E4F032FED5F83801E4F02EFE01
:1033B000D5F82C01E4F02AFED5F82001E4F026FE31
:1033C000D5F81401E4F022FED5F8080104F5C14552
:1033D000E4F01CFE05F164005835F4F759F928466D
:1033E000E4F034FA04F5C1401030E5F08FF904F54B
:1033F000BF405030F1F7BAF804F58240F9F768F8A9
:1034000004F505501830F7F7E5FC04F502503030AC
:1034100014F05EFC04F502501C30F4F7F1FE04F5E4
:1034200002500830F4F7ECFE04F501503430F4F7A4
:10343000E7FE2046F7F7A0FB204638BD486516702A
:1034400010B50446FFF7A6FF46F24811204625F1C5
:10345000CFFA204610BD000038B5804B00F58055EE
:1034600004460360D5F8100DE4F0D0FDD5F8040D46
:10347000E4F0CCFDD5F8F80CE4F0C8FDD5F8EC0C80
:10348000E4F0C4FDD5F8E00CE4F0C0FDD5F8D40CB0
:10349000E4F0BCFDD5F8C80CE4F0B8FDD5F8BC0CE0
:1034A000E4F0B4FDD5F8B00CE4F0B0FDD5F8A40C10
:1034B000E4F0ACFDD5F8980CE4F0A8FDD5F88C0C40
:1034C000E4F0A4FDD5F8800CE4F0A0FDD5F8740C70
:1034D000E4F09CFDD5F8680CE4F098FDD5F85C0CA0
:1034E000E4F094FDD5F8500CE4F090FDD5F8440CD0
:1034F000E4F08CFDD5F8380CE4F088FD04F5DE50DE
:103500001030E5F003F904F5DA501830E5F08EF8E4
:1035100004F5D8501030E5F0F9F804F5D45018301F
:10352000E5F084F804F5D150E5F080F804F5CD50CD
:103530000830E5F07BF804F5CD50E4F0C7FD04F564
:10354000CC501C30E4F0C2FD04F5CC501830E4F04F
:10355000BDFD04F5C750103014F0BAFB04F5C2509D
:10356000083014F0B5FB04F5BD500830EFF7E8FF64
:1035700004F5B2500830F4F7A7FE04F5A95008305E
:10358000F0F7EAF804F59E500830F4F79DFE04F5D4
:1035900095500830F0F7E0F804F590500830EFF758
:1035A000CFFF04F5AC60FAF725FF04F5976014F03F
:1035B0008FFB04F5826014F08BFB04F57D70E4F062
:1035C0004FFD04F57470E4F04BFD04F56B70E4F00E
:1035D00047FD04F56570E4F051FD04F55E70F4F705
:1035E0000FFE04F55A70E4F049FD04F55170E4F063
:1035F00037FD04F54870E4F033FD04F53F70E4F066
:103600002FFD04F53670E4F02BFD04F53070E4F086
:1036100035FD04F52A70E4F031FD04F52170E4F085
:103620001FFD04F51870E4F01BFD04F51170F4F7AC
:10363000E7FD04F50A70E4F013FD04F50170E4F011
:103640000FFD04F5F070E4F00BFD04F5E270F4F703
:10365000D7FD2046F0F7DAFC204638BDC06316706F
:1036600010B50446FFF7F8FE41F61851204625F143
:10367000BFF9204610BD0000174B10B5044603608B
:1036800000F5AD501C30E4F021FD04F5AD501830CC
:10369000E4F01CFD04F5A7501830F0F7F9FF04F62C
:1036A0009830FAF76FFF04F50E70FAF76BFF04F528
:1036B0000870F4F7A5FD04F50370F4F7A1FD04F517
:1036C000F870E4F0CDFC04F5E670E4F0C9FC2046A7
:1036D000F0F79CFC204610BD5063167010B50446F0
:1036E000FFF7CAFF41F2D851204625F181F9204663
:1036F00010BD000038B5644B00F52045044603605A
:10370000D5F84C0AE4F082FCD5F8400AE4F07EFCDF
:10371000D5F8340AE4F07AFCD5F8280AE4F076FC0F
:10372000D5F81C0AE4F072FCD5F8100AE4F06EFC3F
:10373000D5F8040AE4F06AFCD5F8F809E4F066FC70
:10374000D5F8EC09E4F062FCD5F8E009E4F05EFCA1
:10375000D5F8D409E4F05AFCD5F8C809E4F056FCD1
:10376000D5F8BC09E4F052FCD5F8B009E4F04EFC01
:10377000D5F8A409E4F04AFCD5F89809E4F046FC31
:10378000D5F88C09E4F042FCD5F8800904F5294508
:10379000E4F03CFC05F15C005035F3F779FF284676
:1037A00004F52945E4F052F805F134002835F3F723
:1037B0006FFF2846E4F04AF804F52840E030E4F0D2
:1037C000A5FF04F509403830F7F704FB04F5034082
:1037D0009030F1F7BDFE04F50240E83014F078FABD
:1037E00004F502402830F0F7C1FE04F5F940F1F786
:1037F000AFFE04F5BE406830FFF72EFE04F593409F
:103800001030FFF739FF04F587406830F1F7A0FE6C
:1038100004F51B501030FFF71FFE04F5045028304C
:10382000F1F796FE04F504501430F4F7E9FC04F5C2
:103830000450F4F7E5FC04F503502C30F4F7E0FCF9
:1038400004F503501830F4F7DBFC04F503500430A2
:10385000F4F7D6FC04F502503030F4F7D1FC04F54F
:1038600002501C30F4F7CCFC04F502500830F4F799
:10387000C7FC04F501503430F4F7C2FC2046F7F7DA
:103880007BF9204638BD00BF1863167010B504469A
:10389000FFF730FF4AF65021204625F1A9F82046CF
:1038A00010BD000038B500F52434FD4B054603601B
:1038B000D4F8D409E4F0AAFBD4F8C809E4F0A6FBD4
:1038C000D4F8BC09E4F0A2FBD4F8B009E4F09EFB04
:1038D000D4F8A409E4F09AFBD4F89809E4F096FB34
:1038E000D4F88C09E4F092FBD4F88009E4F08EFB64
:1038F000D4F87409E4F08AFBD4F86809E4F086FB94
:10390000D4F85C09E4F082FBD4F85009E4F07EFBC3
:10391000D4F84409E4F07AFBD4F83809E4F076FBF3
:10392000D4F82C09E4F072FBD4F82009E4F06EFB23
:10393000D4F81409E4F06AFBD4F80809E4F066FB53
:10394000D4F8FC08E4F062FBD4F8F008E4F05EFB85
:10395000D4F8E408E4F05AFBD4F8D808E4F056FBB5
:10396000D4F8CC08E4F052FBD4F8C008E4F04EFBE5
:10397000D4F8B408E4F04AFBD4F8A808E4F046FB15
:10398000D4F89C08E4F042FBD4F89008E4F03EFB45
:10399000D4F88408E4F03AFBD4F87808E4F036FB75
:1039A000D4F86C08E4F032FBD4F86008E4F02EFBA5
:1039B000D4F85408E4F02AFBD4F84808E4F026FBD5
:1039C000D4F83C08E4F022FBD4F83008E4F01EFB05
